:020000040800F2
:1000000000800020512D0008A50A0008310B0008CF
:10001000330B0008350B0008370B00080000000008
:10002000000000000000000000000000390B000884
:100030003B0B0008000000003D0B00083F0B0008D0
:10004000A12D0008A12D0008A12D0008A12D000858
:10005000A12D0008A12D0008A12D0008A12D000848
:10006000A12D0008A12D0008A12D0008A12D000838
:10007000A12D0008A12D0008A12D0008A12D000828
:10008000A12D0008A12D0008A12D0008A12D000818
:1000900000000000A12D0008A12D0008A12D0008DE
:1000A000A12D0008A12D0008A12D0008A12D0008F8
:1000B000A12D0008A12D0008A12D0008A12D0008E8
:1000C000A12D0008A12D0008A12D0008A12D0008D8
:1000D000A12D0008A12D0008A12D0008A12D0008C8
:1000E000A12D0008A12D0008A12D0008A12D0008B8
:1000F000A12D00080000000000000000A12D000854
:10010000A12D0008A12D0008A12D0008A12D000897
:10011000A12D0008A12D0008A12D0008A12D000887
:10012000A12D0008A12D0008A12D0008A12D000877
:10013000A12D0008A12D000810B5054C237833B976
:10014000044B13B10448AFF300800123237010BDAA
:100150001000002000000000F82D000808B5034B37
:100160001BB103490348AFF3008008BD0000000045
:1001700014000020F82D000853B94AB9002908BF1F
:1001800000281CBF4FF0FF314FF0FF3000F074B972
:10019000ADF1080C6DE904CE00F006F8DDF804E0DE
:1001A000DDE9022304B070472DE9F047089E0D46B3
:1001B00004468846002B4DD18A42944668D9B2FA4B
:1001C00082F252B101FA02F3C2F1200120FA01F1E8
:1001D0000CFA02FC41EA030894404FEA1C45210C4A
:1001E000B8FBF5FE1FFA8CF705FB1E8341EA0343BB
:1001F0000EFB07F199420BD91CEB03030EF1FF3004
:1002000080F01E81994240F21B81AEF1020E6344E0
:100210005B1AA4B2B3FBF5F005FB103344EA0344C8
:1002200000FB07F7A7420AD91CEB040400F1FF33D7
:1002300080F00881A74240F2058164440238E41B43
:1002400040EA0E4000211EB1D4400023C6E900431D
:10025000BDE8F0878B4208D9002E00F0EE80002127
:10026000C6E900050846BDE8F087B3FA83F1002926
:100270004AD1AB4202D3824200F2F980841A65EB84
:10028000030301209846002EE2D0C6E90048DFE7CC
:1002900002B9FFDEB2FA82F2002A40F09180A1EBAF
:1002A0000C054FEA1C471FFA8CFE0121B5FBF7F342
:1002B00007FB1350250C45EA00450EFB03F0A8424E
:1002C00008D91CEB050503F1FF3802D2A84200F261
:1002D000CB8043462D1AA4B2B5FBF7F007FB1055AF
:1002E00044EA05440EFB00FEA64508D91CEB0404B5
:1002F00000F1FF3502D2A64500F2BB802846A4EBF0
:100300000E0440EA03409EE7C1F120078B4022FA29
:1003100007FC4CEA030C20FA07F405FA01F31C432E
:10032000FD404FEA1C4900FA01F3B5FBF9F8200C37
:100330001FFA8CFE09FB185540EA054508FB0EF034
:10034000A84202FA01F20BD91CEB050508F1FF3AAD
:1003500080F08880A84240F28580A8F102086544B8
:100360002D1AA4B2B5FBF9F009FB105544EA054576
:1003700000FB0EFEAE4508D91CEB050500F1FF346D
:100380006CD2AE456AD90238654440EA0840A0FB09
:100390000294A5EB0E05A542C846A64656D353D0F7
:1003A0005EB1B3EB080265EB0E0505FA07F722FA1A
:1003B00001F3CD401F43C6E900750021BDE8F08779
:1003C000C2F1200320FA03F10CFA02FC25FA03F330
:1003D00095400D434FEA1C471FFA8CFEB3FBF7F123
:1003E00007FB11302B0C43EA004301FB0EF098424F
:1003F00004FA02F408D91CEB030301F1FF382FD2F1
:1004000098422DD9023963441B1AADB2B3FBF7F001
:1004100007FB103345EA034500FB0EF3AB4208D956
:100420001CEB050500F1FF3816D2AB4214D9023897
:100430006544ED1A40EA014138E73146304607E7A6
:100440008646E5E61846FAE64B45A9D2B9EB02081E
:1004500064EB0C0E0138A3E74046EAE7204694E738
:100460004146D1E7D0467BE7023B654432E7084688
:1004700009E76444023842E7704700BF70B50D4D8C
:100480000D4C641BA4100026A64209D10B4D0C4C48
:1004900002F0B2FC641BA4100026A64205D170BD78
:1004A00055F8043B98470136EEE755F8043B98476A
:1004B0000136F2E700310008003100080031000881
:1004C0000431000802440346934200D1704703F808
:1004D000011BF9E710B594B0002404943C22214696
:1004E00005A8FFF7EFFF23E000243EE0013C14AB3A
:1004F0001C44002304F8403C4B4904A802F062FC71
:1005000050B14A4904A802F05DFC28B1484904A84A
:1005100002F058FC002847D1464800F0ADF94648A3
:1005200000F0AAF94022002104A8FFF7CBFF002425
:10053000424B1B68DA6912F0080F01D008221A62D8
:1005400040F6FF7301220DF10F013C4801F018F84D
:100550000028EDD1631C9BB214AA14449DF80F200F
:1005600004F8402C3F2BBFD81C46631E14AA13442A
:1005700013F8403C0D2B01D00A2BD9D1304A01ABE6
:1005800092E8030083E8030003222E4904A802F046
:1005900008FC0028AAD003222B4904A802F001FC81
:1005A0000028A3D00024C3E7284904A802F00AFCCD
:1005B00090B1274904A802F005FCD0B1254904A850
:1005C00002F000FCF0B1244904A802F0FBFB30BBB0
:1005D000224800F051F9A5E7214800F04DF9214BE0
:1005E00001221A704FF001311F4800F0DFF914B0FA
:1005F00010BD1E4800F040F900F034FA1C4800F02D
:100600003BF98FE7BFF34F8F1A49CA6802F4E062E3
:10061000194B1343CB60BFF34F8F00BFFDE7174863
:1006200000F02AF97EE700BF3C2E0008482E0008A3
:10063000542E000800500008642E000878000020A6
:10064000102E0008342E0008382E0008682E0008EE
:10065000902E0008DC2E0008E82E0008F82E000876
:10066000742E00082C00002004400008982E00087A
:10067000AC2E000800ED00E00400FA05042F00088D
:1006800008B5064B1B7813B1012B03D008BDFFF74B
:1006900021FFFBE700F0BCF9F8E700BF2C000020C9
:1006A00072B6FEE700B59BB04822002108A8FFF70C
:1006B00009FF002302930393049305930693079382
:1006C00015490A6822F4C06242F400720A600A689E
:1006D00002F4C0620192019A202208920122109233
:1006E0001193B0221292139308A801F0F5F978B98A
:1006F0004F230293002303930493059306930793D8
:10070000022102A801F024FD20B91BB05DF804FB12
:10071000FFF7C6FFFFF7C4FF0004005808B502F05A
:10072000EFFAFFF7BFFF00F013FA134B1B68B3F1AA
:100730005A3F0AD0104B1B68B3F15A3F16D10F48ED
:1007400000F09AF8FFF79CFFFCE70D4B1A680D4B81
:100750001340B3F1005FEDD1074B5B68B3F1013F8C
:10076000E8D000F007F900F00FF9E3E74FF05A3155
:10077000014800F01BF9E2E700400008182F0008CC
:10078000006000080000FE2F10B584460378302B6F
:1007900003D000242046234654E04378782B35D0FC
:1007A000582B36D00024204623464BE02401A3F1E9
:1007B000300E5FFA8EFEBEF1090F21D8303B1C448B
:1007C00001300A2815D81CF8003093B1A3F141027A
:1007D000D2B2052AEAD9A3F1610E5FFA8EFEBEF10C
:1007E000050FE3D9A3F1300E5FFA8EFEBEF1090FBB
:1007F000DCD91CF80030002B3BD10C60012010BD6F
:10080000052A01D8373BDAE7573BD8E70024022016
:10081000D7E700240220D4E76B2A1ED04B2A1CD035
:100820006D2A20D04D2A1ED0A2F1300E5FFA8EFE26
:10083000BEF1090FE3D804EB840402EB4402A2F1F9
:10084000300401330A2BDAD80028D8D11CF8032051
:10085000002AE1D10C600120F3E7002BE0D0A402D4
:100860000C600120EDE7002BDED024050C60012098
:10087000E7E70020C3E7000008B50146002201E0D9
:10088000013292B28B5C002BFAD16423014800F054
:1008900008FE08BD7800002000B583B08DF8070081
:1008A000094BD3F88430A02B09D0642301220DF129
:1008B0000701054800F0F5FD03B05DF804FB024BAD
:1008C0002022C3F88420F0E77800002000F178406F
:1008D000C00A704710B584B004460023039301F0AA
:1008E000DDFE0E4B4FF400421A612046FFF7EEFF8B
:1008F000C4F1006303F55C33DB0A0222009201902D
:10090000029303A9684601F0ADFF28B9002401F065
:10091000DDFE204604B010BD0124F8E70040005879
:10092000F0B583B005460C46174601F0B7FE002629
:1009300002E0083508340236BE4215D26B46206804
:10094000616803C3DDE900232946012001F002FFAD
:100950000028F0D128686A680099019B9A4208BF74
:100960008842E6D0032400E0002401F0AFFE2046D8
:1009700003B0F0BD08B5034800F038FB02F071F990
:1009800008BD00BF7800002008B5054A5368054936
:100990000B6005490B60126882F30888984708BD10
:1009A00000600008300000203400002070B588B0DE
:1009B00004460D4600230793134ED6E90023CDE9E4
:1009C000042301F06BFE114B4FF400421A613046D4
:1009D000FFF77CFF0223019302900123039307A9F1
:1009E00001A801F03FFF50B9B4420AD00595DDE9F6
:1009F00004230549012001F0ADFE01F067FE08B0B7
:100A000070BD0495F3E700BF0040000800400058A7
:100A100000B583B00023019301A800F0F3F910B1F1
:100A200003B05DF804FB4FF05A310A48FFF7BEFFF0
:100A30004FF002310848FFF7B9FF084B1A68084B1E
:100A40001340B3F1005FEBD1FFF794FFFFF79CFF7A
:100A5000E6E700BF0040000804400008006000080E
:100A60000000FE2F08B54FF05A310A48FFF79EFFED
:100A7000094B1A68094B1340B3F1005F00D008BD61
:100A8000044B5B68B3F1013FF9D0FFF773FFFFF749
:100A90007BFFF4E700400008006000080000FE2F24
:100AA000704700004FF0B0439A6B4FF0FF319963ED
:100AB000DA6BD9639A6B00229A63D86BDA63186C8D
:100AC0001964186C1A64586C5964586C5A64986AA2
:100AD0009962986A9A62D86AD962D86ADA62186B9F
:100AE0001963196B1A635A6C42F001025A645A6C0A
:100AF00022F001025A64D3F8902042F48032C3F805
:100B00009020D3F8902022F48032C3F89020BFF3D5
:100B10004F8F0549CA6802F4E062044B1343CB606F
:100B2000BFF34F8F00BFFDE700ED00E00400FA05C2
:100B3000704770477047FEE770477047704708B5C9
:100B400002F0F4F802F0FEF800F034FA08BD704745
:100B500008B51748174B03604FF4E1334360002397
:100B60008360C36003610C2242618361C3610362DD
:100B70004362836200F0D4FD70B900210C4800F09C
:100B800048FE60B900210A4800F068FE50B90848E4
:100B900000F020FE48B908BDFFF782FDEDE7FFF742
:100BA0007FFDEFE7FFF77CFDF1E7FFF779FDF2E767
:100BB000780000200044004010B596B004460021A3
:100BC00011911291139114911591382203A8FFF7F6
:100BD00079FC22681A4B9A4201D016B010BD02234C
:100BE00003934FF44023059303A801F0E3FB18BBE4
:100BF0004FF0B0439A6D42F400329A659A6D02F458
:100C000000320292029ADA6C42F00102DA64DB6C82
:100C100003F001030193019B0C2311930223129310
:100C200001231393002314930723159311A94FF065
:100C3000904001F057FED0E7FFF732FDD8E700BF44
:100C40000044004008B50268074B9A4200D008BD36
:100C50004FF0B042936D23F4003393650C214FF0B5
:100C6000904001F011FFF2E700440040BFF34F8FC6
:100C70000549CA6802F4E062044B1343CB60BFF33A
:100C80004F8F00BFFDE700BF00ED00E00400FA0554
:100C900041F4807106E080F4815080F0010011F48D
:100CA000803F09D14000490011F4807F00D001301D
:100CB00010F4803FF3D0EEE780B2704738B50446B9
:100CC0004518002004E014F8011B80B2FFF7E0FF94
:100CD000AC42F8D3002180B2FFF7DAFF0021FFF722
:100CE000D7FF38BD2DE9F04182B006460C461546C7
:100CF00000230B60134601220DF10701404800F06C
:100D00003FFC8046002872D19DF80710182919D899
:100D10004BB2002B48D0013917290FD8DFE801F07A
:100D200048310E0C0E0E0E0E0E0E0E0E0E0E0E0E88
:100D30000E0E0E0E0E0E0E3400270AE04FF00108C4
:100D4000002706E0412935D0612937D14FF002084C
:100D500000279DF8073033707F2F49D92B463A1D65
:100D6000B11C274800F00CFC8046002845D1B27821
:100D7000F378DB43DBB29A422AD04FF00108002718
:100D800036E04FF48067E4E72B4601220DF10701BE
:100D90001B4800F0F5FBA8B99DF80730182B15D0BB
:100DA0004FF001080027D4E74FF001080027D0E7F3
:100DB0008027CEE74FF002080027CAE74FF001086E
:100DC0000027C6E74FF001080027C2E70227C0E767
:100DD000F3191A795D7905EB02253946301DFFF7C5
:100DE0006DFFA84204D04FF00108002700E0002763
:100DF0002760404602B0BDE8F0810027F8E700BF59
:100E0000780000202DE9F04F89B001904FF00008E4
:100E10004646DFF888B1C1464546C246BAF1000FE2
:100E200040F0B880002E40F0B5805D4B00221A7073
:100E3000574685E0079D3DB1022D0AD10620FFF7F8
:100E40002BFD3D4602267BE00620FFF725FD01270E
:100E500076E0544B9A78524B1B789A420BD1002B78
:100E600053D1504B1B79CBB90620FFF715FD3D46FA
:100E70000127BA4664E01520FFF70EFD3D465FE00E
:100E80000133494881540132197809B13F2AF7D911
:100E900045490020885401333A4608E03A46434B1E
:100EA000F2E7013308A8104400F8181C0132197841
:100EB000202901D00F2AF4D908AB1A44002302F8E4
:100EC000183C06A902A8FFF75FFC069A384B9A4225
:100ED00013D83248FFF7FEFC069B019A13600620E8
:100EE000FFF7DAFC4320FFF7D7FC2D4A13780133D4
:100EF00013703D464FF0010922E01820FFF7CCFCAB
:100F00001820FFF7C9FC0526E3E7AA082749584639
:100F1000FFF706FD28B9079B9B440620FFF7BCFCA2
:100F2000E3E71820FFF7B8FC1820FFF7B5FC04260C
:100F3000DBE71820FFF7B0FC1820FFF7ADFC2646D2
:100F4000002F7FF46BAF002E7FF468AF4FF4FA727E
:100F500007A91448FFF7C6FE044600283FF46AAF0D
:100F60000228E6D0B9F1000F00D00135052D07D9D0
:100F70001820FFF791FC1820FFF78EFC0226DFE710
:100F80004320FFF789FC08F10108B8F13B0FD7D9DE
:100F9000FFF76CFE304609B0BDE8F08F0060000836
:100FA0000E05002008010020380000200C01002060
:100FB0000110030008B50A4BA3FB00231B0B43F6EB
:100FC000982202FB130343B9064B1B782BB1064A48
:100FD0001278934202D0044A137008BDFFF746FE10
:100FE00073B2E7450E0500200F050020E8B138B5C3
:100FF00005462423C0F884300268136823F00103F7
:101000001360036800241C6003685C6003689C60D4
:10101000FFF718FEC5F88C40C5F88440C5F8884035
:10102000EC6685F88040204638BD012070470000FE
:1010300070B504460168836802691343426913432B
:10104000C269134308689D4A024013430B6022683B
:10105000536823F44053E1680B435360A16922684D
:10106000974B9A4201D0236A1943936823F06E4349
:1010700023F430630B4393602268D36A23F00F0399
:10108000616A0B43D36223688E4A93421CD08E4A16
:10109000934231D08A4A93424BD0102288498B42E6
:1010A00068D0E069B0F5004F00F0A580082A00F292
:1010B0001F81DFE812F0D300F500D1001D01F80018
:1010C0001D011D011D01FB004FF0B042D2F8882028
:1010D00002F0030242F44032A2F54032032A09D85A
:1010E000DFE802F002043C060122D7E70422D5E73C
:1010F0000822D3E71022D1E74FF0B042D2F888207F
:1011000002F00C0242F44022A2F540220C2A0ED832
:10111000DFE802F0070D0D0D090D0D0D260D0D0D6B
:101120000B000022BAE70422B8E70822B6E7102233
:10113000B4E74FF0B042D2F8882002F44062B2F532
:10114000006F0FD005D87AB1B2F5806F0ED10422AE
:10115000A4E7B2F5406F0BD108229FE702229DE77A
:1011600002229BE7022299E7002297E7102295E7E7
:10117000102293E7082A00F29C80DFE802F0089A28
:101180003A9A379A9A9A05004FF4004004E001F029
:10119000F1F8002800F08F80626A4C4B33F812207F
:1011A000B0FBF2F3656805EB4501994200F29480CB
:1011B000B3EB053F00F29280002633463146FEF73E
:1011C000DBFF090241EA106100026B08C0182A46E1
:1011D000334641F10001FEF7CFFFA0F540723C4BD2
:1011E0009A427DD82368D860304650E000F0DCFB9E
:1011F000CFE73848D0E7082A74D8DFE802F007279D
:1012000005732A7373730B00324803E001F0B2F8E0
:10121000002869D0626A2D4B33F81230B0FBF3F02E
:101220006268530803EB4000B0FBF2F080B2A0F11B
:1012300010024FF6EF739A4258D820F00F03C0F314
:10124000420018432368D860002020E001F0A2F893
:10125000DEE700F0A9FBDBE71E4803E001F08AF8B7
:10126000002847D0626A194B33F81230B0FBF3F014
:10127000636800EB5300B0FBF3F080B2A0F1100202
:101280004FF6EF739A4237D82368D86000200123C5
:10129000A4F86A30A4F8683000232367636770BD40
:1012A00001F078F8DCE700F07FFBD9E74FF400406D
:1012B000D8E70120EBE70020E9E700BFF369FFCFA3
:1012C000008000400038014000440040C82F000862
:1012D000FFFC0F000024F4000120D8E70120D6E72E
:1012E0000120D4E70120D2E70020D0E70120CEE79B
:1012F0000120CCE70020CAE70120C8E7836A13F089
:10130000010F06D00268536823F40033C16A0B430F
:101310005360836A13F0020F06D00268536823F407
:101320008033016B0B435360836A13F0040F06D0C4
:101330000268536823F48023416B0B435360836A34
:1013400013F0080F06D00268536823F40043816B42
:101350000B435360836A13F0100F06D00268936842
:1013600023F48053C16B0B439360836A13F0200F07
:1013700006D00268936823F40053016C0B4393601A
:10138000836A13F0400F0AD00268536823F4801375
:10139000416C0B435360436CB3F5801F0BD0836AE1
:1013A00013F0800F06D00268536823F40023C16C49
:1013B0000B43536070470268536823F4C003816C89
:1013C0000B435360EBE72DE9F84305460F461646FD
:1013D0009946DDF820802C68E46937EA04030CBFE5
:1013E0004FF0010C4FF0000CB44557D1B8F1FF3F5E
:1013F000F1D001F0A7FCA0EB090040452FD8B8F1CF
:10140000000F2CD02B681A6812F0040FE3D0DA69B1
:1014100012F4006FDFD04FF400621A622A6852E8BB
:10142000003F23F4D07342E800310029F6D12A6846
:1014300002F1080353E8003F23F00103083242E8B9
:1014400000310029F3D12023C5F88430C5F8883055
:10145000C5F88C30002385F8803003201FE02A680F
:1014600052E8003F23F4D07342E800310029F6D15E
:101470002A6802F1080353E8003F23F00103083211
:1014800042E800310029F3D12023C5F88430C5F8A3
:101490008830002385F88030032000E00020BDE87C
:1014A000F8832DE9F04182B01E46D0F88430202B1D
:1014B00058D104460D469046002957D0002A57D0EF
:1014C00090F88030012B55D0012380F88030002324
:1014D000C0F88C302123C0F8843001F033FC07467B
:1014E000A4F85480A4F85680A368B3F5805F05D0B3
:1014F0004FF00008002384F8803014E0236913B112
:101500004FF00008F6E7A8460025F3E738F8023B5D
:101510002268C3F308039362B4F8562092B2013AEA
:1015200092B2A4F85620B4F856309BB273B100962C
:101530003B46002280212046FFF745FFE0B9002D01
:10154000E4D015F8012B23689A62E5E700963B4644
:10155000002240212046FFF736FF78B92023C4F847
:10156000843000E0022002B0BDE8F0810120FAE7FB
:101570000120F8E70220F6E70320F4E70320F2E772
:101580002DE9F04383B01E46D0F88830202B40F080
:10159000818004460D46904600297FD0002A7FD0E6
:1015A00090F88030012B7DD0012380F8803000231B
:1015B000C0F88C302222C0F88820C36601F0C2FB3C
:1015C0000746A4F85C80A4F85E80A368B3F5805F4A
:1015D00006D0A3B9226972B9FF22A4F8602014E0F2
:1015E000226922B940F2FF12A4F860200DE0FF2228
:1015F000A4F8602009E07F22A4F8602005E0B3F1A0
:10160000805F0DD00022A4F86020B4F86080B3F5AC
:10161000805F0FD04FF00009002384F880301EE077
:1016200022691AB97F22A4F86020EEE73F22A4F8CD
:101630006020EAE7236913B14FF00009ECE7A946FF
:101640000025E9E723685B6A08EA030329F8023BFF
:10165000B4F85E2092B2013A92B2A4F85E20B4F8D7
:101660005E309BB28BB100963B4600222021204683
:10167000FFF7A9FEC0B9002DE4D023685A6A5FFACB
:1016800088F3134005F8013BE2E72023C4F88830D3
:10169000002000E0022003B0BDE8F0830120FAE75B
:1016A0000120F8E70220F6E70320F4E730B583B025
:1016B00004460023C0F88C3001F044FB0546226844
:1016C000126812F0080F0FD123681B6813F0040F83
:1016D00018D12023C4F88430C4F888300020E06694
:1016E00084F8800003B030BD6FF07E430093034662
:1016F00000224FF400112046FFF765FE0028E3D0DA
:101700000320EFE76FF07E4300932B4600224FF457
:1017100080012046FFF757FE0028DAD00320E1E7DA
:1017200078B310B50446D0F884300BB32423C4F842
:1017300084302268136823F0010313602046FFF70A
:1017400077FC012813D0A36ABBB92268536823F43D
:10175000904353602268936823F02A0393602268C1
:10176000136843F0010313602046FFF79FFF10BD8D
:1017700080F88030FFF720FAD8E72046FFF7BEFD5B
:10178000E3E7012070470000436E2BB90123A0F866
:101790006A30A0F86830704730B403689A68C2F3C2
:1017A00042629968490F094D6B5CDB00084C615C33
:1017B00093FBF1F3A0F86A30AB5CDB00A25C93FB17
:1017C000F2F3A0F8683030BC704700BFE82F000883
:1017D000E02F000890F88030012B18D0012380F80A
:1017E00080302423C0F8843003681A68196821F017
:1017F0000101196022F000520023436601680A606B
:101800002022C0F8842080F88030184670470220DB
:10181000704738B590F88030012B1DD00446012365
:1018200080F880302423C0F8843003681D681A686B
:1018300022F001021A600268936823F060431943A2
:101840009160FFF7A1FF23681D602023C4F8843056
:10185000002084F8800038BD0220FCE738B590F8FD
:101860008030012B1DD00446012380F880302423D2
:10187000C0F8843003681D681A6822F001021A60FB
:101880000268936823F0606319439160FFF77CFF5F
:1018900023681D602023C4F88430002084F8800071
:1018A00038BD0220FCE7000030B589B004468C4604
:1018B0002A4B93E803000690ADF81C1003F10802D0
:1018C00092E803000490ADF8141001AD103393E8D2
:1018D000070085E80700BCF5007F07D0002314E06F
:1018E00008AA02EB830353F81C5C1EE00023022BC2
:1018F00008D808AA02EB430232F8082CA242EFD221
:101900000133F4E7002510E00133022B0CD808AABC
:1019100002EB430232F8102CA242F5D308AA02EBE4
:10192000830353F81C5C00E000250D4A136823F084
:1019300007032B43136001F005FA0446084B1B68AC
:1019400003F00703AB4206D001F0FCF9001B0228AC
:10195000F4D9032000E0002009B030BD182E0008A3
:101960000040005810B5C0F303100C4B53F8204052
:101970004FF0B043D3F8083103F00F03084A52F890
:101980002300B4FBF0F401F005F901460548A0FB83
:101990000430800CFFF788FF10BD00BF882F0008BF
:1019A000282F000883DE1B434FF0B0439968DB68A3
:1019B00003F0030311F00C010AD00C2906D004290E
:1019C00047D008293BD00022104626E0012BF6D153
:1019D0004FF0B0431B6813F008030DD04FF0B04335
:1019E0001B6813F0080324D14FF0B042D2F89420C2
:1019F0002E4A52F823200EE04FF0B042126812F047
:101A0000080F12D14FF0B043D3F89430C3F303233F
:101A1000264A52F82320D1B100204FF0B0439B68F2
:101A200003F00C030C2B1AD070474FF0B042126831
:101A3000EEE74FF0B0431B68C3F30313D8E74FF052
:101A4000B0431A6812F4801206D11948E5E710462F
:101A5000E3E700221748E0E700221648DDE74FF0F1
:101A6000B043DB6803F00303022B09D0032B08D13A
:101A70004FF0B0431B6813F4801F15D10C4A00E0EF
:101A80000C4A4FF0B043D868C0F3062000FB02F2C6
:101A9000D868C0F302100130B2FBF0F2D868400FF2
:101AA0000130B2FBF0F0BFE7024AEAE7882F0008F6
:101AB0000048E8010024F40008B5FFF775FF4FF077
:101AC000B0439B68C3F30313024A52F82330B0FBC0
:101AD000F3F008BD282F0008002800F01983F8B59E
:101AE00004464FF0B0439D6805F00C05DE6806F033
:101AF0000306036813F0200F00F08F80EDB10C2D6A
:101B000019D0236A002B00F0BC804FF0B04213685C
:101B100043F00103136001F015F907464FF0B0439D
:101B20001B6813F0020F65D101F00CF9C01B0228ED
:101B3000F4D90320F9E2012EE3D14FF0B0431B6842
:101B400013F0020F03D0236A002B00F0E382A06A97
:101B50004FF0B0431B6813F0080F29D04FF0B0438B
:101B60001B6803F0F00398422AD9FFF7FBFE002818
:101B700040F0D2824FF0B0431A6842F008021A6077
:101B80001A6822F0F002A16A0A431A60616A5A6870
:101B900022F47F4242EA01225A60FFF78DFFB04BE8
:101BA0001860B04B186801F083F8002835D0BCE20B
:101BB0004FF0B043D3F894301B0903F0F003D2E7A1
:101BC0004FF0B0431A6842F008021A601A6822F017
:101BD000F002A16A0A431A60616A5A6822F47F42DD
:101BE00042EA01225A60A06AFFF7BCFE0028D4D066
:101BF00001209AE24FF0B0431A6842F008021A60DE
:101C00001A6822F0F002A16A0A431A60616A5A68EF
:101C100022F47F4242EA01225A60236813F0010F46
:101C200051D0082D45D00C2D41D04FF0B042136853
:101C300023F48013A1680B4313606368B3F5803FFE
:101C400063D0B3F5041F65D04FF0B0431A6822F497
:101C500080321A601A6822F400121A606368002B3E
:101C600063D001F06FF807464FF0B0431B6813F4E0
:101C7000003F28D101F066F8C01B6428F4D9032086
:101C800053E24FF0B042136823F00103136001F0F8
:101C900059F807464FF0B0431B6813F0020FBCD051
:101CA00001F050F8C01B0228F4D903203DE2032EB6
:101CB000BBD14FF0B0431B6813F4003F03D06368FF
:101CC000002B00F02B82236813F0020F52D0042D5A
:101CD0003DD00C2D39D02369002B00F091804FF0BE
:101CE000B042136843F48073136001F02BF806468A
:101CF0004FF0B0431B6813F4806F77D101F022F8E6
:101D0000801B0228F4D903200FE2136843F48033C8
:101D10001360A3E74FF0B0431A6842F400121A6050
:101D20001A6842F480321A6098E701F00BF807460F
:101D30004FF0B0431B6813F4003FC4D001F002F829
:101D4000C01B6428F4D90320EFE1022EC3D14FF069
:101D5000B0431B6813F4806F03D02369002B00F09D
:101D6000DF8161694FF0B042536823F0FE4343EADC
:101D700001635360236813F0080F00F08E80A3699D
:101D8000002B71D04FF0B043D3F89430E16903F0E9
:101D90001002914211D003F00302022A00F0C28126
:101DA00013F0010F42D14FF0B042D2F8943023F03B
:101DB0001003E1690B43C2F894304FF0B042D2F8FF
:101DC000943043F00103C2F8943000F0BBFF0646A4
:101DD0004FF0B043D3F8943013F0020F5DD100F010
:101DE000B1FF801B1128F3D903209EE161694FF0F8
:101DF000B042536823F0FE4343EA01635360B9E7FE
:101E00004FF0B042136823F48073136000F09AFF20
:101E100006464FF0B0431B6813F4806FAAD000F061
:101E200091FF801B0228F4D903207EE14FF0B042DD
:101E3000D2F8943023F00103C2F8943000F082FF0E
:101E400006464FF0B043D3F8943013F0020FAAD0F7
:101E500000F078FF801B1128F3D9032065E100BF53
:101E600000000020080000204FF0B042D2F894306B
:101E700023F00103C2F8943000F064FF06464FF0EF
:101E8000B043D3F8943013F0020F06D000F05AFF9D
:101E9000801B1128F3D9032047E1236813F0040FB6
:101EA00000F0B180A84B1B6813F4807F10D100F0C4
:101EB00069FE00F047FF0646A34B1B6813F4807FC2
:101EC00006D100F03FFF801B0228F5D903202CE14A
:101ED000E368002B61D0852B01D0052B07D14FF093
:101EE000B042D2F8903043F00403C2F8903000F0D2
:101EF00029FF06464FF0B042D2F8903043F001037C
:101F0000C2F890304FF0B043D3F8903013F0020F86
:101F100008D100F017FF801B41F288339842F1D9B5
:101F2000032002E1E368812B01D0852B1AD100F058
:101F300009FF06464FF0B042D2F8903043F08003DC
:101F4000C2F890304FF0B043D3F8903013F4006FE4
:101F500059D100F0F7FE801B41F288339842F1D945
:101F60000320E2E000F0EEFE06464FF0B042D2F869
:101F7000903023F08003C2F890304FF0B043D3F894
:101F8000903013F4006F3ED000F0DCFE801B41F275
:101F900088339842F1D90320C7E000F0D3FE06460B
:101FA0004FF0B042D2F8903023F08003C2F8903066
:101FB0004FF0B043D3F8903013F4006F08D000F026
:101FC000C1FE801B41F288339842F1D90320ACE076
:101FD00000F0B8FE06464FF0B042D2F8903023F041
:101FE0000103C2F890304FF0B043D3F8903013F0B3
:101FF000020F08D000F0A6FE801B41F28833984201
:10200000F1D9032091E0E36A002B00F08D800C2DC4
:1020100062D0022B1FD04FF0B0431A6822F08072BA
:102020001A60DA6822F00302DA60DA6822F0885275
:1020300022F48032DA6000F085FE04464FF0B043AF
:102040001B6813F0007F73D000F07CFE001B0A2891
:10205000F4D9032069E04FF0B042136823F0807395
:10206000136000F06FFE05464FF0B0431B6813F09D
:10207000007F2AD14FF0B042D36834491940236B16
:10208000606B0343A06B43EA0023E06B0343206CC7
:102090000343606C03430B43D360136843F08073C6
:1020A0001360D36843F08053D36000F04BFE0446C6
:1020B0004FF0B0431B6813F0007F37D100F042FEB1
:1020C000001B0A28F4D903202FE000F03BFE401B40
:1020D0000A28C9D9032028E0012B2BD04FF0B043A8
:1020E000DB6803F00301226B914225D103F07002FB
:1020F000616B8A4222D103F4FE42A16BB2EB012F45
:102100001ED103F06043626C93421BD100200CE0AF
:1021100001207047012008E0012006E0012004E0D2
:10212000012002E0012000E00020F8BD0020FCE7D3
:102130000020FAE70120F8E70120F6E70120F4E7A4
:102140000120F2E70120F0E7000400588C80C11163
:10215000002800F0048170B50C460546824B1B68D0
:1021600003F007038B4227D32B6813F0020F39D1FA
:102170002B6813F0400F4DD12B6813F0040F65D17D
:102180002B6813F0080F79D12B6813F0010F00F0C2
:10219000C1806B68022B00F08B80032B00F09080D5
:1021A000002B40F095804FF0B042126812F0020F01
:1021B00040F094800120D1E06B4A136823F00703BC
:1021C0000B43136000F0BEFD0646674B1B6803F02F
:1021D0000703A342C8D000F0B5FD801B0228F4D944
:1021E0000320BBE0AB684FF0B0418A6822F0F002F8
:1021F00013438B6000F0A6FD06464FF0B0439B688A
:1022000013F4803FB4D100F09DFD801B0228F4D967
:102210000320A3E069694FF0B042D2F8083123F0FF
:102220000F0343EA1113C2F8083100F08BFD064694
:102230004FF0B043D3F8083113F4803F9CD100F045
:1022400081FD801B0228F3D9032087E0EB684FF063
:10225000B0418A6822F4E06213438B6000F072FDA3
:1022600006464FF0B0439B6813F4003F88D100F05E
:1022700069FD801B0228F4D903206FE029694FF023
:10228000B042936823F4605343EAC103936000F0C3
:1022900059FD06464FF0B0439B6813F4802F7FF43E
:1022A00073AF00F04FFD801B0228F3D9032055E0E7
:1022B0004FF0B042126812F4003F0FD101204DE000
:1022C0004FF0B042126812F0007F07D1012045E0C4
:1022D0004FF0B042126812F4806F42D04FF0B0411C
:1022E0008A6822F0030213438B6000F02BFD064640
:1022F0004FF0B0439B6803F00C036A68B3EB820FA6
:1023000008D000F01FFD801B41F288339842EFD9BE
:10231000032023E0144B1B6803F00703A34215D9E5
:10232000114A136823F007032343136000F00AFDEA
:1023300005460D4B1B6803F00703A34206D000F0CF
:1023400001FD401B0228F4D9032007E0FFF7B4FB8E
:10235000064B1860064B186800F0AAFC70BD0120FF
:1023600070470120FAE700BF00400058000000203D
:102370000800002008B5FFF79FFB4FF0B0439B68B3
:10238000C3F30223024A52F82330D84008BD00BFED
:10239000682F000808B5FFF78FFB4FF0B0439B682C
:1023A000C3F3C223024A52F82330D84008BD00BF0D
:1023B000682F000870B50446036813F4803F40F0AE
:1023C000AB800025236813F0010F0AD062684FF03C
:1023D000B041D1F8883023EA124392B21343C1F8D6
:1023E0008830236813F0020F0AD0A2684FF0B04182
:1023F000D1F8883023EA124392B21343C1F88830EF
:10240000236813F0200F09D023694FF0B041D1F8B1
:10241000882022F440621343C1F88830236813F403
:10242000007F0CD0206A4FF0B041D1F88830020C08
:10243000120423EA020343EA0043C1F88830236808
:1024400013F4806F0CD0606A4FF0B041D1F888303F
:10245000020C120423EA020343EA0043C1F8883065
:10246000236813F4006F0CD0A06A4FF0B041D1F88C
:102470008830020C120423EA020343EA0043C1F845
:102480008830236813F0400F40F09E80236813F0DB
:10249000800F40F0AA80236813F4807F40F0B6805C
:1024A000236813F0100F0ED0E3684FF0B041D1F85D
:1024B000882022F440721343C1F88830E368B3F5F2
:1024C000807F00F0B480236813F4004F0FD0236B9B
:1024D0004FF0B041D1F8882022F040421343C1F8B8
:1024E0008830236B1BB9CB6843F08073CB602368C3
:1024F00013F4804F0ED0E36A4FF0B041D1F888203A
:1025000022F040521343C1F88830E36AB3F1005F10
:1025100000F09280284670BD00F034FB00F012FC01
:102520000546484B1B6813F4807F06D100F00AFC77
:10253000401B0228F5D9032500E00025002D7FF47B
:1025400041AF4FF0B043D3F8903003F44073626B67
:102550009A4224D04FF0B043D3F8902022F4407236
:10256000D3F8901041F48031C3F89010D3F8901054
:1025700021F48031C3F89010C3F8902012F0020FBC
:102580000FD1002D7FF41EAF636B4FF0B041D1F837
:10259000902022F440721343C1F8903012E70022D9
:1025A000ECE700F0CFFB06464FF0B043D3F8903095
:1025B00013F0020FE5D100F0C5FB801B41F2883318
:1025C0009842F1D90325DCE763694FF0B040D0F8B9
:1025D0008820190901F47F2122EA01021B0103F47A
:1025E0007F231343C0F8883050E7A3694FF0B04011
:1025F000D0F88820190901F47F2122EA01021B0189
:1026000003F47F231343C0F8883044E7E3694FF0B5
:10261000B040D0F88820190901F47F2122EA010294
:102620001B0103F47F231343C0F8883038E7CB68DD
:1026300043F08073CB6046E7CB6843F48033CB60D4
:1026400068E700BF0004005810B4054C616941F010
:10265000010161610260BFF36F8F436010BC70477E
:10266000004000580C4A536943F480235361EFF350
:10267000108C72B6402351F8042B40F8042B013B18
:1026800013F0FF03F7D1044B1B6913F4803FFAD119
:102690008CF31088704700BF00400058094B5B69FD
:1026A000002B01DB00207047064B074A9A6002F1BD
:1026B00088329A605B69002B01DB002070470120A3
:1026C000704700BF0040005823016745054B5A6919
:1026D00042F000425A615B69002B01DB0120704728
:1026E000002070470040005838B5054600F02AFB2E
:1026F0000446164B1B6913F4803F06D000F022FB02
:10270000001BA842F5D3032038BD104B1B6913F002
:10271000010F02D00D4A012111614CF2FA3213402F
:1027200001D00A4A13615BB9084B1B6913F4802F6F
:102730000AD000F007FB001BA842F5D30320E3E713
:10274000034A53600120DFE70020DDE70040005826
:1027500010050020F8B51F46154B1B78012B25D01E
:1027600004460D461646124B01221A7000225A608A
:102770004FF47A70FFF7B8FF70B9012C10D03146D2
:102780002846FFF76FFF4FF47A70FFF7ADFF094A55
:10279000536923EA04045461054B00221A70F8BD02
:1027A00032463B462846FFF74FFFECE70220F6E7AC
:1027B0001005002000400058034A536943F4803359
:1027C00043F004035361704700400058184B1B68E6
:1027D00003F40073012B06D0154B1B6803F48063D0
:1027E000012B12D07047124B1A6822F400721A6043
:1027F0001A6842F400621A601A6822F400621A60D1
:102800001A6842F400721A60E6E7094B1A6822F46B
:1028100080621A601A6842F480521A601A6822F4C0
:1028200080521A601A6842F480621A60DAE700BFC8
:1028300000400058034A536923F47E7323F00203D7
:102840005361704700400058054A536923F47E7372
:1028500043EAC00040F4803040F00200506170470D
:1028600000400058F8B51E4B1B78012B35D00546AB
:102870000F461B4B01221A7000225A604FF47A70E7
:10288000FFF732FF064618BB2B68042B13D04FF01E
:10289000FF333B606C686B68AA681344A34213D98A
:1028A0002046FFF7D1FF4FF47A70FFF71DFF064671
:1028B00048B90134EFE7FFF77FFF4FF47A70FFF775
:1028C00013FF064602E03C60FFF7B4FFFFF77EFF10
:1028D000034B00221A703046F8BD0226FBE700BF0A
:1028E0001005002070B5002369E085685E000324B0
:1028F000B44025EA0405CC68B4402C4384604468A5
:1029000024EA0C0C4C68C4F300149C4044EA0C0408
:10291000446065E0DD08083550F8256003F00704E1
:102920004FEA840C0F2404FA0CF426EA040E0C6916
:1029300004FA0CF444EA0E0440F8254067E002244F
:1029400000E0002404FA0EF42C430CF1020C4B4D71
:1029500045F82C404A4CD4F88050D44325EA02066E
:10296000D1F804C01CF4803F01D042EA0506444D72
:10297000C5F88060D5F8845004EA0506D1F804C093
:102980001CF4003F01D042EA05063D4DC5F88460C5
:102990002D6804EA0506D1F804C01CF4801F01D09C
:1029A00042EA0506364D2E606D682C404E6816F4DE
:1029B000001F01D042EA0504314A546001330A681D
:1029C00032FA03F458D04FF0010C0CFA03FC1CEA65
:1029D0000202F3D04C6804F00304013C012C84D9BA
:1029E0004C6804F00304032C0CD0C4685D004FF065
:1029F000030C0CFA05FC24EA0C0C8C68AC4044EA8D
:102A00000C04C4604C6804F00304022C82D00468F7
:102A10004FEA430E4FF0030C0CFA0EFC24EA0C0CA8
:102A20004C6804F0030404FA0EF444EA0C04046055
:102A30004C6814F4403FC1D04FEA930C0CF10205EE
:102A40000E4C54F8255003F003044FEA840E07247B
:102A500004FA0EF425EA0405B0F1904F3FF471AF8B
:102A6000084CA04206D004F58064A0423FF467AF52
:102A7000072467E7012465E770BD00BF000001403F
:102A80000008005800040048002331FA03F271D016
:102A9000F0B52EE0022500E0002505FA0CFCA44567
:102AA00049D004685D004FF0030C0CFA05FC44EAC1
:102AB0000C0404604FEAD30E0EF1080E50F82E40BD
:102AC00003F00705AE000F25B54024EA050440F8E1
:102AD0002E40846824EA0C048460446824EA0202DC
:102AE0004260C26822EA0C02C260013331FA03F28A
:102AF0003FD001229A4012EA0107F6D09E08B51C89
:102B00001D4C54F8254003F0030C4FEA8C0C4FF099
:102B1000070E0EFA0CFE0EEA0404B0F1904FBBD083
:102B2000164DA84205D005F58065A842B2D007250C
:102B3000B3E70125B1E7124CD4F8805025EA070528
:102B4000C4F88050D4F8845025EA0705C4F88450AE
:102B5000256825EA07052560656825EA0707676097
:102B6000054D023655F8264024EA0E0445F8264065
:102B700097E7F0BD704700BF000001400004004827
:102B800000080058024A136843F4807313607047CA
:102B900000040058024B186800F4C060704700BF82
:102BA00000040058074AD36823F4E0631B041B0C9D
:102BB000000200F4E060034343F0BF6343F40033DA
:102BC000D360704700ED00E000B5194BDB68C3F33C
:102BD0000223C3F1070CBCF1040F28BF4FF0040C13
:102BE00003F1040EBEF1060F18D9033B4FF0FF3E70
:102BF0000EFA0CFC21EA0C0199400EFA03F322EACA
:102C00000303194300280BDB0901C9B200F160403E
:102C100000F5614080F800135DF804FB0023E5E750
:102C200000F00F000901C9B2024B1954F4E700BFCC
:102C300000ED00E014ED00E00138B0F1807F0BD230
:102C40004FF0E0235861054AF02182F8231000205C
:102C5000986107221A6170470120704700ED00E07B
:102C6000704710B54FF0B0439A6B4FF0FF329A6344
:102C7000D96BDA63996B00249C63D96BDC63196CA4
:102C80001A64196C1C64596C5A64596C5C64996AB6
:102C90009A62996A9C62D96ADA62D96ADC62196BB3
:102CA0001A631A6B1C63FFF7DBFF204610BD0000A0
:102CB000114B1B780BB90120704710B50446FEF785
:102CC000FBFE0D4B1A784FF47A73B3FBF2F3B0FBB3
:102CD000F3F0FFF7B1FF68B90F2C01D901200AE02A
:102CE000002221464FF0FF30FFF76EFF034B1C60C0
:102CF000002000E0012010BD04000020080000209A
:102D000010B50320FFF74EFFFEF7D6FE064B186006
:102D10000F20FFF7CDFF10B10124204610BD04465F
:102D2000FDF7BEFEF9E700BF00000020034B1B7853
:102D3000034A11680B441360704700BF0400002071
:102D400028050020014B1868704700BF28050020A7
:102D50000D488546FDF7FBFE0C480D490D4A002342
:102D600002E0D458C4500433C4188C42F9D30A4A40
:102D70000A4C002301E013600432A242FBD3FDF7AA
:102D80007DFBFDF7CBFCFEE700800020000000206B
:102D90001000002020500008100000203005002006
:102DA000FEE710B501390244904201D1002005E050
:102DB000037811F8014FA34201D0181B10BD013058
:102DC000F2E7000030B50B4D044614F8013B5A5DA4
:102DD00002F00302012A11F8012BA85C00F00300A5
:102DE00008BF2033012808BF2032981A01D1002AD9
:102DF000EBD130BDF12F0008F8B500BFF8BC08BC1E
:102E00009E467047F8B500BFF8BC08BC9E467047A8
:102E1000342E0008382E0008120024003000000074
:102E200006000C001000000000000000010000007F
:102E30000200000061742B0041542B0061742B765A
:102E4000657273696F6E000061742B7665723D3F29
:102E50000000000061742B626F6F747665723D3FF5
:102E6000000000000D0A000061742B75706461742D
:102E7000650000005374617274206669726D776139
:102E8000726520757067726164652E2E2E0D0A00C2
:102E900061742B72756E000053746F7020426F6FF7
:102EA00074204D6F64650D0A000000004A756D7056
:102EB000206661696C65642E204E6F206C656761C9
:102EC0006C206170706C69636174696F6E206465F9
:102ED0007465637465642E0D0A00000061742B72C2
:102EE000657365740000000061742B626F6F74730A
:102EF0007461747573000000426F6F74204D6F64CD
:102F0000650D0A004154206E6F7420737570706FE8
:102F100072742E0D0A0000003C424F4F54204D4F5A
:102F200044453E0D0A0000000100000003000000BF
:102F30000500000001000000010000000600000084
:102F40000A00000020000000020000000400000051
:102F50000800000010000000400000008000000099
:102F6000000100000002000000000000000000005E
:102F7000000000000000000001000000020000004E
:102F80000300000004000000A0860100400D0300C3
:102F9000801A060000350C0040420F0080841E009D
:102FA00000093D0000127A000024F40000366E0192
:102FB0000048E801006CDC02000000000000000096
:102FC00000000000000000000100020004000600F4
:102FD00008000A000C0010002000400080000001E2
:102FE00008040204080101010101010307010000B6
:102FF00000202020202020202020282828282820C9
:1030000020202020202020202020202020202020C0
:103010002088101010101010101010101010101028
:103020001004040404040404040404101010101018
:1030300010104141414141410101010101010101E2
:103040000101010101010101010101011010101034
:1030500010104242424242420202020202020202B4
:103060000202020202020202020202021010101008
:103070002000000000000000000000000000000030
:103080000000000000000000000000000000000040
:103090000000000000000000000000000000000030
:1030A0000000000000000000000000000000000020
:1030B0000000000000000000000000000000000010
:1030C0000000000000000000000000000000000000
:1030D00000000000000000000000000000000000F0
:1030E00000000000000000000000000000000000E0
:1030F0000000000000000000B0D0FF7F01000000D1
:103100005D01000800000000390100080000000017
:104000005A5A5A5A00000000390100080000000006
:105000005255495F424F4F545F302E385F53544DD5
:105010003332574C45354343000000000000000088
:1050200000093D0001000000100000000000000029
:1060000000FC002009780008857800081179000854
:106010007D7900087F790008817900080000000080
:10602000000000000000000000000000837900086C
:10603000857900080000000087790008877900084A
:106040005978000859780008A5790008597800089F
:106050005978000859780008FB790008017A00088F
:10606000077A00080D7A0008137A0008B179000851
:10607000BD790008C9790008D57900085978000869
:1060800059780008597800085978000859780008AC
:106090005978000859780008197A000859780008DA
:1060A000597800085978000859780008597800088C
:1060B000597800085978000859780008597800087C
:1060C000C57A0008D17A0008597800085978000884
:1060D000E1790008F9790008AD7A000859780008DC
:1060E00059780008597A00088D7900085978000815
:1060F000597800085978000859780008597800083C
:10610000597800085978000899790008DD7A000864
:10611000597800085978000859780008597800081B
:10612000597800085978000859780008597800080B
:1061300059780008597800085978000859780008FB
:1061400010B5054C237833B9044B13B10448AFF3B1
:1061500000800123237010BDA00D0020000000006E
:1061600070D3020808B5034B1BB103490348AFF3D2
:10617000008008BD00000000A40D002070D30208BC
:1061800010F8012B11F8013B012A28BF9A42F7D0E1
:10619000D01A7047034613F8012B002AFBD1181AB6
:1061A00001387047000000000000000000000000FF
:1061B00001F0FF01102A2BDB10F0070F08D010F8B8
:1061C000013B013A8B422DD010F0070F42B3F6D1BC
:1061D000F0B441EA012141EA014122F007047FF0D5
:1061E00000070023F0E80256083C85EA010586EA2C
:1061F000010685FA47F5A3FA87F586FA47F6A5FA68
:1062000087F68EB9EED1F0BC01F0FF0102F0070273
:1062100032B110F8013B013A83EA010313B1F8D11E
:106220000020704701387047002D06BF35460338FF
:10623000073815F0010F07D1013015F4807F02BF38
:10624000013015F4C03F0130F0BC0138704700BF89
:1062500081F0004102E000BF83F0004330B54FEA17
:1062600041044FEA430594EA050F08BF90EA020F84
:106270001FBF54EA000C55EA020C7FEA645C7FEA17
:10628000655C00F0E2804FEA5454D4EB5555B8BF3A
:106290006D420CDD2C4480EA020281EA030382EAAB
:1062A000000083EA010180EA020281EA0303362D3D
:1062B00088BF30BD11F0004F4FEA01314FF4801C10
:1062C0004CEA113102D0404261EB410113F0004F22
:1062D0004FEA03334CEA133302D0524263EB4303D9
:1062E00094EA050F00F0A780A4F10104D5F1200E77
:1062F0000DDB02FA0EFC22FA05F2801841F10001D2
:1063000003FA0EF2801843FA05F359410EE0A5F1A5
:1063100020050EF1200E012A03FA0EFC28BF4CF0D6
:10632000020C43FA05F3C01851EBE37101F000458C
:1063300007D54FF0000EDCF1000C7EEB00006EEB99
:106340000101B1F5801F1BD3B1F5001F0CD3490823
:106350005FEA30004FEA3C0C04F101044FEA44527A
:1063600012F5800F80F09A80BCF1004F08BF5FEA01
:10637000500C50F1000041EB045141EA050130BDE1
:106380005FEA4C0C404141EB0101013C28BFB1F5F3
:10639000801FE9D291F0000F04BF01460020B1FA3E
:1063A00081F308BF2033A3F10B03B3F120020CDA11
:1063B0000C3208DD02F1140CC2F10C0201FA0CF0EF
:1063C00021FA02F10CE002F11402D8BFC2F1200C54
:1063D00001FA02F120FA0CFCDCBF41EA0C0190400A
:1063E000E41AA2BF01EB0451294330BD6FEA040453
:1063F0001F3C1CDA0C340EDC04F11404C4F120023E
:1064000020FA04F001FA02F340EA030021FA04F34F
:1064100045EA030130BDC4F10C04C4F1200220FAA6
:1064200002F001FA04F340EA0300294630BD21FAE4
:1064300004F0294630BD94F0000F83F4801306BFAA
:1064400081F480110134013D4EE77FEA645C18BF9E
:106450007FEA655C29D094EA050F08BF90EA020F35
:1064600005D054EA000C04BF1946104630BD91EA2D
:10647000030F1EBF0021002030BD5FEA545C05D130
:106480004000494128BF41F0004130BD14F580046F
:106490003CBF01F5801130BD01F0004545F0FE41E3
:1064A00041F470014FF0000030BD7FEA645C1ABF18
:1064B000194610467FEA655C1CBF0B46024650EA4F
:1064C000013406BF52EA033591EA030F41F400217B
:1064D00030BD00BF90F0000F04BF0021704730B501
:1064E0004FF4806404F132044FF000054FF00001D6
:1064F00050E700BF90F0000F04BF0021704730B597
:106500004FF4806404F1320410F0004548BF40426B
:106510004FF000013EE700BF42004FEAE2014FEAC0
:1065200031014FEA02701FBF12F07F4393F07F4F9B
:1065300081F06051704732F07F4208BF704793F09E
:106540007F4F04BF41F40021704730B54FF46074B1
:1065500001F0004521F000411CE700BF50EA0102B4
:1065600008BF704730B54FF000050AE050EA01025D
:1065700008BF704730B511F0004502D5404261EBCD
:1065800041014FF4806404F132045FEA915C3FF40E
:10659000D8AE4FF003025FEADC0C18BF03325FEAAB
:1065A000DC0C18BF033202EBDC02C2F1200300FA5C
:1065B00003FC20FA02F001FA03FE40EA0E0021FA81
:1065C00002F11444BDE600BF70B54FF0FF0C4CF46F
:1065D000E06C1CEA11541DBF1CEA135594EA0C0F21
:1065E00095EA0C0F00F0DEF82C4481EA030621EA5C
:1065F0004C5123EA4C5350EA013518BF52EA033597
:1066000041F4801143F4801338D0A0FB02CE4FF048
:106610000005E1FB02E506F00042E0FB03E54FF078
:106620000006E1FB03569CF0000F18BF4EF0010E70
:10663000A4F1FF04B6F5007F64F5407404D25FEA6C
:106640004E0E6D4146EB060642EAC62141EA55511F
:106650004FEAC52040EA5E504FEACE2EB4F1FD0C61
:1066600088BFBCF5E06F1ED8BEF1004F08BF5FEADF
:10667000500E50F1000041EB045170BD06F0004691
:1066800046EA010140EA020081EA0301B4EB5C043E
:10669000C2BFD4EB0C0541EA045170BD41F4801136
:1066A0004FF0000E013C00F3AB8014F1360FDEBF5B
:1066B000002001F0004170BDC4F10004203C35DA37
:1066C0000C341BDC04F11404C4F1200500FA05F3BA
:1066D00020FA04F001FA05F240EA020001F000425B
:1066E00021F0004110EBD37021FA04F642EB0601D1
:1066F0005EEA430E08BF20EAD37070BDC4F10C04FB
:10670000C4F1200500FA04F320FA05F001FA04F2BE
:1067100040EA020001F0004110EBD37041F10001AA
:106720005EEA430E08BF20EAD37070BDC4F12005B5
:1067300000FA05F24EEA020E20FA04F301FA05F21D
:1067400043EA020321FA04F001F0004121FA04F2C5
:1067500020EA020000EBD3705EEA430E08BF20EA95
:10676000D37070BD94F0000F0FD101F000464000CF
:1067700041EB010111F4801F08BF013CF7D041EA51
:10678000060195F0000F18BF704703F00046520055
:1067900043EB030313F4801F08BF013DF7D043EA26
:1067A0000603704794EA0C0F0CEA135518BF95EADC
:1067B0000C0F0CD050EA410618BF52EA4306D1D163
:1067C00081EA030101F000414FF0000070BD50EA82
:1067D000410606BF1046194652EA430619D094EA0C
:1067E0000C0F02D150EA013613D195EA0C0F05D1F6
:1067F00052EA03361CBF104619460AD181EA03014A
:1068000001F0004141F0FE4141F470014FF0000001
:1068100070BD41F0FE4141F4780170BD70B54FF09C
:10682000FF0C4CF4E06C1CEA11541DBF1CEA13551C
:1068300094EA0C0F95EA0C0F00F0A7F8A4EB0504FE
:1068400081EA030E52EA03354FEA013100F08880F5
:106850004FEA03334FF0805545EA131343EA1263BE
:106860004FEA022245EA111545EA10654FEA002673
:106870000EF000419D4208BF964244F1FD0404F52C
:10688000407402D25B084FEA3202B61A65EB030588
:106890005B084FEA32024FF480104FF4002CB6EB45
:1068A000020E75EB030E22BFB61A754640EA0C00C5
:1068B0005B084FEA3202B6EB020E75EB030E22BF05
:1068C000B61A754640EA5C005B084FEA3202B6EB46
:1068D000020E75EB030E22BFB61A754640EA9C0005
:1068E0005B084FEA3202B6EB020E75EB030E22BFD5
:1068F000B61A754640EADC0055EA060E18D04FEA93
:10690000051545EA16754FEA06164FEAC30343EA32
:1069100052734FEAC2025FEA1C1CC0D111F4801FFF
:106920000BD141EA00014FF000004FF0004CB6E7F8
:1069300011F4801F04BF01430020B4F1FD0C88BF97
:10694000BCF5E06F3FF6AFAEB5EB030C04BFB6EBA2
:10695000020C5FEA500C50F1000041EB045170BD95
:106960000EF0004E4EEA113114EB5C04C2BFD4EBC2
:106970000C0541EA045170BD41F480114FF0000E46
:10698000013C90E645EA060E8DE60CEA135594EAC2
:106990000C0F08BF95EA0C0F3FF43BAF94EA0C0FC5
:1069A0000AD150EA01347FF434AF95EA0C0F7FF43A
:1069B00025AF104619462CE795EA0C0F06D152EA8E
:1069C00003353FF4FDAE1046194622E750EA410672
:1069D00018BF52EA43067FF4C5AE50EA41047FF483
:1069E0000DAF52EA43057FF4EBAE12E74FF0FF3CE8
:1069F00006E000BF4FF0010C02E000BF4FF0010CB9
:106A00004DF804CD4FEA410C7FEA6C5C4FEA430C31
:106A100018BF7FEA6C5C1BD001B050EA410C0CBF80
:106A200052EA430C91EA030F02BF90EA020F0020E2
:106A3000704710F1000F91EA030F58BF994208BF49
:106A400090422CBFD8176FEAE37040F00100704706
:106A50004FEA410C7FEA6C5C02D150EA013C07D15D
:106A60004FEA430C7FEA6C5CD6D152EA033CD3D0A8
:106A70005DF8040B704700BF8446104662468C46A2
:106A80001946634600E000BF01B5FFF7B7FF0028D5
:106A900048BF10F1000F01BD4DF808EDFFF7F4FFFE
:106AA0000CBF012000205DF808FB00BF4DF808ED89
:106AB000FFF7EAFF34BF012000205DF808FB00BFAC
:106AC0004DF808EDFFF7E0FF94BF012000205DF8CE
:106AD00008FB00BF4DF808EDFFF7CEFF94BF012083
:106AE00000205DF808FB00BF4DF808EDFFF7C4FF7C
:106AF00034BF012000205DF808FB00BF4FEA410CC5
:106B00007FEA6C5C02D150EA013C0AD14FEA430CA7
:106B10007FEA6C5C02D152EA033C02D14FF00000E4
:106B200070474FF0010070474FEA410212F5001222
:106B300015D211D56FF47873B3EB625212D94FEAC4
:106B4000C12343F0004343EA505311F0004F23FAAE
:106B500002F018BF404270474FF00000704750EA03
:106B6000013005D111F0004008BF6FF000407047C0
:106B70004FF00000704700BF4FEA4102B2F1E0431E
:106B800024BFB3F5001CDCF1FE5C0DD901F0004C14
:106B90004FEAC0024CEA5070B2F1004F40EB830064
:106BA00008BF20F00100704711F0804F21D113F190
:106BB0003872BCBF01F00040704741F480114FEAC9
:106BC0005252C2F11802C2F1200C10FA0CF320FA52
:106BD00002F018BF40F001004FEAC1234FEAD3236F
:106BE00003FA0CFC40EA0C0023FA02F34FEA4303D9
:106BF000CCE77FEA625307D150EA01331EBF4FF062
:106C0000FE4040F44000704701F0004040F0FE407C
:106C100040F40000704700BF80F0004002E000BF79
:106C200081F0004142001FBF5FEA410392EA030F77
:106C30007FEA226C7FEA236C6AD04FEA1262D2EBC1
:106C40001363C1BFD218414048404140B8BF5B42C6
:106C5000192B88BF704710F0004F40F4000020F05F
:106C60007F4018BF404211F0004F41F4000121F075
:106C70007F4118BF494292EA030F3FD0A2F10102BF
:106C800041FA03FC10EB0C00C3F1200301FA03F1FD
:106C900000F0004302D5494260EB4000B0F5000F20
:106CA00013D3B0F1807F06D340084FEA310102F1DF
:106CB0000102FE2A51D2B1F1004F40EBC25008BF91
:106CC00020F0010040EA03007047490040EB00005B
:106CD000013A28BFB0F5000FEDD2B0FA80FCACF15C
:106CE000080CB2EB0C0200FA0CF0AABF00EBC25089
:106CF00052421843BCBFD0401843704792F0000F77
:106D000081F4000106BF80F400000132013BB5E7C9
:106D10004FEA41037FEA226C18BF7FEA236C21D03F
:106D200092EA030F04D092F0000F08BF08467047A4
:106D300090EA010F1CBF0020704712F07F4F04D172
:106D4000400028BF40F00040704712F100723CBF85
:106D500000F50000704700F0004343F0FE4040F4AF
:106D6000000070477FEA226216BF08467FEA23636D
:106D70000146420206BF5FEA412390EA010F40F458
:106D8000800070474FF0000304E000BF10F00043A4
:106D900048BF40425FEA000C08BF704743F096438B
:106DA00001464FF000001CE050EA010208BF7047A6
:106DB0004FF000030AE000BF50EA010208BF70472D
:106DC00011F0004302D5404261EB41015FEA010C42
:106DD00002BF84460146002043F0B64308BFA3F13A
:106DE0008053A3F50003BCFA8CF2083AA3EBC2531C
:106DF00010DB01FA02FC634400FA02FCC2F120023B
:106E0000BCF1004F20FA02F243EB020008BF20F071
:106E10000100704702F1200201FA02FCC2F12002D7
:106E200050EA4C0021FA02F243EB020008BF20EACC
:106E3000DC7070474FF0FF0C1CEAD0521EBF1CEAFA
:106E4000D15392EA0C0F93EA0C0F6FD01A4480EAE8
:106E5000010C400218BF5FEA41211ED04FF00063D1
:106E600043EA501043EA5111A0FB01310CF00040FD
:106E7000B1F5000F3EBF490041EAD3715B0040EA23
:106E8000010062F17F02FD2A1DD8B3F1004F40EBF3
:106E9000C25008BF20F00100704790F0000F0CF0C6
:106EA000004C08BF49024CEA502040EA51207F3A8A
:106EB000C2BFD2F1FF0340EAC250704740F4000065
:106EC0004FF00003013A5DDC12F1190FDCBF00F056
:106ED00000407047C2F10002410021FA02F1C2F104
:106EE000200200FA02FC5FEA310040F1000053EAA0
:106EF0004C0308BF20EADC70704792F0000F00F0EE
:106F0000004C02BF400010F4000F013AF9D040EAF3
:106F10000C0093F0000F01F0004C02BF490011F487
:106F2000000F013BF9D041EA0C018FE70CEAD15385
:106F300092EA0C0F18BF93EA0C0F0AD030F0004C05
:106F400018BF31F0004CD8D180EA010000F00040B9
:106F5000704790F0000F17BF90F0004F084691F077
:106F6000000F91F0004F14D092EA0C0F01D14202B1
:106F70000FD193EA0C0F03D14B0218BF084608D17A
:106F800080EA010000F0004040F0FE4040F40000C4
:106F9000704740F0FE4040F4400070474FF0FF0C57
:106FA0001CEAD0521EBF1CEAD15392EA0C0F93EA9E
:106FB0000C0F69D0A2EB030280EA010C49024FEAF0
:106FC000402037D04FF0805343EA111143EA1013A9
:106FD0000CF000408B4238BF5B0042F17D024FF461
:106FE000000C8B4224BF5B1A40EA0C00B3EB510F3C
:106FF00024BFA3EB510340EA5C00B3EB910F24BF25
:10700000A3EB910340EA9C00B3EBD10F24BFA3EBA9
:10701000D10340EADC001B0118BF5FEA1C1CE0D171
:10702000FD2A3FF650AF8B4240EBC25008BF20F024
:10703000010070470CF0004C4CEA50207F32C2BF78
:10704000D2F1FF0340EAC250704740F400004FF015
:107050000003013A37E792F0000F00F0004C02BF46
:10706000400010F4000F013AF9D040EA0C0093F010
:10707000000F01F0004C02BF490011F4000F013B6A
:10708000F9D041EA0C0195E70CEAD15392EA0C0FD2
:1070900008D142027FF47DAF93EA0C0F7FF470AF0A
:1070A000084676E793EA0C0F04D14B023FF44CAF4D
:1070B00008466EE730F0004C18BF31F0004CCAD1E2
:1070C00030F000427FF45CAF31F000437FF43CAF1E
:1070D0005FE700BF4FF0FF3C06E000BF4FF0010C40
:1070E00002E000BF4FF0010C4DF804CD4FEA400222
:1070F0004FEA41037FEA226C18BF7FEA236C11D06C
:1071000001B052EA530C18BF90EA010F58BFB2EB1E
:10711000030088BFC81738BF6FEAE17018BF40F09E
:10712000010070477FEA226C02D15FEA402C05D152
:107130007FEA236CE4D15FEA412CE1D05DF8040BD7
:10714000704700BF844608466146FFE70FB5FFF76A
:10715000C9FF002848BF10F1000F0FBD4DF808ED22
:10716000FFF7F4FF0CBF012000205DF808FB00BF13
:107170004DF808EDFFF7EAFF34BF012000205DF86D
:1071800008FB00BF4DF808EDFFF7E0FF94BF0120BA
:1071900000205DF808FB00BF4DF808EDFFF7D2FFB7
:1071A00094BF012000205DF808FB00BF4DF808EDFA
:1071B000FFF7C8FF34BF012000205DF808FB00BFC7
:1071C00053B94AB9002908BF00281CBF4FF0FF314E
:1071D0004FF0FF3000F074B9ADF1080C6DE904CE4A
:1071E00000F006F8DDF804E0DDE9022304B07047A2
:1071F0002DE9F047089E0D4604468846002B4DD1E8
:107200008A42944668D9B2FA82F252B101FA02F384
:10721000C2F1200120FA01F10CFA02FC41EA030854
:1072200094404FEA1C45210CB8FBF5FE1FFA8CF781
:1072300005FB1E8341EA03430EFB07F199420BD97C
:107240001CEB03030EF1FF3080F01E81994240F2E7
:107250001B81AEF1020E63445B1AA4B2B3FBF5F0DE
:1072600005FB103344EA034400FB07F7A7420AD9A1
:107270001CEB040400F1FF3380F00881A74240F2C8
:10728000058164440238E41B40EA0E4000211EB12F
:10729000D4400023C6E90043BDE8F0878B4208D9FB
:1072A000002E00F0EE800021C6E900050846BDE88A
:1072B000F087B3FA83F100294AD1AB4202D382426C
:1072C00000F2F980841A65EB030301209846002E32
:1072D000E2D0C6E90048DFE702B9FFDEB2FA82F287
:1072E000002A40F09180A1EB0C054FEA1C471FFAE1
:1072F0008CFE0121B5FBF7F307FB1350250C45EA83
:1073000000450EFB03F0A84208D91CEB050503F16C
:10731000FF3802D2A84200F2CB8043462D1AA4B215
:10732000B5FBF7F007FB105544EA05440EFB00FEE1
:10733000A64508D91CEB040400F1FF3502D2A6458E
:1073400000F2BB802846A4EB0E0440EA03409EE70F
:10735000C1F120078B4022FA07FC4CEA030C20FA0B
:1073600007F405FA01F31C43FD404FEA1C4900FAFB
:1073700001F3B5FBF9F8200C1FFA8CFE09FB185538
:1073800040EA054508FB0EF0A84202FA01F20BD9CB
:107390001CEB050508F1FF3A80F08880A84240F216
:1073A0008580A8F1020865442D1AA4B2B5FBF9F056
:1073B00009FB105544EA054500FB0EFEAE4508D911
:1073C0001CEB050500F1FF346CD2AE456AD90238DA
:1073D000654440EA0840A0FB0294A5EB0E05A542D7
:1073E000C846A64656D353D05EB1B3EB080265EB50
:1073F0000E0505FA07F722FA01F3CD401F43C6E94F
:1074000000750021BDE8F087C2F1200320FA03F1E6
:107410000CFA02FC25FA03F395400D434FEA1C4792
:107420001FFA8CFEB3FBF7F107FB11302B0C43EA7C
:10743000004301FB0EF0984204FA02F408D91CEB59
:10744000030301F1FF382FD298422DD9023963444A
:107450001B1AADB2B3FBF7F007FB103345EA034547
:1074600000FB0EF3AB4208D91CEB050500F1FF3819
:1074700016D2AB4214D902386544ED1A40EA0141F4
:1074800038E73146304607E78646E5E61846FAE62D
:107490004B45A9D2B9EB020864EB0C0E0138A3E707
:1074A0004046EAE7204694E74146D1E7D0467BE7ED
:1074B000023B654432E7084609E76444023842E784
:1074C000704700BF10B59AB04822002108A822F0EA
:1074D000FDFD1822002102A822F0F8FD0EF0DCF8D4
:1074E0004FF0B0420024D2F8903023F01803C2F8D5
:1074F0009030D2F8003423F4C06343F40073C2F830
:107500000034D2F80034119403F4C06301934FF4B3
:107510008072019B0C922E234022089381230B93AF
:107520000D920123B02208A8CDE90E3410931292D7
:1075300013940DF057FC08B100F07CFB4F2302219F
:1075400002A8CDE90234CDE90444CDE906440DF0AA
:10755000EBFE08B100F06EFB1AB010BD13B5037856
:10756000082B2DD8DFE803F013848B2C9494052C82
:107570009A00047920460AF065F9204605F0C2FF1A
:107580000021204602B0BDE810400AF063B9002097
:107590000AF058F9012826D101200AF053F90128F0
:1075A00004D001200BF026FE00282ADC02200AF07D
:1075B00049F9012804D002200BF01CFE00283BDC16
:1075C00002B010BD012201A900200BF0DBFC00205D
:1075D0000AF038F9044630B90BF0E8FD48B99DF8D7
:1075E000041005F0FBFE00200BF004FE0028E9DC8F
:1075F000D2E70128F7D19DF8041020460BF030FDAA
:10760000F1E7012201A910460BF0BCFC01200AF0B1
:1076100019F90028C5D101200BF0C8FD28B99DF843
:107620000410012005F0DAFEBBE70128B9D19DF86E
:1076300004100BF015FDB4E7012201A902200BF0A4
:10764000A1FC02200AF0FEF80028B4D102200BF0C1
:10765000ADFD28B99DF80410022005F0BFFEAAE791
:107660000128A8D19DF8041002200BF0F9FCA2E734
:1076700014F06CFA02B0BDE8104002F0BFBC0A4B37
:107680001B68002B9CD0406802B0BDE81040184732
:10769000406802B0BDE810400BF046BE406802B042
:1076A000BDE810400BF0F6BAF823002030B5284BA7
:1076B000284A9A6085B00BF0C7FEFFF703FF4FF032
:1076C000B0430B209A6C42F004029A649A6C02F068
:1076D00004020392039A9A6C42F001029A649B6C32
:1076E000002203F0010311460293029B0DF02CFFD0
:1076F0000B200DF05BFF0BF00BFE0BF041F90AF0D5
:1077000051F9002401460546234603220120CDE914
:1077100000440BF077FB2346032229460220CDE9E3
:1077200000440BF06FFB0AF0DBF903F09BFAE5B2C3
:1077300028460AF087F810B9284605F0E3FE013420
:10774000032CF4D105B0BDE830400BF0C7BD00BF3D
:1077500000ED00E000600008F7B5FFF7A7FF224E3C
:10776000224C05F026FF224B341B142747430025EB
:107770001C44BD4216D320F03BFB1E480BF0C6FB59
:1077800001F068FE012822D0022822D010B91A4840
:107790000BF0BCFB194C0BF0AFFD2378DBB920F0EC
:1077A00029FBF8E701AA042160190BF02BF901A9C4
:1077B0003246042312F801CB11F8010B844518BF9F
:1077C00002F8010C013BF5D104350436D1E70C4831
:1077D000DEE70C48DCE70AF07DF80028DBD000206B
:1077E0000BF0DAFAD7E700BF8C0100200000002080
:1077F000200C0308E6D50208FAD50208BC0D0020CB
:1078000006D6020811D602080D48854620F093FCE2
:107810000C480D490D4A002302E0D458C4500433EB
:10782000C4188C42F9D30A4A0A4C002301E01360C1
:107830000432A242FBD322F0CDFBFFF78DFFFEE71F
:1078400000FC002000000020A00D0020200C0308F8
:10785000A00D0020A873002000F05AB80368074A62
:10786000934206D1DA69D20606D510221A6200F0D8
:107870004FBC034A9342F5D0704700BF00800040E0
:10788000003801404FF0B0434FF0FF319A6B9963DD
:10789000DA6BD9639A6B00229A63D86BDA63186C3F
:1078A0001964186C1A64586C5964586C5A64986A54
:1078B0009962986A9A62D86AD962D86ADA62186B51
:1078C0001963196B1A635A6C42F001025A645A6CBC
:1078D00022F001025A64D3F8902042F48032C3F8B7
:1078E0009020D3F8902022F48032C3F89020BFF388
:1078F0004F8F0549054BCA6802F4E0621343CB6021
:10790000BFF34F8F00BFFDE700ED00E00400FA0574
:107910004FF0B0434FF0FF319A6B9963DA6BD96344
:107920009A6B00229A63D86BDA63186C1964186C2E
:107930001A64586C5964586C5A64986A9962986AC7
:107940009A62D86AD962D86ADA62186B1963196BBD
:107950001A635A6C42F001025A645A6C22F0010216
:107960005A64D3F8902042F48032C3F89020D3F8C0
:10797000902022F48032C3F89020FEE7FEE7FEE775
:10798000FEE7704770470BF075BD0000014812F02C
:1079900057BD00BFC00D002001480FF0B4BA00BFB2
:1079A000946F0020014812F01BBF00BFC00D0020E3
:1079B00001480EF041B800BFC012002001480EF08F
:1079C0003BB800BFF80D002001480EF035B800BFED
:1079D000580E002001480EF02FB800BF20130020E1
:1079E00010B5044C20460CF079FA2046BDE8104052
:1079F000FFF734BF10140020704701200EF0B2B919
:107A000002200EF0AFB904200EF0ACB908200EF041
:107A1000A9B910200EF0A6B90E4BDA68920602D56D
:107A200020200EF09FB9DA68500601D54020F8E713
:107A3000DA68110601D58020F3E7DA68D20502D5AD
:107A40004FF48070EDE7DB689B0502D54FF40070C2
:107A5000E7E7704700080058134BDA68510503D573
:107A60004FF480600EF07EB9DA68120502D54FF44B
:107A70000060F7E7DA68D00402D54FF48050F1E7F0
:107A8000DA68910402D54FF40050EBE7DA6852044B
:107A900002D54FF48040E5E7DB681B0402D54FF4C4
:107AA0000040DFE7704700BF0008005810B5044CE5
:107AB00020460CF013FA2046BDE81040FFF7CEBE7A
:107AC0008013002001480EF0F5BA00BFD015002049
:107AD00001480EF07BBF00BFD0150020014810F018
:107AE000B3B800BF2016002000B58DB02C220021B5
:107AF00001A822F0EBFA1748174B03604FF08042C1
:107B00000023C0E90433C0E90723836083614FF495
:107B10008073436212F012FD08B100F08BF80D483B
:107B200012F034FE08B100F085F84FF07C530022CB
:107B30000793084808924FF4807301A902920692B5
:107B40000B9312F057FD08B100F074F800200DB04F
:107B50005DF804FBC00D00200028004007B5074B6E
:107B60000DF106001B699847BDF806304FF47A7294
:107B700002FB0030002103B05DF804FB5005030850
:107B80007047704708B50A480FF06FFA0022114697
:107B90000C200DF0D9FC0C200DF008FD00220D206A
:107BA00011460DF0D1FCBDE808400D200DF0FEBCE3
:107BB000040000207047000038B5054D002415F87A
:107BC000013B0BB1FFF7DEFF0134042CF7D138BDC8
:107BD000B80E0020BFF34F8F0549064BCA6802F468
:107BE000E0621343CB60BFF34F8F00BFFDE700BFE0
:107BF00000ED00E00400FA054FF0B04382B09A6C4B
:107C000002439A649B6C18400190019B02B070473C
:107C100010B5064C0649802220460CF0ABFE2268C7
:107C2000136843F01003136010BD00BF80130020E1
:107C3000A014002008B5FFF7CDFF0000012810B503
:107C40000BD1094C0949802220460CF093FE226892
:107C5000136843F01003136010BD0228FCD1BDE887
:107C60001040FFF7D5BF00BF1014002028150020DA
:107C70002DE9F04385B0012B9DF830509DF83480FC
:107C800014BF00274FF40057012D04460E4639D08B
:107C9000032D3AD0002D3BD00025013AD2B2022A62
:107CA00038D85F4B53F82290012C65D10420FFF7A0
:107CB000A3FF2046FFF7A0FF002211460E200DF083
:107CC00043FC0E200DF072FC564B574883F80180A0
:107CD000564B0561C0E900360C240023C0E9029729
:107CE000C0E90543C0E907334362B8F1000F17D07C
:107CF000082383624FF4004383630CF0AFFDA0B10F
:107D0000FFF768FF4FF4C065C7E74FF48065C4E72D
:107D1000022A02D04FF00009C6E74FF08059C3E7AE
:107D2000C0F828800CF068FDE9E700213E480CF01F
:107D300005FF01460028E3D13B480CF024FF002852
:107D4000DED139480CF0DBFE0028D9D10120FFF745
:107D500075FF4FF44013019A3348009319460CF015
:107D600057FE0028CCD14FF0B042936843F4004353
:107D7000936005B0BDE8F083022CFAD1294B2C4C5E
:107D800083F802800420FFF737FF0120FFF734FF5C
:107D9000002211460B200DF0D7FB0B200DF006FC46
:107DA000244B2561C4E900360C2200232046C4E997
:107DB0000297C4E90523C4E90833A36263660CF0A3
:107DC0001BFD014600289BD120460CF0B7FE014662
:107DD000002895D120460CF0D6FE002890D12046F0
:107DE0000CF08DFE00288BD1FFF712FF4FF44013EB
:107DF000029304AB13E9060020460CF009FE0028AC
:107E00007FF47EAF0C4AD2F8803043F08053C2F842
:107E100080302268936843F480039360A3E700BF37
:107E200018D60208CC15002010140020003801409C
:107E30008013002000800040000800582DE9F34125
:107E40009DF820809DF824C0CDE9008C16461D4683
:107E500004460F46FFF70CFF064B0C20444318194D
:107E600001221A5547600672457280F80A8002B0F6
:107E7000BDE8F081A8150020022810B5044605D100
:107E800007480BF08BFF28B1FFF7A4FE012801D1B2
:107E90000448F6E70C20044B444300221A5510BD59
:107EA0008013002010140020A8150020012870B5B0
:107EB0000D461E4620D194B2144A5278013A012A46
:107EC00014D813480CF0DDF92246114833462946F0
:107ED0000CF002FC04460E480CF0F8F99CB1022CA0
:107EE00014BF6FF006006FF0050070BD0848224611
:107EF0000CF0F2FB0446F1E7022802D1054892B2E9
:107F0000F6E70020F1E72046EFE700BFCC150020A0
:107F10001014002080130020012802D1044800F032
:107F2000A9BF022801D10348F9E76FF006007047A6
:107F3000680000207C000020012807B507D1084810
:107F40000DF1070100F0DCFF03B05DF804FB02282F
:107F500003D104480DF10701F4E76FF00600F3E7E1
:107F6000680000207C000020012802D1034800F0B6
:107F7000BEBF022801D10248F9E77047680000201F
:107F80007C000020012802D1044800F017BF02281D
:107F900001D10348F9E76FF0060070476800002040
:107FA0007C000020F8B5224D224F00240C23224AE9
:107FB00063439B5CCBB1022C1BD1204E3368DA6942
:107FC000D103FCD4DA695202FCD51C480CF06BFDDD
:107FD00033681A4810221A621A6822F010021A60D6
:107FE0000BF0FDFEF06F0DF015FC0134032CDDD11C
:107FF000F8BD012CF9D108232B624FF480132B62BA
:1080000055E8003F43F0020345E80032002AF7D16B
:1080100057E8003F43F4800347E80032002AF7D1D5
:10802000074AD2F8803043F08063C2F88030DCE742
:108030000038014008380140A815002080130020B6
:108040000008005873B50B4C0B4E4FF0FF35012D57
:108050000BD923784BB133780193A37A0093227A1A
:10806000637A61680020FFF703FE0135022DEED12F
:1080700002B070BDA8150020CC15002070B51D4BB6
:1080800002689A42044615D10BF0A9FE1A4E00254B
:1080900016F8011B022001350BF0C0F8802DF7D136
:1080A000154916482A4600F098FE13492A462046EC
:1080B0000CF060FC2268124B9A4216D120460BF05D
:1080C0008EFE104E002516F8011B012001350BF025
:1080D000A5F8802DF7D10B490B482A4600F07DFE0C
:1080E00008492A4620460CF045FCBDE87040074888
:1080F0000BF0FCB800800040A01400207C000020A1
:1081000000380140281500206800002020150020BC
:10811000F8B52C4B02689A4204461DD10BF05FFE65
:10812000294B2A4F1B685D68C5F18005ADB200265A
:10813000B54239DC254926482A4600F04EFE802209
:10814000224920460CF016FC224B1A78012A03D152
:1081500000221A700AF018FE22681F4B9A421ED1A4
:1081600020460BF03CFE1D4B1D4F1B685D68C5F1A2
:108170008005ADB20026B5421DDC194919482A46D2
:1081800000F02BFE8022164920460CF0F3FB114B29
:108190001A78012A03D100221A700AF0F5FDBDE811
:1081A000F84011480BF0A2B817F8011B02200BF0A1
:1081B00035F80136BCE717F8011B01200BF02EF84B
:1081C0000136D8E700800040C0120020A014002033
:1081D0007C000020BC0E002000380140201300204D
:1081E00028150020680000202015002073B5314BB1
:1081F00000261E7003685A6A8DF807202E4A9342A3
:10820000054619D12D482E4C0CF063FC2D492662F1
:108210001523C4E9001320468023C4E90266C4E99B
:108220000436C4E906660DF083FA08B1FFF7D2FC04
:10823000EC67A562FFF7ECFC2A68234B9A421AD13F
:108240002248234C0CF045FC224A1123C4E90023A8
:10825000204600238022C4E90233C4E90423C4E990
:10826000063323620DF064FA0028DFD1EC670120A9
:10827000A562FFF7E3FC2C680F4B9C420DD19DF8E3
:10828000071002200AF0CAFF2B68A34205D112484A
:1082900001220DF1070100F0A0FD10480BF026F8B7
:1082A0000F4B1A781AB901221A700AF065FD02B054
:1082B00070BD00BF5A510020008000408013002094
:1082C000C0120020080002400038014010140020B5
:1082D00020130020440002407C00002020150020D4
:1082E000BC0E002008B5164B164A1A605A680AB927
:1082F000154A5A6000220121C3E90221C3E9042280
:10830000C3E906221A620E48102283F842200DF0BB
:10831000BBFD08B1FFF78EFC094800210EF096FB6B
:1083200008B1FFF787FC064800210EF0BBFB08B13F
:10833000FFF780FCBDE808404FF400100EF0DCBBF6
:10834000D0150020005800405C08700010B50446AD
:10835000FFF7C8FF014B01221A5510BD1C16002063
:1083600010B5044604480DF0E8FD08B1FFF762FCC3
:10837000024B00221A5510BDD01500201C160020FB
:1083800008B5164B9942164B20D8164A5A601B68FE
:1083900013B313480DF0D1FD11480DF075FD08B170
:1083A000FFF748FC0E4800210EF050FB08B1FFF724
:1083B00041FC0B4800210EF075FB08B1FFF73AFCB9
:1083C000BDE808404FF400100EF096BB064A9142FB
:1083D00094BF064A064AD9E708BD00BFA08601003F
:1083E000D0150020DB0A301090D003009F0D7000E4
:1083F0005C08700013B59DF81000002814BF4FF002
:1084000000700020009049000A480DF0AFFD50B9FF
:10841000084C20460EF015FB2028FAD105480EF036
:1084200013FB042803D16FF0030002B010BD00203D
:10843000FBE700BFD015002013B54FF0007000908F
:1084400049000A480DF0E4FD50B9084C20460EF0F2
:10845000F8FA2028FAD105480EF0F6FA042803D1DC
:108460006FF0030002B010BD0020FBE7D015002024
:108470007047000038B5054D002415F8013B0BB1DD
:10848000FFF730FF0134042CF7D138BD1C16002053
:108490000A4B00F11002C178197081785970417847
:1084A000997010F8041BD970904203F10403F2D1C3
:1084B000034B10221A800020704700BF2C170020A9
:1084C000900000202DE9F04FDFF8FC80DFF8FCC0C1
:1084D000DFF8FCB085B002AF0446164640460022E5
:1084E000C8E900C2C8E909223D8ED7F834A07960F6
:1084F0009946C8F80820C8F80CB0C8F81420C8F885
:108500002C200EF09BFF08B1FFF794FB2E480EF0D5
:10851000B8FF08B1FFF78EFB2C480422C8E900021F
:108520000022C8F80820002C3AD1C8F814400022D4
:1085300001212548C8F80CB0C8E90912C8F82C2058
:108540000EF07CFF08B1FFF775FB2B071DBF25F070
:108550000F041034A4B22C46A300073323F0070302
:10856000ADEB030D02AE22460021304621F0AEFDF8
:108570002A464946304621F081FD7A68FF23009360
:108580005346BAB91048224631460FF0F1F970B996
:108590000D480EF076FF98B90C37BD46BDE8F08F58
:1085A000012C0CBF20224022C8E90462BFE76FF013
:1085B0000600F1E72246314603480FF06DFAE6E780
:1085C000FFF738FB0020E7E72016002000180058CE
:1085D0003C17002021F00803102B10B501D02029F2
:1085E00013D10B4B00F11002C4781C7084785C70BE
:1085F00044789C7010F8044BDC70904203F1040343
:10860000F2D1044B0020198010BD6FF01F00FBE772
:108610003C1700204C17002007B5CDE900120022BE
:10862000034611461046FFF74DFF03B05DF804FB0B
:1086300070B586B004460D4616460021102202A8E9
:1086400021F044FD074B08491A8802A821F016FDC5
:10865000CDE90056234602AA00210120FFF732FF90
:1086600006B070BD900000202C17002070B586B0B9
:1086700004460D4616460021102202A821F026FDD0
:10868000074B08491A8802A821F0F8FC0121CDE91E
:108690000056234602AA0846FFF714FF06B070BD35
:1086A000900000202C17002008B5FFF793FFC0B200
:1086B00008BD08B510230A461946FFF7ADFFC0B242
:1086C00008BD70B51446054618460E46FFF7E0FE95
:1086D00023019BB2324619462846FFF7A9FFC0B2D4
:1086E00070BD70B51446054618460E46FFF7D0FE1D
:1086F00023019BB2324619462846FFF7B7FFC0B2A6
:1087000070BD4FF0B04382B0DA6C0243DA64DB6CC8
:1087100018400190019B02B0704700001FB514285B
:108720004FF00003CDE902330C460CD8092812D9CA
:108730000A380A280FD8DFE800F07B0E0E0E0E82F2
:108740000E0E74116D00FE2800F08380FF2800F0EB
:108750008280FD287AD06FF0030059E03F4A404BF9
:108760000193137843F0010313703E483E4A4FF0E3
:108770000043C0E900233D4B04221B688360426133
:1087800000230122C2614FF4805106220383C0E915
:108790000333C0E90933C0E90C12837680F8203036
:1087A00080F82C30836380F83C30C3640AF09AFE72
:1087B00008B1FFF73FFA2B480BF05EFA08B1FFF75C
:1087C00039FA0023274801A9CDE902330BF012F84A
:1087D00008B1FFF72FFA23480BF078F908B1FFF73B
:1087E00029FA0A211F480AF0A7FF1E480BF026FAB3
:1087F0001C480AF0FCFF1E4B019A80B29A4220806E
:1088000004BF00EB4000208016480BF0C3F90020A5
:1088100004B010BD114A174B0193137843F00203C3
:10882000A2E70E4A144B0193137843F004039BE72D
:108830000A4A124B0193137843F0080394E7074A5E
:108840000F4B0193137843F010038DE70D4B019309
:108850008BE70D4BFBE7064BF9E700BF4E170020F7
:10886000040000085017002000240140940000205C
:10887000004000B80800000C100000104000001874
:108880000008002C001000B0002000B470477047B2
:108890000128084A084B04D0022806D1107008228B
:1088A00001E0107010221A6070470321117000223D
:1088B000F9E700BF9900002094000020014B1878D0
:1088C000704700BF99000020014B1878704700BF27
:1088D0009800002010B5044686B01422002101A89B
:1088E00021F0F4FB22685E4B9A4240F08E804FF0FC
:1088F000B0435C4C1A6E42F400721A661B6E03F4AD
:1089000000730093009B2378DA0708D5132000F04A
:108910004BF9B0F1904F7AD10120FFF7F2FE2378A6
:108920009B0708D5142000F03FF9B0F1904F76D1A5
:108930000120FFF7E6FE2378580708D5122000F043
:1089400033F9B0F1904F72D10120FFF7DAFE2378AE
:10895000190708D50A2000F027F9B0F1904F6ED121
:108960000120FFF7CEFE2378DA0608D50F2000F0AD
:108970001BF9B0F1904F6AD10120FFF7C2FE00232E
:108980004FF0030CCDE902C32378DB0709D5132090
:1089900000F00FF90190132000F006F901A90DF085
:1089A000B5F82378980709D5142000F002F9019052
:1089B000142000F0F9F801A90DF0A8F82378590760
:1089C00009D5122000F0F5F80190122000F0ECF823
:1089D00001A90DF09BF823781A0709D50A2000F0A9
:1089E000E8F801900A2000F0DFF801A90DF08EF8F8
:1089F0002378DB0609D50F2000F0DBF801900F206B
:108A000000F0D2F801A90DF081F806B010BD1320D6
:108A100000F0CAF8144B984281D102207DE714205F
:108A200000F0C2F8104B984285D1022081E7122055
:108A300000F0BAF80C4B984289D1022085E70A2051
:108A400000F0B2F8084B98428DD1022089E70F2040
:108A500000F0AAF8044B984291D102208DE700BFA4
:108A6000002401404E1700200004004838B5334B65
:108A700002689A4260D14FF0B042314C136E23F439
:108A8000007313662378DD070ED5132000F08CF8F1
:108A90000546132000F08DF8014628460DF0E8F851
:108AA000237823F001032370237898070ED5142030
:108AB00000F07AF80546142000F07BF801462846BD
:108AC0000DF0D6F8237823F002032370237859079A
:108AD0000ED5122000F068F80546122000F069F863
:108AE000014628460DF0C4F8237823F004032370D0
:108AF00023781A070ED50A2000F056F805460A20FA
:108B000000F057F8014628460DF0B2F8237823F01C
:108B1000080323702378DB060ED50F2000F044F8FD
:108B200005460F2000F045F8014628460DF0A0F854
:108B3000237823F01003237038BD00BF00240140C8
:108B40004E170020034B00221A70034B01221A70AB
:108B5000704700BF5A51002058510020024B53F873
:108B6000203003B118477047B41F002000220123B2
:108B70000342D1B202F101020DD02F290ED8084BC9
:108B8000084800221A70082300F8313000EBC100B9
:108B900041600AF0ABBB5B009BB2E9E7704700BFE6
:108BA0005A510020341F0020000900F59010800267
:108BB000704700F00F030120984080B2704700001A
:108BC0002F28F8B5054600F28280414E1422424318
:108BD00000F00F040123B018A340B35003294FF055
:108BE0000202C2602DD801292ED94FF488124260AA
:108BF0002846FFF7D9FFC76893FAA3F2B2FA82F2C8
:108C0000510003228A403A4093FAA3F3B3FA83F364
:108C10005B0022FA03F3012B4FF014021ED0022B4B
:108C20001CD0142101FB05610CF070FFD4B90620A3
:108C3000224602210CF088FC0620BDE8F8400CF02A
:108C4000B5BC0439012906D9142202FB05624FF490
:108C500044115160CCE74FF40412C8E702FB0562EF
:108C60009360DEE7012C06D10720002202210CF0E0
:108C70006BFC0720E1E7022C06D1082000222146E8
:108C80000CF062FC0820D8E7032C06D10920002252
:108C900002210CF059FC0920CFE7042C06D10A2050
:108CA000002202210CF050FC0A20C6E7053C042CEF
:108CB0004FF000024FF0020104D816200CF044FCE3
:108CC0001620BAE729200CF03FFC2920B5E7F8BDB3
:108CD000B4170020044B00F00F0053F820200AB90D
:108CE00043F8201000207047B41F00202DE9F843FE
:108CF000174E184D184FDFF86480DFF86490002499
:108D00000F2C05DDA4F11203052B01D91C2C15D164
:108D100057F8243093B973682B60B3686B60F368BD
:108D2000AB603369EB602B7C43B198F800102046B0
:108D3000FFF746FF49462046FFF7CCFF0134302CB1
:108D400006F1140605F11405DAD1BDE8F88300BF79
:108D5000B4170020741B0020B41F00209A000020CC
:108D6000458B0008F8B5124E124D134F00240F2CFE
:108D700005DDA4F11203052B01D91C2C10D157F8E5
:108D800024306BB933686B607368AB60B368EB60B9
:108D90002046F3682B612946FFF706FF0CF0B6FE6C
:108DA0000134302C06F1140605F11405DFD1F8BDAD
:108DB000741B0020B4170020B41F0020C268036990
:108DC0009A4282BF40681B180133981A704708B551
:108DD0004168FFF7F3FF081A08BD2DE9F743044681
:108DE00001A8164688460AF08BFA2046FFF7EFFFE7
:108DF000864228BF06462046FFF7E9FFE36825695B
:108E0000A268AB429CBF636801335D1B8146236946
:108E10002068AE4202FB030013D87243414621F0A2
:108E20002DF9236962683344934296BF2369002376
:108E30009B19236101A80AF065FA304603B0BDE82A
:108E4000F08305FB02F73A46414621F017F9A26884
:108E50002068751B6A4308EB070121F00FF94E45A6
:108E60002561E7D923696268934234BF0133002347
:108E7000E360DFE72DE9F341044601A81646884682
:108E80000AF03EFA2046FFF799FFE768E568236994
:108E9000A2682168864228BF06469D4284BF636857
:108EA00001335D1BAE4202FB071110D872434046EE
:108EB00021F0E4F862683744974288BF0027E760F2
:108EC00001A80AF01FFA304602B0BDE8F08105FBA8
:108ED00002F73A46404621F0D1F8A2682168751B96
:108EE0006A4308EB070021F0C9F8E560E8E710B530
:108EF00004461422002121F0E9F82369E36010BD43
:108F000010B504460846E26823699A4223D0A26855
:108F1000E1682368541E072C18D8DFE804F0040821
:108F2000170C171717105B5C0370002010BD33F887
:108F300011300380F9E753F821300360F5E703EBC4
:108F4000C103D3E90023C0E90023EEE701FB0231AE
:108F500021F094F8E9E76FF00E00E7E7704710B5ED
:108F600086B00A2301A88DF8043014F09DF9044658
:108F700001A814F099F9201E18BF0120404206B044
:108F800010BD10B513F076FC0128044604D030B9AA
:108F90000AF0C8F9204610BD6FF00500FBE76FF03E
:108FA0000600F8E738B50B78013B044615461A4829
:108FB000092B2CD8DFE803F0052B2B1B23272B2BA9
:108FC0002B1F09F0A3FF154809F0A0FF144809F072
:108FD0009DFF144B144853F8241009F097FF0B2CF5
:108FE00019D129461148BDE8384009F08FBF09F072
:108FF0008DFF0F48E8E709F089FF0E48E4E709F024
:1090000085FF0D48E0E709F081FF0C48DCE709F037
:109010007DFF0B48D8E738BD24D602085AD602088F
:109020008FD6020828DE0208CDD70208DFD7020853
:10903000C4D60208F9D602082ED7020863D7020860
:1090400098D7020838B50B78012B0446154607D08F
:10905000032B1CD003BB134809F058FF124803E050
:10906000104809F053FF114809F050FF104809F06B
:109070004DFF104B104853F8241009F047FF0B2CFC
:109080000FD129460D48BDE8384009F03FBF0548DB
:1090900009F03CFF0A48E7E7024809F037FF0948B2
:1090A000E2E738BDF7D7020862D802082DD80208D7
:1090B0008FD6020828DE0208CDD70208DFD70208C3
:1090C00097D80208CCD8020870B5474E8AB004463B
:1090D000052556F8043B1BB11B6A0BB12046984787
:1090E000013D15F0FF05F4D123780B2B0FD00F2B8A
:1090F0000BD13E4809F00AFF3D4B8DF8045001A802
:109100001D708DF8085013F0FDFC0AB070BD637837
:109110000E2B63D1374809F0F9FE354B1A78042A33
:109120001BD0022628461E700AF0FCF832492A4657
:1091300028460AF0F3F8B8B921F0FEFC434203F0E8
:109140001F0300F01F004FF47A7158BF584200FB14
:109150000111324628460AF0E3F8637D032B1FD83D
:10916000DFE803F00B24272A4FF42571234809F088
:10917000CDFE28460AF0D6F8EFE7214A00231380F7
:10918000E37D217E1B0243EA0143A17D0B43536033
:10919000A37EE17E1B0243EA0143617E0B439360A1
:1091A000D4E90101174B83E80300AEE7144A012319
:1091B000E5E7134A0223E2E7E37D217E104A1B0222
:1091C00043EA0143A17D0B43D360A37EE17E1B02F2
:1091D00043EA0143617E0B431361E1E70F2BDFD1CB
:1091E000094809F093FEDBE76821002001D9020855
:1091F000CC2100200CD90208019A000819D90208D4
:10920000B0210020C421002029D9020870B5164BD6
:10921000164A1B680446407860B92179117003B181
:1092200098472378012B1CD123792BB1104809F0E2
:109230006DFE05E00021F1E761780E4809F066FE59
:10924000002002F0EDFD0C4E052556F8043B1BB145
:109250005B690BB120469847013D15F0FF05F4D13D
:1092600070BD0648E3E700BF04240020D32200209D
:1092700036D902084FD902086821002070D90208A7
:1092800008F05EBC08F084BC08F0FABC08B519F020
:10929000C5FF08BD08F052BD072801D808F054BD2D
:1092A0006FF00200704708F05BBD08F05FBD000082
:1092B000014B1878704700BFD322002008F010BC83
:1092C0007FB5054608F00CFC431EDBB2012B0446BB
:1092D00003D900F0FD03082B1DD101A808F012FCF2
:1092E000002201A91346012011F8016B1EB100FAFA
:1092F00002F633439BB201320C2AF5D104F0FD0291
:10930000082A01D0012C02D123F480739BB22B8058
:10931000002004B070BD6FF00200FAE7F0B58FB026
:1093200006460F4608F0DCFBFF23ADF804304FF48F
:109330007F43ADF80630431EDBB20024012BCDE99C
:1093400002440546049403D900F0FD03082B7ED1A6
:10935000FFF717FE044600286FD1338823B9012D8B
:1093600050D140F2FF1333800C22002102A820F0DC
:10937000ADFE3088002240FA02F1CE07D3B20ED5FE
:109380000EAE03F0FE0103F00103314406EB43038C
:1093900031F8306C33F8343C334321F8303C01323F
:1093A0000C2AE8D105F0FD03082B01D0012D0ED1C8
:1093B000BDF81030002203F47F43ADF810301146A1
:1093C0000126D5B2072D28D909B1ADF810302323D5
:1093D0008DF8143005A802AB069313F093FB0546F5
:1093E00068B924238DF8143005A802AB069313F056
:1093F00089FB08F06BFED8B913F034FA00B36FF0B4
:1094000006041AE005F0FD03082B04BFFF23338098
:10941000022DA9D140F6FF73A5E740FA02F5ED074A
:1094200041BF06FA02F10B439BB201210132C8E7AA
:10943000284608F051FE0028DED020460FB0F0BDCF
:10944000002FFAD002A808F067FB0446F5E76FF09A
:109450000204F2E708B508F095FCC0B208BD022886
:1094600008B503D808F094FC002008BD6FF0060092
:10947000FBE708F099BC00B58BB0012301A88DF87B
:10948000043013F063FA38B99DF80800003818BFAB
:1094900001200BB05DF804FB0020FAE730B58BB07B
:1094A00005460C4608F080FC30B9214628460BB032
:1094B000BDE8304008F094BB0F2C03D86FF00600D5
:1094C0000BB030BDFFF7D7FF044630B9014610227C
:1094D000284620F0FBFD2046F2E70F2301A88DF877
:1094E000043013F033FA04460028E7D10299102221
:1094F000284620F0C3FDEEE730B58BB005460C469C
:1095000008F052FC30B9214628460BB0BDE8304087
:1095100008F08EBB032C03D86FF006000BB030BDF3
:10952000FFF7A9FF044630B901460422284620F07F
:10953000CDFD2046F2E7072301A88DF8043013F093
:1095400005FA0028E8D1029B1BBA2B60E6E730B58C
:109550008BB005460C4608F027FC30B9214628465A
:109560000BB0BDE8304008F0B3BB032C03D86FF05C
:1095700006000BB030BDFFF77EFF044630B9014650
:109580000422284620F0A2FD2046F2E7062301A887
:109590008DF8043013F0DAF904460028E7D10422EC
:1095A00002A9284620F06AFDEEE730B58BB00546EB
:1095B0000C4608F0F9FB30B9214628460BB0BDE84F
:1095C000304008F093BB0F2C03D86FF006000BB0AF
:1095D00030BDFFF750FF044630B90146102228463F
:1095E00020F074FD2046F2E70E2301A88DF8043028
:1095F00013F0ACF904460028E7D10299102228465E
:1096000020F03CFDEEE708F0E1BB08F0F1BB08B547
:1096100008F076FE003818BF012008BD38B50C46AA
:10962000054613F0A7FF24B12846BDE8384008F0EE
:109630005BBE204638BD00B58BB02C2301A88DF849
:10964000043013F083F99DF808000BB05DF804FBBB
:1096500008F004BC08F014BC08F036BC00B58BB0B0
:1096600008F0A2FB01280DD1FFF705FF50B1272319
:1096700001A88DF8043013F069F900B902980BB015
:109680005DF804FB0BB05DF804EB08F02FBC08F0AC
:109690003FBC08F04FBC08F071BC08F075BC1FB5AA
:1096A0002F238DF8083008F01BFA02A917F03FFAB3
:1096B00005B05DF804FB1FB531238DF8083008F0C4
:1096C0000FFA02A917F033FA05B05DF804FB0000A9
:1096D000014B1868704700BFC4210020014BB3F94B
:1096E00000007047F4230020014B93F900007047FD
:1096F0000824002010B590B0044605A810F046FDDF
:10970000059807A9123810F0C9FD0C9B094903F20E
:109710006C7303930A9B02930B9B01330193079B8A
:1097200000932046DDE9083221F05CFA002010B0F9
:1097300010BD00BF7FD9020800B58BB01F2301A860
:109740008DF8043013F002F918B902980BB05DF8E7
:1097500004FB6FF00600F9E700B58BB01F2301A8EA
:109760008DF8043013F0F2F820B99DF80C000BB01E
:109770005DF804FBF920FAE708F0EEBB022801D8F7
:1097800008F0F0BB6FF00200704700002DE9F041D7
:1097900098B00D4602A981E80C00804608F03AFB1B
:1097A0000746FFF768FE0646002800F0058111F025
:1097B0003BFE044610B16FF0050093E008F018FB83
:1097C000022840F092808DF840000FA88DF83C40B0
:1097D00013F098F98DF8227008F0BEFB60B108F024
:1097E000BBFB012802D10020FFF7C8FF04230FA80C
:1097F0008DF83C3013F058FD724B1B78012B05D1CE
:109800000A230FA88DF83C3013F04EFD04A9E8B2EE
:1098100013F042F807461FF011FE60B19DF81030BA
:109820009DF811206849694851F82710D21A009212
:109830002A4609F06BFB002F76D000238DF81430F8
:109840000793ADF8203005A813F0E4FD05461FF09E
:10985000F5FD00283FD033230FA88DF83C3013F0DE
:1098600075F80FA813F072F8002834D1584F109BE8
:109870003A7893F84C6057484FF00C0808FB0233D5
:10988000D3F8E41309F042FB012E109A01D0082E00
:1098900073D13B78D2F8B4204F4903F0070301FBA2
:1098A00003214E4809F032FB109B4D48D3F8B41009
:1098B00009F02CFB109B4B4893F9451009F026FB4F
:1098C000109B494893F9441009F020FB109B47482E
:1098D000D96809F01BFB002D61D1002C0CBF6FF083
:1098E0000200002018B0BDE8F08108F081FA0128DC
:1098F0007FF470AF3E4B1B787BB1022B7FF46AAFD5
:10990000204609F00FFD0D238DF8283008F036FBB6
:1099100000F007008DF82C0002E00A238DF82830B3
:109920000AA813F0C1FC55E79DF808308DF81830EF
:109930009DF80930ADF82050CDF81C808BB19DF812
:109940000A308DF823309DF80B3083B19DF80C3030
:109950008BB900238DF81430264B00221A70344640
:1099600071E708F0EBF901308DF82300EBE708F020
:10997000F7F90028EDD00123ECE7022E397809D160
:109980003023B1FBF3F003FB1011CBB2D2F8B420BB
:10999000194984E708FB0121D1F8E41381E7A5F117
:1099A0000E03DBB2012B7FF606AF0B2D07D1099911
:1099B000124809F0ABFAFEE66FF00B0092E76FF089
:1099C00006008FE70924002028DE0208A1D902083A
:1099D000D02E0020F6D90208C0270900F3D90208CA
:1099E00005DA020817DA02082DDA020842DA02085C
:1099F000CC210020D3220020400D03004EDA0208C3
:109A00001FB500384FF0010318BF012000210322C9
:109A10008DF808308DF809308DF80B308DF80C007A
:109A20008DF80A20009104AB13E90C000248FFF7FF
:109A3000ADFE05B05DF804FB00DF02087FB501262E
:109A400003788DF808300C4605468DF8096008F05B
:109A500075F9B44230448DF80A008DF80B6002D1DC
:109A60008DF80C4001E0002CFAD00023009304ABE9
:109A700013E90C0069786868FFF788FE003818BFA2
:109A80000120404204B070BD2DE9F04F43788DB005
:109A90000446002B40F0AF80B0F90E007B4F7C4EA7
:109AA000237C388040B2337002F0C4FB237B002B50
:109AB0003BD0607C7749B7F9002051F8201096F927
:109AC00000307548DFF8D491DFF8D4A109F01EFA10
:109AD000A378012B0CBF7348734809F017FAE1789B
:109AE000724809F013FA4FF000085FFA88FB5846F5
:109AF00007F0A8FE054640B9227BEBB29A4200F27D
:109B0000AB805146584609F0CBF908F10108B8F18D
:109B1000030FEAD1227BA168654820F0AFFA654BBC
:109B2000227B1A70644BE2781A706379012B00F083
:109B30009B802378012B02D10020FFF761FF5F4B50
:109B40001A782AB3DFF8789100221A7099F8003059
:109B5000F3B996F900305B4DDFF86C8100932A78F9
:109B6000B7F9003098F80010584809F0CFF9584B71
:109B70001B686BB1574899F80020027098F80020D4
:109B800042702A7882703A8882803278827198474F
:109B9000E278E02A11D0504B1B6873B14F48027035
:109BA00022794270A2684260227B0272E28942817D
:109BB000227C0273626902619847494E052556F876
:109BC000043B1BB19B690BB120469847013D15F042
:109BD000FF05F4D1434890F8023163B180F8025197
:109BE0008DF80F508DF80D500095DDE90323B0F886
:109BF0000011FFF7CBFD1FF021FC50B3332303A866
:109C00008DF80C3012F0A2FE03A812F09FFE00287F
:109C100038D1637C73BB344809F078F9A1693348C3
:109C200009F074F9E178324809F070F9B4F90E10CE
:109C3000304809F06BF994F910102F4809F066F9D3
:109C400021792E4809F062F9049B2D48996909F0A1
:109C50005DF90DB0BDE8F08FA2684946D25C584668
:109C600009F01EF9013547E708F0C2F800287FF433
:109C700060AF61E7012B01D12248CDE7022BCDD1A6
:109C80002148C9E7214809F041F9E2E7F42300201F
:109C900008240020A8DE020866DA02088BDA02082F
:109CA000FEDE020877DA020882DA0208E8E102083A
:109CB000D4220020D4230020D5230020DE2300203E
:109CC000DF230020A82100206621002090DA02086E
:109CD000FC230020D623002000240020E0230020C5
:109CE00068210020CE210020AFDA02080CDB020838
:109CF0001EDB020828DB020832DB02083BDB02081D
:109D00004BDB0208CCDA0208E9DA020859DB020868
:109D1000014B1878704700BF0924002010B5044695
:109D2000FFF7A9FB28B1012C06D8054B00201C70B9
:109D300010BD6FF00B00FBE76FF00200F8E700BF0B
:109D40000924002008F02CB908F03CB908F04CB9FF
:109D500008F05CB970B5094E3478944228BF1446B7
:109D6000054622460846064920F088F9054B1A7830
:109D70002A7000221A703270204670BDD423002051
:109D8000D4220020D523002070B5044D0646044699
:109D90000FCD0FC42B682360304670BDB02100206A
:109DA000F0B591B0002604ACC4E9016605460496FE
:109DB00007F096FE431EDBB2012B0AD9082808D013
:109DC00005286AD00A2804D06FF00604204611B096
:109DD000F0BD15BB2046ADF81C5007F093FE0028DF
:109DE000F2D1BDF81C302A46012114F8010B20B134
:109DF00001FA05F213439BB2012201350C2DF4D177
:109E00000AB1ADF81C30002107A8FFF787FA044615
:109E10000028D9D108F060F9D8E71B2302A98DF8F2
:109E2000083016F084FE1E230190C6B207A88DF8F4
:109E30001C3012F08BFD089B0022A3F10C010C20BA
:109E4000D3B29E4203D859D16FF00204BEE701326B
:109E500000FB02F7CF59AF42F2D11A0910A901EB6A
:109E6000420203F00F03012101FA03F322F8303C10
:109E700007A823238DF81C30089412F043FE002815
:109E8000A2D1242307A808948DF81C3012F03AFEC2
:109E90000446002898D12846BCE7CDB90723ADF881
:109EA000103007A823238DF81C30089412F02AFEE6
:109EB000002889D1242307A88DF81C30089412F0BB
:109EC00021FE002880D1284608F006F904467DE7E7
:109ED0001E2307A88DF81C3012F038FD0899334670
:109EE0000C2000FB03F28A58AA4203D1012202FA95
:109EF00003F3D4E70133042BF3D1A5E7002465E78E
:109F000008B507F0EDFD431EDBB2012B03D900F0CD
:109F1000FD00082803D1BDE8084008F0D7B86FF06D
:109F2000060008BD08B5FFF7EBFF024658B1064B27
:109F3000064900209A4208BF042003F5C31303F525
:109F400020638B42F6D108BDC0AFD235C0FF953635
:109F500008B5FFF7D5FF024658B1064B0649002069
:109F60009A4208BF062003F5C31303F520638B4212
:109F7000F6D108BD6086973660D65A37FFF7C0BF66
:109F8000FFF7BEBF014B1878704700BFCC210020FF
:109F900038B50D46044610B14FF0FF3038BD03F020
:109FA00019FA0028F8D0094B09491860094B436297
:109FB000094B8362094BC362094B0363094B43633B
:109FC000F2224368284698472046E7E768210020A8
:109FD0007420002045900008A58F0008EDA6000819
:109FE0003D9A00085F8F0008034B53F820309868B3
:109FF00000B10047704700BF6821002038B50B4D05
:10A00000002455F8043BE4B24BB11B693BB1204638
:10A01000FFF7EAFF18B155F8043C1B699847013473
:10A02000E3B2052B64B2ECD138BD00BF682100203B
:10A0300000B58BB02F238DF8043001A819230293AB
:10A0400012F060FD0BB05DF804FB07F0F1BF07F004
:10A05000F5BF07F0FFBF08F003B808F00DB808F02F
:10A0600011B810B5044616F05DFD40B914B1143CAA
:10A07000022C04D8BDE81040002016F053BD10BDDE
:10A0800030B58BB00D46044607F02AFDFFF7E9FF17
:10A09000A0B1032301A88DF80430029412F032FD20
:10A0A00038B101280CBF6FF005006FF006000BB04F
:10A0B00030BD2946204607F051FDF8E76FF010004B
:10A0C000F5E730B58BB00D46044607F009FDFFF704
:10A0D000C8FFE8B1082301A88DF80430029412F0FB
:10A0E00011FD38B101280CBF6FF005006FF00600BC
:10A0F0000BB030BD092301A88DF80430029412F092
:10A1000001FD0028EED12946204607F04FFDEFE77C
:10A110006FF01000ECE730B58BB00D46044607F049
:10A12000DFFCFFF79EFFA0B10F2301A88DF80430DC
:10A13000029412F0E7FC38B101280CBF6FF0050063
:10A140006FF006000BB030BD2946204607F056FDE3
:10A15000F8E76FF01000F5E730B58BB00D46044618
:10A1600007F0BEFCFFF77DFFB0B107238DF8043088
:10A17000236801A81BBA029312F0C4FC38B101286D
:10A180000CBF6FF005006FF006000BB030BD294624
:10A19000204607F05BFDF8E76FF01000F5E730B5FB
:10A1A0008BB00D46044607F09BFCFFF75AFFD8B171
:10A1B00007F0E8FDC0B201280FD1022301A88DF8F5
:10A1C0000430029412F09EFC38B101280CBF6FF0ED
:10A1D00005006FF006000BB030BD294620460BB0DD
:10A1E000BDE8304007F05ABD6FF01000F3E730B51E
:10A1F0008BB00D46044607F073FCFFF732FF30B317
:10A200000C2301A88DF80430029412F07BFC38B1C5
:10A2100001280CBF6FF005006FF006000BB030BDD9
:10A220000D2301A88DF80430029412F06BFC002875
:10A23000EED10E2301A88DF80430029412F062FCD6
:10A240000028E5D12946204607F05EFDE6E76FF0DD
:10A250001000E3E72DE9F04393B004460E46904624
:10A260001F4607F0A1FD611C054629D1721C0AD0CA
:10A27000003E18BF012607F0A5FE864203D03046F7
:10A2800007F0A6FE50BBB8F1FF3F07D007F0ACFEC9
:10A29000804503D0404607F0ADFEF8B97B1C07D0DF
:10A2A00007F0B4FE874203D0384607F0B5FEA8B9E0
:10A2B000BCB9204609F036F8704B1C6000200DE058
:10A2C000B4F1000918BF4FF0010907F069FE81459C
:10A2D000CCD0484607F06AFE0028C7D013B0BDE8CE
:10A2E000F08307F0FDFBFFF7BCFE002800F0C28002
:10A2F000012D40F09080002368468DF824508DF8A1
:10A3000000508DF8043012F0FDFB0446002840F0A8
:10A31000838007F07FFD8DF8280009A812F0C4FFA4
:10A320000546002849D107F063FD012801D1544BAF
:10A330001D701FF083F80028D0D0332309A88DF8B2
:10A34000243012F003FB09A812F000FB0028B5D15D
:10A350004C4D0A9B2A7893F84C404B480C2606FB40
:10A360000233D3F8E41308F0D1FD012C0A9A01D08E
:10A37000082C6DD12B78D2F8B420444903F00703A0
:10A3800001FB0321424808F0C1FD0A9B4148D3F874
:10A39000B41008F0BBFD0A9B3F4893F9451008F044
:10A3A000B5FD0A9B3D4893F9441008F0AFFD0A9BA8
:10A3B0003B48D96808F0AAFD80E7012811D00B2896
:10A3C0002AD12E4E204608F0ADFF356801353560A4
:10A3D00007F01CFE854207D934600D99314808F01A
:10A3E00095FD6FF0050079E7224620462E4908F0DA
:10A3F00095FF044648B907F0F7FD4FF47A714143E1
:10A400002246204608F08CFFE7E74FF4E561274835
:10A4100008F07CFDE1E715B16FF006005EE701236F
:10A4200068468DF800308DF8043012F06BFB002880
:10A43000F2D107F0DDFC022807D18DF80400684650
:10A440008DF8005012F05EFB73E707F0D1FC70E767
:10A45000022C297809D13023B1FBF3F003FB101152
:10A46000CBB2D2F8B42012498AE706FB0121D1F819
:10A47000E41387E76FF0100030E700BFAC21002045
:10A48000CC210020D02E0020F6D90208C0270900D8
:10A49000F3D9020805DA020817DA02082DDA0208F1
:10A4A00042DA02084EDA0208B5A400087DDB020891
:10A4B000400D03004FF0FF331A4619460120FFF705
:10A4C000C9BE30B58BB00C46054607F009FBFFF757
:10A4D000C8FD88B1052301A88DF804308DF8085017
:10A4E00012F010FB03280AD001280BD06CB12846CB
:10A4F00007F072FC0BB030BD6FF01000FAE76FF0A0
:10A500000200F7E76FF00500F4E72046F2E70000ED
:10A5100030B58BB00C46054607F0E2FAFFF7A1FD17
:10A5200000283AD0FEF7A7FFB8B1002301A88DF8A4
:10A53000043012F00BFA10B16FF0060011E09DF834
:10A540000830012B1CD0022B22D0002BF4D1012D7E
:10A5500009D0022D0BD0002DEED10CB3284607F008
:10A560004DFC0BB030BD0F4B00221A70F5E70223F3
:10A570008DF8083001A812F0C5FA0028EDD0DBE70D
:10A58000012DF7D0022DF2D0002DD5D10023EFE719
:10A59000012DE8D0022DF7D1DFE76FF01000E0E7E2
:10A5A0002046DEE7CC21002070B58EB00E46054671
:10A5B00007F096FAFFF755FD002800F0948001237C
:10A5C0008DF81430002D4AD18DF8183005A812F0FE
:10A5D00099FA002847D101AC002D4FD11021204617
:10A5E00007F0FEFA0F2305A88DF81430069412F038
:10A5F00089FA002837D10421204607F019FB0723E8
:10A600008DF81430019B05A81BBA069312F07AFA54
:10A6100048BB1021204607F069FB0C2305A88DF8E4
:10A620001430069412F06EFAE8B90D2305A88DF8DF
:10A630001430069412F066FAA8B90E2305A88DF816
:10A640001430069412F05EFA68B907F0D1FB29467F
:10A65000FFF75EFF48B9002E41D1304605E005A85E
:10A6600012F074F918B16FF006000EB070BD9DF8CD
:10A670001830012B08BF8DF81800A7E708212046E5
:10A6800007F0FEFA022305A88DF81430069412F0A4
:10A6900039FA0028E7D10821204607F051FA0323B0
:10A6A00005A88DF81430069412F02CFA0028DAD19F
:10A6B0001021204607F06CFA082305A88DF8143005
:10A6C000069412F01FFA0028CDD1092305A88DF8B1
:10A6D0001430069412F016FA0028BCD0C3E72846BE
:10A6E00007F068FBC1E76FF01000BEE710B501216D
:10A6F0000846FFF759FF4FF0FF33BDE810401A46F8
:10A7000019460120FFF7A6BD30B58BB00C460546B3
:10A7100007F0E6F9FFF7A5FCB8B12C2301A88DF8E6
:10A7200004308DF8085012F0EDF938B9094B9D60EE
:10A7300074B1284607F074FB0BB030BD03280CBF82
:10A740006FF002006FF00600F6E76FF01000F3E71D
:10A750002046F1E7C0000020F0B5874E8BB00446DC
:10A76000052556F8043B1BB1DB690BB12046984721
:10A77000013D15F0FF05F4D12378013B0C2B4BD89C
:10A78000DFE813F00D004A004A00C7004A004A0003
:10A790004A004A004A008D004A00EA00AF0065788E
:10A7A000764E774F002D39D1764808F0AFFB28461A
:10A7B00008F0B8FD356007F01BFB02280AD18DF8C0
:10A7C000080001A88DF8045012F09CF910B16E48F1
:10A7D00008F09CFB3B680BB10020984707F01AFB80
:10A7E0000021FFF791FF07F003FB1EF027FE98B151
:10A7F000332301A88DF8043012F0A8F801A812F054
:10A80000A5F8002847D1614808F080FB029B60480A
:10A81000D3F8D01008F07AFB0BB0F0BD022D1CD09D
:10A82000EB1E012B1BD85B4808F070FB002008F0E2
:10A8300079FD35680135356007F0E8FB854213D9AD
:10A84000002333603B6823B153486378436008F0CA
:10A850004DFD524BDB6A9847C5E75148E4E729466E
:10A86000504808F053FBE1E700224F49104608F03A
:10A8700055FD054648B907F0B7FB4FF47A714143DF
:10A880002A46284608F04CFDDCE740F2D91145483D
:10A8900008F03CFBD6E7454808F038FBBCE7444DE0
:10A8A00064782B78ACB9012B03D1424808F02EFB19
:10A8B0002C7007F09DFA0128AED13F4B1A78042A7C
:10A8C000AAD018700C2301A88DF8043012F0ECFC0B
:10A8D000A2E7012BA0D1394808F018FB00232B7008
:10A8E0009AE76378002B97D10421334A8DF804301E
:10A8F0000DEB0100012311708DF8083012F002F900
:10A90000002889D12E4808F001FB0220FFF778F8D3
:10A9100082E72C4B01221A702B4B227A1A702B4B98
:10A92000627A1A7063782A4C2370002B3FF474AF5C
:10A93000284808F0EBFA284B1A68002A3FF46CAF5D
:10A9400026482378037000234370837083808371CB
:10A950000BB0BDE8F04010476378002B3FF45CAFCC
:10A960001F4808F0D3FA144B1A78042A1CBF03229C
:10A970001A700A23A7E700BF68210020AC2100203D
:10A98000F823002093DB0208A1DB0208F2DB0208B7
:10A9900008DC0208B6DB0208AC000020280003082F
:10A9A000D4DB02087DDB0208B5A4000859DB0208ED
:10A9B0000924002017DC0208CC21002029DC020831
:10A9C0003FDC0208DE23002066210020A8210020B1
:10A9D000DF2300204ADC0208FC230020D6230020CD
:10A9E00029D9020830B58BB00C46054607F078F837
:10A9F000FFF737FB68B1292301A88DF804300295D1
:10AA000012F080F840B954B1284607F02DFA0BB087
:10AA100030BD6FF01000FAE76FF00600F7E7204650
:10AA2000F5E730B58BB00C46054607F059F8FFF74F
:10AA300018FB68B12A2301A88DF80430029512F0A2
:10AA400061F840B954B1284607F020FA0BB030BD88
:10AA50006FF01000FAE76FF00600F7E72046F5E721
:10AA600030B58BB00C46054607F03AF8FFF7F9FA17
:10AA700070B11D2301A88DF804308DF8085012F034
:10AA800041F840B954B1284607F024FA0BB030BD64
:10AA90006FF01000FAE76FF00600F7E72046F5E7E1
:10AAA00070B58AB00C46054607F01AF8FFF7D9FAD8
:10AAB00000B3272301A88DF80430029512F022F884
:10AAC00018B16FF006000AB070BD282305F57A763C
:10AAD00001A88DF80430029612F014F80028F0D185
:10AAE0005CB1304607F01AFA0028ECD1284607F08E
:10AAF00003FAE8E76FF01000E5E72046E3E770B5FA
:10AB00008AB00C46054606F0EBFFFFF7AAFA00B341
:10AB1000282301A88DF80430029511F0F3FF18B135
:10AB20006FF006000AB070BD2723A5F57A7601A85C
:10AB30008DF80430029611F0E5FF0028F0D15CB1E9
:10AB4000304607F0D9F90028ECD1284607F0E6F99D
:10AB5000E8E76FF01000E5E72046E3E770B58AB05C
:10AB60000C46054606F0BCFFFFF77BFAC8B12D2363
:10AB70006EB201A88DF804308DF8086011F0C2FFA4
:10AB800040B90A4B83F8246074B1284607F0D8F91D
:10AB90000AB070BD03280CBF6FF002006FF0060012
:10ABA000F6E76FF01000F3E72046F1E7C000002061
:10ABB00030B58BB00C46054606F092FFFFF751FA10
:10ABC00088B11F2301A88DF8043011F0BFFE68B9C9
:10ABD00001A8029511F096FF58B96CB1284607F00C
:10ABE00061F90BB030BD6FF01000FAE76FF00600AE
:10ABF000F7E76FF00200F4E72046F2E770B58AB09D
:10AC00000C46054606F06CFFFFF72BFA30B31F2603
:10AC100001A88DF8046011F099FEB8B9212301A8AC
:10AC20008DF804308DF80C5011F06CFF01A88DF8F0
:10AC300004608DF80C5011F065FF28B94CB128461E
:10AC400007F000F90AB070BD032804D06FF00600C9
:10AC5000F8E72046F6E76FF00200F3E76FF0100028
:10AC6000F0E70000F0B58FB005461DF063FA07F07D
:10AC700089F8C0B2012829D001F020FD002407F096
:10AC8000B7F8022805D007F08FF810B1864BDB6AC1
:10AC9000984707F077F8C0B2012814D19CB907F0A3
:10ACA00091F980B107F07CF9054607F08BF906466B
:10ACB00007F09AF9074607F0A9F93A4603463146E4
:10ACC0002846FFF7C7FA20460FB0F0BDC5B914F00B
:10ACD0000DFC7648764B0360764B4360764B7749A4
:10ACE0008360774BC3600023C1E900338B602A4641
:10ACF000744BCB6011F002FC88B16FF00604BEE724
:10AD0000142D04D1022014F0F1FB0025E1E7152DEC
:10AD100001D10320F7E7162DDBD10420F3E76A4BBE
:10AD200001221A7034238DF8143005A8674B06935E
:10AD300011F0E8FE0028E0D16B1E012B03D905F0CD
:10AD4000FD03082B28D1002302A8ADF8063006F039
:10AD5000D9FE0446002892D1BDF8063002AA014669
:10AD6000012412F8016B26B104FA00F10B439BB2E7
:10AD7000012101300C28F4D109B1ADF80630FFF7FC
:10AD8000BFF8014600287DD0FFF7BAF8FFF708F8B2
:10AD9000044600287FF473AF052D78D007F004F83F
:10ADA0000021FFF701FC044600287FF468AF01F0A2
:10ADB000F3F9044600287FF462AF07F019F8214642
:10ADC000FFF7A6FB044600287FF459AF06F0FEFF0C
:10ADD0002146FFF776FB044600287FF450AF07F0CA
:10ADE00019F82146FFF790FC044600287FF447AF8E
:10ADF00007F022F82146FFF701FF044600287FF400
:10AE00003EAF07F05BF82146FFF7D2FE07F026F8C9
:10AE10002146FFF7E7FD044600287FF430AF07F036
:10AE200053F82146FFF71CFE044600287FF427AFA5
:10AE300007F05CF82146FFF733FE044600287FF454
:10AE40001EAF07F077F82146FFF788FE044600287A
:10AE50007FF415AF07F054FA12F08CFB1C4815F084
:10AE600059FE1C4816F046FFFFF7E2F811F0FAFC15
:10AE700000287FF442AF1849FFF78AF800283FF412
:10AE8000FEAE3AE70DF10600FEF748FA80E7FFF75D
:10AE900037F8002882D00020FEF782FF0446002801
:10AEA0003FF47CAFEBE600BF2800030898210020A8
:10AEB0000D920008899A000859A7000888210020EF
:10AEC000C99000085D8F0008D22200200003000115
:10AED0009C000020A40000207C21002038B506F052
:10AEE00051FFC0B2012809D007F03EFCD8B11E497D
:10AEF0001E4808F00BF86FF0060412E006F0F0FDB3
:10AF0000A0F11403DBB2022B054698BF0025FEF723
:10AF100038F804460028E7D0284615F003FE00283C
:10AF2000E2D0204638BD01F069F90028E3D106F0EF
:10AF300029FFC0B2012801D00024F2E706F0D0FDBD
:10AF4000A0F11403DBB2022B054698BF002506F0E2
:10AF5000C7FDFFF787FE04460028EDD0284615F010
:10AF6000E1FD0028E8D0DCE788DE020865DC0208A5
:10AF7000F0B58BB0064606F0B3FD864200F098802F
:10AF80003046FFF76EF8002800F09480FDF7F9FFD7
:10AF9000044618B1494B1B78002B60D101F02EF903
:10AFA00000285CD107F098F80746002857D1002EFA
:10AFB00058D1012014F09AFA3546414941482A46B1
:10AFC00011F09CFA002870D12B2301A88DF80430D1
:10AFD00011F0BCFC002868D19DF8080006F020FFA5
:10AFE000044600283BD1202701A88DF8047011F0F9
:10AFF000ADFC002859D19DF80C0006F023FF044653
:10B0000068BB01A88DF8047011F0A0FC00284CD199
:10B01000029806F047FF044608BB2E2301A88DF8CE
:10B02000043011F093FC00283FD19DF8080006F091
:10B0300087FF044698B96B1EDBB2012B24D905F0BB
:10B04000FD03082B20D0002E18BF3546284606F0F9
:10B050004DFD044618B92846FFF704FE0446204675
:10B060000BB0F0BD142E04D1022014F03FFA3D467F
:10B07000A3E7152E01D10320F7E7162E01D10420F6
:10B08000F3E73546064698E7242301A88DF80430F7
:10B0900011F05CFC48B9029806F03EFD0446002819
:10B0A000DDD107F019F80028CDD06FF00604D6E7FF
:10B0B0000024D4E76FF01004D1E700BFD2220020B3
:10B0C000882100209821002013B5064C636898471A
:10B0D00028B9E36A019302B0BDE81040184702B0F6
:10B0E00010BD00BF28000308014B5B68184700BF74
:10B0F0002800030808B5034B5B689847003818BF61
:10B10000012008BD2800030808B507F035FE024AF3
:10B1100013680133136008BD68270020F7B5164C8B
:10B12000164E2368164D30682F68013B2360154B7F
:10B1300021681A6864234343511A3844B3FBF0F37F
:10B14000114807F0E3FE236810493BB14B6B0193B4
:10B1500041F2883003B0BDE8F04018470C48336036
:10B1600002782B600B6B019322F00802027003B08F
:10B17000BDE8F040184700BF6026002030240020C2
:10B180003424002064260020C0DE020828000308C2
:10B1900038240020024A136801331360FFF7BEBF52
:10B1A00030240020FFF7F6BF10B5064C20680130B0
:10B1B0002060114604481A4607F0A8FEBDE810407A
:10B1C000FFF7ACBF34240020DEDE0208F8B52D4DB9
:10B1D0002D4F2B78BA6A2D4C2D4E002B33D0236D7A
:10B1E0002C48013B2365E17D9047616C2A4807F0BC
:10B1F0008DFE3268216D2948511A07F087FEE26CF6
:10B20000636C13446364626CA36C9A4282BF244BE8
:10B210001B686364606CFB689847236D23B1BDE8CD
:10B22000F84020480EF088BE1F4A1E48137823F0CD
:10B23000040313700EF0E8FD10B11A480EF02CFE56
:10B2400000232B70F8BD194D12482B68013B2B6071
:10B25000E17D9047326829681048511A07F056FE80
:10B260002B68002BDBD1104A0E48137823F004031F
:10B2700013700EF0C9FD0028E4D0BDE8F84009487D
:10B280000EF00ABE5C26002028000308C000002043
:10B29000642600206826002001DF020813DF020870
:10B2A000582600203C24002038240020602600205E
:10B2B000F8B52E4D2E4F2B78BA6A2E4C2E4E002B01
:10B2C00035D0236D2D48013B2365E17D9047616CAE
:10B2D0002B4807F01BFE3268216D2A48511A07F0EF
:10B2E00015FE226D33689B1A274A1278B3FBF2F1E0
:10B2F00002FB1133254A52F823306364606CFB680B
:10B300009847236D23B1BDE8F84021480EF014BEE4
:10B31000204A1F48137823F0040313700EF074FDC5
:10B3200010B11B480EF0B8FD00232B70F8BD1A4D6C
:10B3300012482B68013B2B60E17D904732682968F9
:10B340001048511A07F0E2FD2B68002BDBD1114A9F
:10B350000F48137823F0040313700EF055FD0028F6
:10B36000E4D0BDE8F8400A480EF096BD5C26002007
:10B3700028000308C0000020642600206826002062
:10B3800001DF020813DF02085424002058240020A3
:10B390003C240020382400206026002010B5094BF2
:10B3A0001B6813B1084B1B6D3BB9084C236823B1D4
:10B3B00007F0EAFC2368013B2360BDE81040044825
:10B3C00007F0A4BD60260020C000002068270020F0
:10B3D0002FDF020870B50D4CC0000022022182420E
:10B3E00000D170BDC1F3001383EA1123D51043EAE5
:10B3F000410302F00706C3F3080103F00103B34061
:10B40000665D334363550132E9E700BF68260020DB
:10B41000064B10B5064C1B6B9847236823B107F009
:10B42000B3FC2368013B236010BD00BF2800030864
:10B430006827002038B50D4D287810F0010411D18F
:10B44000FFF762FE2B7843F001032B70084B186B5B
:10B4500093F82410074B4FF6FF72DB6B49B2984705
:10B46000204638BD6FF00500FBE700BF3824002000
:10B47000C0000020280003080F4B104810B5002220
:10B480001A700EF0C1FC10B10C480EF005FD0C480E
:10B490000EF0BAFC10B10A480EF0FEFC094B0A4C43
:10B4A000DB6A9847236803B910BD07F06DFC236879
:10B4B000013B2360F6E700BF382400203C24002035
:10B4C0006028002028000308682700202DE9F04F9D
:10B4D000284A137899078DB0064648D4264C274D44
:10B4E000206B43F002031370EB689847206894F8D0
:10B4F0002410A26A6368A7680A9394F80CB00B97AB
:10B50000A78A94F816C094F818E094F8198094F873
:10B510001A9094F81BA0E36ABFB2CDE907A30B9B76
:10B520000093CDE901B70A9BEF69CDE90589CDE923
:10B5300003CE49B2C0B2B847636BB3B96B6B6FF05F
:10B540007F409847322007F059FA2B6C002098472B
:10B55000EB6A30809847074AB6F90000137823F069
:10B56000020313700DB0BDE8F08F6B6EE7E76FF06C
:10B570000500F7E738240020C00000202800030859
:10B5800010B50446FFF7C0FD226B144B1344144A58
:10B59000934220D894F824300933DBB21F2B1AD8F9
:10B5A0006368062B17D8A368053B072B13D8237BAA
:10B5B000013B032B0FD82368022B0CD8A36A094A3E
:10B5C000A3F59653934206D807485422214607F024
:10B5D000E0FE002010BD6FF00200FBE7802E0FF7A9
:10B5E000809E4730780D0700C000002008B5034951
:10B5F000542207F0CEFE002008BD00BFC00000208E
:10B600002DE9F04F324C25788DB015F004050B90E4
:10B610005BD1FFF779FD23782E482F4E43F00403CA
:10B62000237007F073FC2D482D4B03602D4B836076
:10B630002D4B43602D4B2E4CC3602E4B0361336862
:10B640009847E07DFFF7C6FE206BF36898472068B7
:10B6500094F82410A26A6368A7680A9794F80CC04B
:10B66000A78A94F816E094F8188094F8199094F842
:10B670001AA094F81BB0E46ABFB2CDE907B40A9CE3
:10B680000094CDE903E8CDE901C749B2C0B2CDE9E4
:10B69000059AF469A047184B0B9A1A601A68174B61
:10B6A00017481A604FF0FF31164B00952A460EF0EE
:10B6B00091FB4FF4FA7112480EF078FC10480EF02E
:10B6C0003BFC28460DB0BDE8F08F6FF00500F9E7B0
:10B6D000382400203ADF0208280003080C24002048
:10B6E0009DB30008A9B1000811B4000895B1000885
:10B6F000C0000020A5B100086026002064260020BC
:10B700003C240020CDB100082DE9F04F2C4D04461B
:10B71000287810F008088DB04FD1002C4DDDFFF7D0
:10B72000F3FC2B78274843F008032B70264B03606B
:10B73000264B8360264B274D4360274BC360274B26
:10B7400003612B689847264B1C601A68254C264BD2
:10B75000206B1A60EB68984720686168A268237BB9
:10B7600026690A96A68A276A94F816C094F817E004
:10B7700094F81890CDF82C9094F8199094F81AA099
:10B7800094F81BB0247FCDF80CC0CDE908B40B9C15
:10B79000B6B2CDE904E4BFB20A9C0094C0B2CDE9D0
:10B7A000069ACDE90167AC69A04741F288306B6B1E
:10B7B000984740460DB0BDE8F08F6FF00500F9E7FF
:10B7C000382400200C2400209DB30008A9B10008F3
:10B7D00011B400082800030895B10008A5B10008BD
:10B7E00060260020C0000020642600202DE9F04FD4
:10B7F000364C257815F004058DB0074663D1FFF768
:10B8000083FC23783248334E43F004032370324BD9
:10B81000324C01221A70324B0360324B8360324B40
:10B820004360324BC360324B0361336898477B6C93
:10B830006364BB6CA364FB6CE3643B6D2365E07DD8
:10B84000FFF7C8FD2B4B626C1A602B4B226D1A6000
:10B85000606CF3689847206894F82410A26A6368C3
:10B86000A7680B9794F80CC0A78A94F816E094F890
:10B87000188094F8199094F81AA094F81BB0E46A10
:10B88000BFB2CDE907B40B9C0094CDE903E8CDE944
:10B8900001C749B2C0B2CDE9059AF469A047174B78
:10B8A000174800952A464FF0FF310EF093FA4FF4F7
:10B8B000FA7113480EF07AFB11480EF03DFB284652
:10B8C0000DB0BDE8F08F6FF00500F9E738240020D7
:10B8D0000C240020280003085C260020C000002063
:10B8E0009DB30008A9B1000811B4000895B1000883
:10B8F000A5B100085826002064260020CDB100081C
:10B900003C2400202DE9F04F964D297811F00404D5
:10B910008BB0064640F02381DFF84C82FFF7F4FB42
:10B92000214692484FF400721EF0D0FB88F8004088
:10B93000214623468D4C8029CAB203D163B188F8D1
:10B94000001009E0F06C736C00FB0133B06C8342B3
:10B9500021D9013A88F80020022007F04DFA1FF0A3
:10B96000BDF800276FF0004998F80030BB4217DCA3
:10B97000FDF7A4FC7E4B0A2800F2EE80DFE810F011
:10B980004A00B600BC00C200C800CE00D400DA00F5
:10B99000E000EC00E60044F8213001310123CAE761
:10B9A0001FF0CAF898F8002054F82710D31B99FB11
:10B9B000F3F3013390FBF3F33B449F4208BF0023B2
:10B9C00054F82300414044F8271054F8271054F845
:10B9D0002300414044F8231054F8271054F8230062
:10B9E000414044F8271054F8231054F822004140F5
:10B9F00044F8231054F8231054F82200414044F82E
:10BA0000221054F8231054F822204A4044F82320EE
:10BA10000137A9E79A68574998688F56564916F032
:10BA200095FC04462B785548DFF8548143F0040315
:10BA30002B70544B4E4D01221A70534B0360534BE5
:10BA40008360534B4360534BC360534B0361D8F83F
:10BA500000309847454B1B686B64B36CAB64F36C68
:10BA6000EB64336D2B65E87DFFF7B4FC4B4B6A6CE0
:10BA70001A604B4B2A6D1A60686CD8F80C309847E6
:10BA8000286895F82410AA6A2E7BAB8A95F816C010
:10BA900095F818E095F8199095F81AA095F81BB04C
:10BAA000ED6A00979BB2CDE903CECDE907B5CDE9AC
:10BAB000016349B22346C0B20024CDE9059AD8F803
:10BAC0001C50A847374B3848009422464FF0FF31AE
:10BAD0000EF080F94FF4FA7133480EF067FA3248ED
:10BAE0000EF02AFA20460BB0BDE8F08F9A682F4975
:10BAF00098688F562E4992E79A682E4998688F5613
:10BB00002D498CE79A682D4998688F562C4986E70D
:10BB10009A682C4998688F562B4980E79A682B4978
:10BB200098688F562A497AE79A682A4998688F5602
:10BB3000294974E79A68294998688F5628496EE719
:10BB40009A68284998688F56274968E79A6827496C
:10BB500098688F56264962E70024072762E76FF04E
:10BB60000500C0E738240020542400205824002079
:10BB7000C0000020D4E0020844DF02080C240020AA
:10BB8000280003085C2600209DB30008A9B1000826
:10BB900011B4000895B10008A5B10008582600208E
:10BBA00064260020B1B200083C240020DCE002083A
:10BBB00064DF0208ECE00208A4DF0208D4E0020817
:10BBC000BCDF0208D4E00208DCDF0208D4E002088F
:10BBD000FCDF0208ECE002083CE00208D4E00208C6
:10BBE0001CE00208F2E0020894E00208DCE002082F
:10BBF00054E0020808B503490C2207F0CAFB0020F4
:10BC000008BD00BFB400002038B505460B4CFFF757
:10BC10007BFAAB68A3602B68094823606B68094D09
:10BC20006360094B43602B6898472068EB6B22895F
:10BC300094F904109847002038BD00BFB4000020DC
:10BC40000C2400202800030811B4000808B5E0B156
:10BC50004FF0FF331A4619460120FEF7FBFA002089
:10BC600011F088FC01220B49042007F057FB024623
:10BC700030B941F27071042007F052FB002008BD7A
:10BC80003621054807F042F9F8E7042007F04AFB9F
:10BC9000F4E700BFDDBC000863D902081FB50D4AF8
:10BCA000034601210C4811708DF80830432200230F
:10BCB0008DF809308DF80B300270009304AB13E956
:10BCC0000C00FDF763FD003818BF0120404205B0AD
:10BCD0005DF804FB5E2800206C27002010B5FDF7FE
:10BCE000CAFB40B94FF0FF33BDE810401A46194671
:10BCF0000120FEF7AFBA094CE368984720B9BDE8C8
:10BD000010400220FFF7CABFE368984720B1BDE8A2
:10BD10001040002001F0DEB910BD00BF1C01002062
:10BD2000F0B54FF4807285B000213948394D3A4C56
:10BD30001EF0CCF900232B700FF084FB80B2C828D2
:10BD400084BF143880B2E36806389842606143D3F8
:10BD50000021A17023712B782D4E2278F2545A1CA9
:10BD6000D2B26078B0549A1CD2B2A078B054DA1C27
:10BD7000D2B2E078B054581D0433DBB22279F254C9
:10BD8000A368C0B21944287030441EF077F92B78AC
:10BD900021791944C9B200233046DAB291422FD832
:10BDA0001E4B1B481B788DF8083001238DF80B3093
:10BDB000A369003B18BF01238DF80C3000238DF8D8
:10BDC00009300093013104ABC9B213E90C002970AA
:10BDD000FDF7DCFC05B0F0BD21695B1AB3FBF0F6A2
:10BDE000F2B200FB16364EB9A270A278984202F168
:10BDF000FF3228BF1846A2702071ACE70132F3E78A
:10BE000016F8012B475C3A4442540133C5E700BFA2
:10BE10007828002078290020802D00207929002012
:10BE20000D4A1378BBB10D4B80B9997809B91170DF
:10BE300070471A78197960F341021A70DA78013282
:10BE4000DA701A690A441A61FFF76ABF1A7842F079
:10BE500002021A70F8E770479C2D0020802D002008
:10BE60002DE9F8431C46431EDBB2DE2B0E46054689
:10BE700011462AD8B4F5806F27D8164F164BDFF835
:10BE80005C904FF001082246384683F800801EF08F
:10BE9000F5F8C9F80040124C237823F0030343EA75
:10BEA00008032370FF2007F02FFA00232361D9F83D
:10BEB0000030E3600B4B607084F80380A760A661DC
:10BEC0001D70BDE8F843FFF72BBF6FF00200BDE81F
:10BED000F88300BF7A2900209C2D00207C2D0020B3
:10BEE000802D00207929002084B0F0B58BB010ACF3
:10BEF00084E80F00684D00238DF8073005EB8302BE
:10BF00005268914200F0C5800D33342BF6D1624B5C
:10BF100000245A68E6B2002A40F0B08010AB012736
:10BF200013F8080B8DF87040CDE9031316ABCDE97B
:10BF3000053202284FF6FF7307938DF808201A9BED
:10BF40008DF809008DF80A708DF80B6059D163B334
:10BF500008939DF86C308DF8243002A811F05AF83F
:10BF6000002840F096809DF80B000DF1070208A90B
:10BF700011F0F6F89DF8073023F003031843C0B220
:10BF8000002840F08680342210A902FB04501EF0E5
:10BF900075F8414806F086F8002818BF6FF00600D3
:10BFA0000BB0BDE8F04004B07047FDF787F90A28F0
:10BFB0006FD8DFE800F0060A161A1C1E20220A2499
:10BFC0000A00364B0893022302E0354B08930823FE
:10BFD0008DF82430089B1A939DF824308DF86C302E
:10BFE000BBE7304B08930023F2E72F4BFAE72F4BC8
:10BFF000F8E72F4BF6E72F4BF4E72F4BE2E72F4BF9
:10C00000F0E74BB108939DF86C308DF82430BDF803
:10C010006E30ADF82630A0E7FDF750F90A2838D881
:10C02000DFE800F0060A161A1C1E20220A26280045
:10C03000234B0893032302E0194B089308238DF840
:10C040002430089B1A939DF824308DF86C30DEE77D
:10C050001C4B08930223F2E71B4BEAE7134BE8E77C
:10C06000134BE6E7194BE4E7134B08930423E6E789
:10C07000174BDEE70A4B08930A23E0E70134042C50
:10C0800003F134037FF445AF1248342200211EF03F
:10C090001DF86FF00F0083E7A02D002000EA06379F
:10C0A000A070083720441E1E8068D92E2876E81913
:10C0B00008E6D333E013F336F080A633E069CD33DE
:10C0C00040F7093720937F1D4026CA2E606305374D
:10C0D00010D62D05702E0020104A38B500231446C6
:10C0E0005168814213D1342505FB034494F8300094
:10C0F00011F00CF8014638B92A4620461DF0E6FF3B
:10C10000064805F0CFFF08B16FF0060038BD0133D7
:10C11000042B02F13402E3D1F6E700BFA02D00208A
:10C12000F0B58FB01B4E05463422002101A81DF04A
:10C13000CDFF012386F83130022386F865300323D2
:10C1400086F89930042334220DEB0301284686F843
:10C15000CD301DF083FF40B90E49342228461DF032
:10C160008DFF6FF00D000FB0F0BD37460024342274
:10C17000394628461DF072FF30B9032CF3D0342223
:10C1800004FB02213144E9E70134042C07F13407B0
:10C19000EDD1E1E7A02D00202DE9F043BFB005F07F
:10C1A0007DFFD02201460AA81DF068FF0AAE4FF0BD
:10C1B00000084FF03409736853B908F10108B8F169
:10C1C000040F06F13406F6D100203FB0BDE8F0833D
:10C1D0003EAB09FB0834A4F1D007C03C0FCC6D4640
:10C1E0000FC50FCC0FC523682B6097E80F00FFF732
:10C1F0007BFE0028E1D06FF00600E6E738B5094D78
:10C20000002405EB8403586820B90D34342CF8D190
:10C21000002038BDFFF760FF0028F6D06FF0060061
:10C22000F7E700BFA02D0020014B1870704700BF3A
:10C23000D02E0020024B034A1B78D054704700BF19
:10C24000D02E0020702E00202DE9F0438BB0232348
:10C25000054601A88DF8043010F078FB024600284E
:10C2600052D12B4B2B4ED3F800E093F906800746B2
:10C27000BCB2002006EB020C00EB0209CE4581B2F5
:10C2800030D11CF90090C1452CD10F291CD1052CAF
:10C2900006D14FF0FF321A6000200BB0BDE8F083EA
:10C2A0000134A4B22101029A196032F8142002F07C
:10C2B00001029A80725C9A711549082228461DF085
:10C2C000DDFE6FF00D00E8E7013188B212FA81F26D
:10C2D0000121814002981A6030F81700B25C0140D9
:10C2E0009980E8E701301028C6D10137062F02F106
:10C2F0001002BDD100221A60029A128802F00102D7
:10C300009A80044A1278D6E76FF00600C5E700BFAE
:10C3100014010020702E002010B5064B1B68044647
:10C3200003B19847044B0CB100225A7000225A7195
:10C3300010BD00BF10300020F72F002038B5104C82
:10C3400000236370A37005F01DFDC0B2A0B90D48B5
:10C3500006F0DCFD0C4B1D681DB10C4B93E807008B
:10C36000A847E37853B9237943B9094B1B6B984726
:10C37000BDE8384006F008BD0648E9E738BD00BF13
:10C38000F72F002002E102080C30002000300020CE
:10C39000280003081DE1020813B5144C0023637044
:10C3A0001DF04CF818B11249124806F0AFFD124BBF
:10C3B0001B6803B1984705F0E5FCC0B290B90F487F
:10C3C00006F0A4FD06F0E0FC23796BB10123637055
:10C3D0000B4C236B9847636B0193002002B0BDE8C0
:10C3E000104018470748EBE702B010BDF72F0020B8
:10C3F000EDE1020809E202081430002038E10208E9
:10C40000280003084AE1020808B5064B00225A70CA
:10C410001DF014F828B1BDE808400349034806F0B0
:10C4200075BD08BDF72F0020F6E1020809E20208F9
:10C4300010B5114B00225A709A781AB9DA780AB9F5
:10C440001A7912B101225A7010BD05F09BFCC0B2DE
:10C4500080B90A4806F05AFD094B1C681CB1094B0B
:10C4600093E80700A047084B1B6B9847BDE81040B6
:10C4700006F08ABC0548EDE7F72F00205CE10208D2
:10C480000C300020003000202800030879E1020869
:10C4900008B505F077FCC0B208BD0000044B587821
:10C4A00020B9987810B9D87800B91879704700BFCA
:10C4B000F72F002005F01CBE044B054A03449342AD
:10C4C0008CBF6FF002000020704700BF802E0FF776
:10C4D000809E473005F01EBE053807288CBF6FF0E0
:10C4E00002000020704708B505F026FE7D2806D022
:10C4F000FA2806D0B0F5FA7F08BF022008BD002058
:10C50000FCE70120FAE700002DE9F04F99B005F0B3
:10C5100015FF0A9005F0FAFE0B9005F009FF0E904A
:10C5200005F0DCFE0F9005F0D3FE0C9005F018FF2F
:10C5300006F044FA002800F09E8012A806F04AFA9D
:10C54000129F9DF85CB09DF84CA0BDF85A5005F0C4
:10C5500019FCC0B2002840F08680149C9DF85890C9
:10C5600009F1010805F00EFC10F0FF02524E3DD11A
:10C57000109205F0DDFE6FF07F4308930B9B07934D
:10C580000A9B109A0D90CDE90253F3691093012094
:10C590005FFA88F9CDE90522DDF840C00490234612
:10C5A0004FFA8BF1CDE900A91192E0470D9B119A4A
:10C5B0000092B3FA83F35B0909930B9B08930A9BE0
:10C5C0000393BDF83830CDE90153B3690A930120D4
:10C5D000CDE90420CDE906224B462146DDF828C0EE
:10C5E0005246E047736DFF210120984705F0CAFBD2
:10C5F000C0B202282FD100206FF07F43CDE907039E
:10C600000C9B0093F3690A934FF0010A5FFA88F9D3
:10C61000CDE90500CDE9030ACDE901950F9ADDF8D2
:10C6200028C023464FFA8BF1E04700200523CDE9CF
:10C630000153CDE90700CDE905A0CDE90300009045
:10C640004B462146B5690C9ACDF824A0A847736DD6
:10C65000FF2150469847184B3846DB689847002022
:10C6600019B0BDE8F08F05F08DFBC0B2022804BF01
:10C67000159C640872E705F03BFD074605F09CFD3C
:10C68000834605F047FD824605F084FD054605F02A
:10C6900079FBC0B238B9FFF726FF044605F068FD04
:10C6A00000F101085EE705F06DFBC0B20228F5D18C
:10C6B000FFF719FF4408F1E7280003080A4808B506
:10C6C0000A4B03600A4B83600A4B43600A4BC3600A
:10C6D0000A4B03610A4B83610A4B1B689847FFF7BB
:10C6E00013FF002008BD00BFD42E002099C300080E
:10C6F0001DCF000809C4000831C400083DC300086C
:10C7000019C3000828000308B0F5803F70B504463F
:10C7100041D2431E0D2B214898BF0F240C2200212B
:10C720001DF0D4FC1E4B5CB19A781AB9DA780AB9BC
:10C730001A792AB11B4806F0E9FB6FF0050070BDBD
:10C740000122194D5A704CB99C705C70DC701C71E0
:10C7500006F01AFB2B6B98470020F0E74FF6FF71AD
:10C760008C426E6B09D19A70FFF7CEFE2B6B984707
:10C770000020B04706F000FBEEE74FF6FE718C425A
:10C7800001D1DA70F0E74FF6FD718C4201D11A71D8
:10C79000EAE72046EDE76FF00200D0E70030002026
:10C7A000F72F002096E102082800030808B5074B80
:10C7B000074A0344934205D805F0A0FCFFF7A4FE06
:10C7C000002008BD6FF00200FBE700BF802E0FF7CE
:10C7D000809E473008B5431F072B05D805F0A0FC05
:10C7E000FFF792FE002008BD6FF00200FBE700009B
:10C7F00010B5044605F0C6FA10F0FF000CD17D2CF0
:10C8000014D0FA2C1CD0B4F5FA7F1BD0092C0ED909
:10C810006FF00204204610BD05F0B4FAC0B2022841
:10C8200005D1094BA4F596529A42F0E704462046FA
:10C8300005F08CFC04460028ECD1FFF765FEE9E723
:10C840000124F4E70224F2E7780D070010B504464E
:10C8500005F098FAC0B268B97D2C01D1002010BD56
:10C86000FA2CFBD0B4F5FA7FF8D0092CF6D96FF08A
:10C870000200F4E705F086FAC0B20228EED1024BBE
:10C88000A4F596549C42F1E7780D070005F070BCC2
:10C89000032808B505D805F071FCFFF735FE002028
:10C8A00008BD6FF00200FBE703288CBF6FF00200A9
:10C8B0000020704705F06EBC042808B505D905F0C6
:10C8C0006FFCFFF721FE002008BD6FF00200FBE7C0
:10C8D000042894BF6FF002000020704705F06CBC84
:10C8E00008B5431F112B05D805F06CFCFFF70CFEB3
:10C8F000002008BD6FF00200FBE7053811288CBF4F
:10C900006FF002000020704705F068BC05F06CBCB9
:10C9100005F076BC05F082BC05F09ABC05F0A6BC1B
:10C9200008B505F02FFD003818BF012008BD05F03F
:10C930002FBD2DE9F041FF29ADF5087D0C461746C6
:10C9400033D848AE0A46014630461DF097FB14F036
:10C950000F030ABF1022C3F110031346204618BF6D
:10C96000DAB21C4484421DDC102107A8FFF7D4FF73
:10C970000DF12C08102103A8FFF7CAFF4246102131
:10C9800003A8FBF791FEE5B2CDF8008007ABC4F336
:10C99000031239463046FBF794FE28460DF5087D14
:10C9A000BDE8F08132540130DCE76FF00200F5E7BA
:10C9B000F8B5254D6B7806460C46174623B12B7902
:10C9C00013B96FF00500F8BDFFF79EFD05F006FCFA
:10C9D00010B321461D4A3046FFF7ABFFC4B21C4ED0
:10C9E00006F0CAF9336B984701236B70D7B9B36A65
:10C9F0001648214698471CF021FD0028E3D0214627
:10CA00001448124D144E06F081FAA4B2A4B913488A
:10CA100006F07CFA2046D6E7224631460B481DF048
:10CA20002DFBDCE76B71B36B98476B79002BFCD166
:10CA30006B78002BDBD1C4E715F8011B3046013CB5
:10CA400006F064FAA4B2E1E7F72F0020F82E0020E8
:10CA500028000308AAE10208C4E10208FEDE020879
:10CA6000F0B5C9B00D460646102107A814460BAF15
:10CA7000FFF752FF102103A8FFF74AFF3A461021A3
:10CA800003A8FBF711FE07AB2A09009721463046A1
:10CA9000FBF727FE6219284612F8013C012B03D14F
:10CAA000681EC0B249B0F0BD022B05D112F8023C9D
:10CAB000022BF6D1A81EF4E7032B09D112F8023C91
:10CAC000032BEED112F8033C032BEAD1E81EE8E772
:10CAD000042B0DD112F8023C042BE2D112F8033CD6
:10CAE000042BDED112F8043C042BDAD1281FD8E73E
:10CAF000052B11D112F8023C052BD2D112F8033CC0
:10CB0000052BCED112F8043C052BCAD112F8053CF6
:10CB1000052BC6D1681FC4E7062B15D112F8023CBD
:10CB2000062BBED112F8033C062BBAD112F8043CF6
:10CB3000062BB6D112F8053C062BB2D112F8063CF2
:10CB4000062BAED1A81FACE7072B19D112F8023C77
:10CB5000072BA6D112F8033C072BA2D112F8043CF4
:10CB6000072B9ED112F8053C072B9AD112F8063CF0
:10CB7000072B96D112F8073C072B92D1E81F90E7BC
:10CB8000082B22D112F8023C082B8AD112F8033C60
:10CB9000082B86D112F8043C082B82D112F8053CF0
:10CBA000082B7FF47EAF12F8063C082B7FF479AF98
:10CBB00012F8073C082B7FF474AF12F8083C082BDE
:10CBC0007FF46FAFA5F108006BE7092B2AD112F8AB
:10CBD000023C092B7FF465AF12F8033C092B7FF46C
:10CBE00060AF12F8043C092B7FF45BAF12F8053CF0
:10CBF000092B7FF456AF12F8063C092B7FF451AF96
:10CC000012F8073C092B7FF44CAF12F8083C092BB3
:10CC10007FF447AF12F8093C092B7FF442AFA5F12E
:10CC200009003EE70A2B2FD112F8023C0A2B7FF4B1
:10CC300038AF12F8033C0A2B7FF433AF12F8043CF0
:10CC40000A2B7FF42EAF12F8053C0A2B7FF429AF94
:10CC500012F8063C0A2B7FF424AF12F8073C0A2B8B
:10CC60007FF41FAF12F8083C0A2B7FF41AAF12F8BA
:10CC7000093C0A2B7FF415AF12F80A3C0A2B7FF40B
:10CC800010AFA5F10A000CE70B2B34D112F8023CCF
:10CC90000B2B7FF406AF12F8033C0B2B7FF401AF94
:10CCA00012F8043C0B2B7FF4FCAE12F8053C0B2B66
:10CCB0007FF4F7AE12F8063C0B2B7FF4F2AE12F8BD
:10CCC000073C0B2B7FF4EDAE12F8083C0B2B7FF4E6
:10CCD000E8AE12F8093C0B2B7FF4E3AE12F80A3CE5
:10CCE0000B2B7FF4DEAE12F80B3C0B2B7FF4D9AE8E
:10CCF000A5F10B00D5E60C2B39D112F8023C0C2B18
:10CD00007FF4CFAE12F8033C0C2B7FF4CAAE12F8BE
:10CD1000043C0C2B7FF4C5AE12F8053C0C2B7FF4C1
:10CD2000C0AE12F8063C0C2B7FF4BBAE12F8073CE9
:10CD30000C2B7FF4B6AE12F8083C0C2B7FF4B1AE8E
:10CD400012F8093C0C2B7FF4ACAE12F80A3C0C2B09
:10CD50007FF4A7AE12F80B3C0C2B7FF4A2AE12F8B6
:10CD60000C3C0C2B7FF49DAEA5F10C0099E60D2B2D
:10CD70003ED112F8023C0D2B7FF493AE12F8033C27
:10CD80000D2B7FF48EAE12F8043C0D2B7FF489AE90
:10CD900012F8053C0D2B7FF484AE12F8063C0D2BE7
:10CDA0007FF47FAE12F8073C0D2B7FF47AAE12F8B9
:10CDB000083C0D2B7FF475AE12F8093C0D2B7FF467
:10CDC00070AE12F80A3C0D2B7FF46BAE12F80B3CE0
:10CDD0000D2B7FF466AE12F80C3C0D2B7FF461AE88
:10CDE00012F80D3C0D2B7FF45CAEA5F10D0058E65A
:10CDF0000E2B43D112F8023C0E2B7FF452AE12F8E8
:10CE0000033C0E2B7FF44DAE12F8043C0E2B7FF446
:10CE100048AE12F8053C0E2B7FF443AE12F8063CE8
:10CE20000E2B7FF43EAE12F8073C0E2B7FF439AE8A
:10CE300012F8083C0E2B7FF434AE12F8093C0E2B8E
:10CE40007FF42FAE12F80A3C0E2B7FF42AAE12F8B4
:10CE50000B3C0E2B7FF425AE12F80C3C0E2B7FF40E
:10CE600020AE12F80D3C0E2B7FF41BAE12F80E3CD8
:10CE70000E2B7FF416AEA5F10E0012E60F2B48D153
:10CE800012F8023C0F2B7FF40CAE12F8033C0F2B70
:10CE90007FF407AE12F8043C0F2B7FF402AE12F8B9
:10CEA000053C0F2B7FF4FDAD12F8063C0F2B7FF4F1
:10CEB000F8AD12F8073C0F2B7FF4F3AD12F8083CE5
:10CEC0000F2B7FF4EEAD12F8093C0F2B7FF4E9AD88
:10CED00012F80A3C0F2B7FF4E4AD12F80B3C0F2B39
:10CEE0007FF4DFAD12F80C3C0F2B7FF4DAAD12F8B3
:10CEF0000D3C0F2B7FF4D5AD12F80E3C0F2B7FF4B9
:10CF0000D0AD12F80F3C0F2B7FF4CBADA5F10F0085
:10CF1000C7E5102B08BFA5F11000C2E52DE9F04FC1
:10CF2000334D4FF00009C1B080460C4617461E46EF
:10CF300085F8019085F8029005F050F900283FD05F
:10CF40004FF48072494668461DF0C0F823071EBFA3
:10CF500024F00F041034A4B221466A464046FFF77D
:10CF60007FFDC4B22246694622481DF087F804F0CE
:10CF700009FFC0B23246394628BB1F48DFF874A00B
:10CF8000DFF878B005F0C2FFA046D146B8F1000F37
:10CF90001BD11B4805F0BAFF1A4B1B481B68C78002
:10CFA00006720471C0F800900BB107C89847EB787F
:10CFB0000BB92B799BB101236B7041B0BDE8F08FA9
:10CFC00022464146D0E71148D8E71AF8011B5846D7
:10CFD00008F1FF3805F09AFF1FFA88F8D6E70C4BE6
:10CFE0001B6B984741B0BDE8F04F05F0CDBE00BFC8
:10CFF000F72F0020F82E0020C9E10208C4E1020842
:10D00000FEDE02080C30002000300020DBE10208C8
:10D010002800030805F05CB905F060B9084BA0F5DD
:10D0200016729A4210B5044606D8FFF76DFA2046EC
:10D03000BDE8104005F034B96FF0020010BD00BF2C
:10D04000E80A0300084BA0F516729A4210B5044690
:10D0500006D8FFF759FA2046BDE8104005F02CB974
:10D060006FF0020010BD00BF8891040005F04EB9BA
:10D0700005F052B905F062B905F066B905F070B96E
:10D0800010B505F073F904461BF054F8FFF73CFAAD
:10D09000204610BD10B5064B064C30B129B19A712F
:10D0A0002060996001221A7010BD00222260FAE708
:10D0B0001830002044300020014B1878704700BF22
:10D0C00018300020024B187800B15878704700BF24
:10D0D0001830002008B5054B05480122DA7006F02B
:10D0E00005F9044B00221A7008BD00BF183000205B
:10D0F000580100205A51002030B5894C23788DB05A
:10D1000033B1437B33B9637813B1A3890133A3816E
:10D110000DB030BDC378E02BFAD16578002D3ED13B
:10D12000037B042BF4D183681A78012AF0D15A7852
:10D13000012AEDD19A78012AEAD1DB78012BE7D1D7
:10D140000222E2714FF460426380A280E560052212
:10D1500003A863708DF810308DF80C2025740FF043
:10D16000D1FC284610F006FA6E4B1B685B6803B1D1
:10D17000984700226C4B00924FF0FF316B480CF047
:10D1800029FE41F2883169480CF010FF02A81AF01C
:10D19000CDFF012302A8E3701AF0CAFFB8E7A38904
:10D1A0000133A38183681A78A2700A2AB0D8DFE815
:10D1B00002F0062B2E32364A5677A3A5AF005B4805
:10D1C0000CF022FE10B159480CF066FE0023A3813A
:10D1D000637005238DF80C3004F0F8FD003818BF9B
:10D1E00001208DF8100003A80FF08CFC05F088F8E2
:10D1F000003818BF012010F0BDF94A4B1B689B682E
:10D20000002B85D0984783E70223E37180E7012351
:10D210002371A3707CE7002323710123F9E7A5683C
:10D22000037BE37104222A70A2799A4228BF1A462E
:10D2300000230133D9B28A427FF66AAF8168C95CA4
:10D240000131E954F5E704238DF80C30384B03A87D
:10D250009C6A10F029F8002203A9A04758E7002390
:10D26000A381637005238DF80C3004F0AFFD003806
:10D2700018BF01208DF8100003A80FF043FC05F043
:10D280003FF8003818BF012010F074F9254B1B68D7
:10D290009B6803B19847264B0120DB6A984737E724
:10D2A000027B032A10D105228DF80C20B3F801303F
:10D2B0005BBAADF810301E4B03A89D6A0FF0F4FF67
:10D2C000002203A9A847A8E7072AF4D106228DF86F
:10D2D0000C20B3F8012052BAADF810201A79D97891
:10D2E000120242EA014259790A4364214A430592F3
:10D2F0009B798DF81830DEE70A23A5E700228DF828
:10D300000C205B788DF8103003A80FF0FBFBFFE6D4
:10D310000D228DF80C205B788DF8103096E700BF59
:10D320001830002044300020D5D000082C300020D8
:10D330001C010020074B1A7852B15A7842B102788A
:10D34000042A05D1017A427AD973012098731A749C
:10D35000704700BF183000207FB51C4C01A81AF0A0
:10D36000E5FEE678002501A8E5701AF0E1FE1EB39F
:10D3700023780BB36378FBB1A27BA3685AB1032275
:10D38000E27105221A70E27B5A70227CA5739A70B2
:10D390000122A27004E0A278012A0FD0042AF7D05B
:10D3A000E02203930A4B8DF80820E2791B6B217968
:10D3B0008DF8092002A8984704B070BD0222E271DE
:10D3C000A2895A70110A1970EAE700BF18300020CC
:10D3D0001C010020004870471C0100201B2937B5A4
:10D3E000434B05460C460FD00CD80A2934D00D29E2
:10D3F00032D008290BD01A78012A5FD15B2C65D175
:10D40000022202E07F29F5E701221A7054E039492F
:10D4100000221A700B68002B4ED0013B0B6036497E
:10D420000824CA54284601220DF107018DF807404F
:10D4300005F010FD202301220DF1070128468DF88B
:10D44000073005F007FD01220DF1070128468DF890
:10D45000074005F0FFFC2FE0002227481A70F8F77C
:10D4600099FE00B304F018FB88B10A2301220DF1E4
:10D47000070128468DF8073005F0ECFC0D2301224A
:10D480000DF1070128468DF8073005F0E3FC1A4836
:10D49000F8F780FE18490246284600F08DF8174933
:10D4A000174805F033FD40F60102134800211CF037
:10D4B0000DFE104B00221A6003B030BD022A05D1C8
:10D4C000A4F14102012A01D800229EE70949002067
:10D4D00018700B6840F2FE729342EDD85A1C0A6035
:10D4E0000549CC54885404F0D7FA0028E4D0AAE7C0
:10D4F00048300020A03800209C30002000DF0208C7
:10D5000002E2020808B50B490B4805F0FFFC1422A3
:10D5100000210A481CF0DAFD40F60102084800210B
:10D520001CF0D4FD074B00221A60BDE8084000F053
:10D530003DBB00BF00DF020802E202084C300020C1
:10D540009C300020A0380020F8B505460C46164651
:10D55000F8F720FE07462846F8F71CFE38B30123EB
:10D56000002E63664FF0000308BF19262560184699
:10D57000626EB24219DAEA1814E01146013291F8EB
:10D5800000C0BCF13A0F0CD108705A1CA918AA5C53
:10D590005AB1626E02F1010CC4F864C044F8221062
:10D5A000E6E70133BB42E8DBEFD10020F8BD022003
:10D5B000FCE77020704700002DE9F04F0024ADF625
:10D5C000AC0D934681468846682221460FA8CDE9D6
:10D5D00003441CF07BFDBBF1010F0AD198F8003029
:10D5E0000D2B01D00A2B0ED120460DF6AC0DBDE857
:10D5F000F08FBBF1000F06D18C4B8D48996805F078
:10D6000085FC0224F0E7434600241D4613F8012B55
:10D6100012F0DF0F02D03D2A40F0AA802246414698
:10D6200007A81CF02BFD07AB00271F55013C95F800
:10D6300000A01B5D3F2B00F0A1807E4E002514232F
:10D6400003FB05F207A990591DF0ECFA14230446D8
:10D65000002840F04F81BAF13D0F40F0938007A8B9
:10D66000F8F798FD0130584500F0408114236B43D2
:10D6700006EB030AF058F8F78DFD01309AF8082000
:10D680000FA94044FFF760FF002F00F0ED80002D50
:10D6900040F097806848674C684E694FDFF8A48176
:10D6A00005F034FC6848CDE9055505F02FFC7025E0
:10D6B000E068F8F76FFDE0B10822002105A81CF032
:10D6C00005FD237CD80662D5604905A81DF0C4FA83
:10D6D000237CDB0707D505A8F8F75CFD05AB3946C9
:10D6E00018441DF0B9FAE368216805AA304605F030
:10D6F0000DFC013D04F11404DAD1554D554E564F41
:10D70000DFF8588140242B683BB33246394629A8BC
:10D710001DF068FA2869F8F73DFDF0B108220021F4
:10D7200005A81CF0D3FC2B7DD8063DD5474905A89C
:10D730001DF092FA2B7DDB0707D505A8F8F72AFD27
:10D7400005AB3F4918441DF087FA2B6900936B68BD
:10D7500005AA29A9404605F0D9FB013C05F11805A9
:10D76000D1D1324B53F824103D4805F0CFFB3BE7B5
:10D770000134202C7FF449AF0124F2E707AB1F5599
:10D7800001275AE7BAF1000F3FF47EAF6EE7590761
:10D7900001D5344999E79A079AD505A8F8F7FAFC14
:10D7A00005AB4146184491E7590701D52D49BEE71D
:10D7B0009A07BFD505A8F8F7EDFC05AB2149184439
:10D7C000B6E70822002103A81CF080FC142303FB09
:10D7D00005631B7CDF061BD51C4903A81DF03CFA22
:10D7E000142303FB05631B7CDA0707D503A8F8F7AE
:10D7F000D1FC03AB124918441DF02EFA14235D43EB
:10D8000073197159DB6803AA0C4805F07FFBA8E780
:10D81000580701D51349E0E79907E1D503A8F8F7C0
:10D82000B9FC03AB07491844D8E700BF60010020EA
:10D8300007E202088C0100200EE2020887E20208DB
:10D840000DF6020877F90208FEDE02087CE2020803
:10D85000A438002093E2020898E202089DE2020840
:10D8600004E2020884E20208142404FB0564237C19
:10D87000DB0681D47A490F98F8F782FC18B9237C2B
:10D8800013F0060F32D076490F98F8F779FC074667
:10D8900060B1289B002B2BDD142303FB05631B7C4D
:10D8A0005F0721D51C073FF567AF012714235D43B0
:10D8B00006EB05087159D8F804300FAA4846984776
:10D8C0000446002840F0C68098F8103059077FF5CC
:10D8D00048AF1A073FF545AF002F3FF442AF43F082
:10D8E000080388F810303CE7D807DED4022438E774
:10D8F0000027DBE70135702D7FF4A2AEDFF864B1BD
:10D9000000265D46DBF80020002A00F09B80564888
:10D91000042207A91DF0A8F9002840F09380DBF845
:10D92000000008A91DF07EF90446002840F08A8016
:10D93000BAF1000F0DD01823734305EB030AE85822
:10D94000F8F728FC05309AF80C200FA94044FFF79F
:10D95000FBFD1823734305EB0308434AEB58434987
:10D9600029A81DF03FF967B30822002103A81CF085
:10D97000ADFB95F8943ADF0616D53D4903A81DF096
:10D980006BF995F8943ADA0707D503A8F8F702FC83
:10D9900003AB384918441DF05FF9182303FB065503
:10D9A00003AA2B6929A92FE7580701D53249E5E7D2
:10D9B0009907E6D503A8F8F7EDFB03AB2F49184408
:10D9C000DDE798F81430DB063FF5D6AE24490F9812
:10D9D000F8F7D6FB28B998F8143013F0060F3FF487
:10D9E000CBAE1F490F98F8F7CBFB074660B1289BD9
:10D9F000002B25DD182303FB06531B7D5F071BD57A
:10DA00001C073FF5B9AE0127182303FB06550FAAE3
:10DA1000AB6829A9484698470446D8B92B7D5907D1
:10DA20007FF59FAE1A073FF59CAE002F3FF499AEED
:10DA300043F008032B7594E6D8077FF557AFE2E76C
:10DA40000027E1E70136402E0BF1180B7FF45AAFA7
:10DA5000092486E60A2C7FF684AE094B596883E6D2
:10DA60002DFF0208A438002093E2020898E2020881
:10DA70007CE202080DF6020884E2020877F9020847
:10DA80006001002002EBD2722DE9F84306465410E3
:10DA90004D1C0027BC4201DCBDE8F88315F8010CE1
:10DAA00095F800901DF014FAC0B2A0F130035FFAAF
:10DAB00083F8B8F1090F84BF37385FFA80F8484619
:10DAC0001DF006FAC2B2A2F13003DBB2092B84BF0B
:10DAD000373AD3B203EB0813F35502350137D9E7D0
:10DAE000F8B50F4606461446F8F754FBB84205460B
:10DAF00001D00120F8BD10F00107FAD1BBB29D4260
:10DB000007D86CB120462A463146FFF7BBFF0020FC
:10DB1000F0E7F05C1CF08AFA01370028EED1E8E764
:10DB20002046E7E713B50C4601AA0421FFF7D8FF0A
:10DB300028B9BDF804305BBA238002B010BD0120C3
:10DB4000FBE713B50C4601AA0821FFF7C9FF20B96E
:10DB5000019B1BBA236002B010BD0120FBE700004F
:10DB6000F8B505460C46F8F715FB0A28064601D914
:10DB70000120F8BD0C4928461DF098F807462846B4
:10DB8000F8F708FB8742F3D128461CF010FA20B9B9
:10DB9000012EEDD11CB12060EBE714B12060002014
:10DBA000E7E72046E5E700BFADE202082DE9F341D3
:10DBB00000F03AF8064600F041F8044628B302B0F7
:10DBC000BDE8F0812146684600F044F8104D70270A
:10DBD000009928681DF026F820B9019AD00609D5C9
:10DBE00085F81080013F05F11405F1D10134B442EC
:10DBF000E8DBE4E751072B7C03D59B07F2D02A74BE
:10DC0000F0E7134018BF2B74ECE74FF01008EEE775
:10DC10008C0100201130C0B211289ABF014B185C52
:10DC20000120704716FD0208024B0348C01AC008C5
:10DC3000704700BF200C0308200C0308034B186832
:10DC4000034B1B68C31A584258417047200C030805
:10DC5000200C030838B50546FFF7F0FF044640B92D
:10DC6000054B082203EBC10128461CF007FA2046A9
:10DC700038BD0120FCE700BF200C030870B5074E3B
:10DC80000446451814F8011B304605F03FF9AC4234
:10DC9000F8D1BDE87040024805F038B9C4E1020887
:10DCA000FEDE0208F0B58BB00E461546FBF7D2FB40
:10DCB000012859D16C6E012C01D0022415E02B49AA
:10DCC0002868F8F75DFA98B908210DEB0100FBF719
:10DCD000D7FA054648B93146254805F017F9082115
:10DCE0000DEB0100FFF7CAFF2C4620460BB0F0BD3C
:10DCF0006B6E012BE1D11F4B28681B88ADF80430F7
:10DD000000248DF80640F8F745FA1028D5D12B6885
:10DD1000185D1CF08BF90028CFD00134102CF6D1FF
:10DD200002AE0024374629680222214401A81CF0D3
:10DD3000A5F91022002101A81DF0C0F80234102C12
:10DD400006F8010BEFD108213846FCF799F9044693
:10DD50000028CAD0831D05D010F1110F0CBF0A2472
:10DD60000124C2E70324C0E70824BEE72DFF020810
:10DD700028FD020888D30208F0B58BB00E46154680
:10DD8000FBF768FB012857D16C6E012C01D00224EF
:10DD900013E02A492868F8F7F3F988B9102102A896
:10DDA000FBF770FA054640B93146254805F0AEF854
:10DDB000102102A8FFF762FF2C4620460BB0F0BDF1
:10DDC0006B6E012BE3D11F4B28681B88ADF8043024
:10DDD00000248DF80640F8F7DDF92028D7D12B680C
:10DDE000185D1CF023F90028D1D00134202CF6D185
:10DDF00002AE0024374629680222214401A81CF003
:10DE00003DF91022002101A81DF058F80234202C01
:10DE100006F8010BEFD110213846FCF752F9044601
:10DE20000028CAD0831D05D010F1110F0CBF0A24A1
:10DE30000124C2E70324C0E70824BEE72DFF02083F
:10DE400028FD020888D30208F0B58BB00E461546AF
:10DE5000FBF700FB012857D16C6E012C01D0022486
:10DE600013E02A492868F8F78BF988B9102102A82D
:10DE7000FBF714FB054640B93146254805F046F846
:10DE8000102102A8FFF7FAFE2C4620460BB0F0BD89
:10DE90006B6E012BE3D11F4B28681B88ADF8043053
:10DEA00000248DF80640F8F775F92028D7D12B68A3
:10DEB000185D1CF0BBF80028D1D00134202CF6D11D
:10DEC00002AE0024374629680222214401A81CF032
:10DED000D5F81022002101A81CF0F0FF0234202CFC
:10DEE00006F8010BEFD110213846FCF714F904466F
:10DEF0000028CAD0831D05D010F1110F0CBF0A24D1
:10DF00000124C2E70324C0E70824BEE72DFF02086E
:10DF100028FD020888D30208F7B50E461546FBF720
:10DF200099FA012862D16C6E012C01D002241EE006
:10DF30002F492868F8F724F9E0B904210DEB010016
:10DF4000FBF7DAFA054690B931462A4804F0DEFFBD
:10DF50002C46294D01AE16F8011B2846013404F069
:10DF6000D5FF042CF7D1254804F0D0FF002420462B
:10DF700003B0F0BD6B6E012BD8D1214B28681B88F4
:10DF8000ADF8003000248DF80240F8F703F90828B6
:10DF9000CCD12B68185D1CF049F80028C6D001349C
:10DFA000082CF6D101AE002437462968022221440C
:10DFB00068461CF063F81022002168461CF07EFFC2
:10DFC0000234082C06F8010BEFD104213846FCF787
:10DFD000C3F804460028CAD0831D05D010F1110FE4
:10DFE0000CBF0A240124C2E70324C0E70824BEE7CB
:10DFF0002DFF020828FD0208C4E10208FEDE020827
:10E0000088D30208F0B58BB00E461546FBF722FA0E
:10E01000012859D16C6E012C01D0022415E02B4946
:10E020002868F8F7ADF898B908210DEB0100FBF767
:10E030002BF9054648B93146254804F067FF082109
:10E040000DEB0100FFF71AFE2C4620460BB0F0BD89
:10E050006B6E012BE1D11F4B28681B88ADF8043093
:10E0600000248DF80640F8F795F81028D5D12B68D4
:10E07000185D1BF0DBFF0028CFD00134102CF6D147
:10E0800002AE0024374629680222214401A81BF071
:10E09000F5FF1022002101A81CF010FF0234102C03
:10E0A00006F8010BEFD108213846FCF778F8044652
:10E0B0000028CAD0831D05D010F1110F0CBF0A240F
:10E0C0000124C2E70324C0E70824BEE72DFF0208AD
:10E0D00028FD020888D3020873B50E461546FBF7E3
:10E0E000B9F901282CD16C6E012C03D002242046F2
:10E0F00002B070BD13492868F8F742F80028F5D13E
:10E1000004210DEB0100FBF722FA05460028EED1B1
:10E1100031460D4804F0FAFE9DF806100B4804F055
:10E12000F5FE9DF80510094804F0F0FE9DF8041076
:10E13000064804F0EBFE064804F0E8FE2C46D6E75D
:10E140000824D4E72DFF020828FD0208C4E10208D4
:10E15000FEDE0208F0B58BB00E461546FBF77AF9E5
:10E16000012857D16C6E012C01D0022413E02A49FA
:10E170002868F8F705F888B9102102A8FBF715FA06
:10E18000054640B93146254804F0C0FE102102A8DA
:10E19000FFF774FD2C4620460BB0F0BD6B6E012BD3
:10E1A000E3D11F4B28681B88ADF8043000248DF89C
:10E1B0000640F7F7EFFF2028D7D12B68185D1BF03A
:10E1C00035FF0028D1D00134202CF6D102AE002436
:10E1D000374629680222214401A81BF04FFF102274
:10E1E000002101A81CF06AFE0234202C06F8010B65
:10E1F000EFD110213846FBF7FAFF04460028CAD0B9
:10E20000831D05D010F1110F0CBF0A240124C2E7B1
:10E210000324C0E70824BEE72DFF020828FD0208FA
:10E2200088D30208F0B5556E012D85B00F4614460F
:10E230001ED110491068F7F7A3FF064680B968465B
:10E24000FBF724F8012808D139460B4804F05EFE9C
:10E2500010216846FFF712FD3546284605B0F0BD8F
:10E26000636E012B04D12068F7F794FF2028F4D0C7
:10E270000225F2E72DFF020828FD020873B50E46BD
:10E280001546FBF7E7F8012826D16B6E012B01D06C
:10E2900002240CE011492868F7F772FF044648B9D8
:10E2A000FAF7F8FF314602460D4804F02FFE2046EB
:10E2B00002B070BD6B6E012BEAD128680DF1070129
:10E2C000FFF74EFC0028E3D19DF807000728DFD8B0
:10E2D000FAF7E2FF0446EAE70824E8E72DFF020820
:10E2E0002CFD020870B50E461546FBF7B3F8012861
:10E2F00032D16B6E012B02D00224204670BD17492B
:10E300002868F7F73DFF044638B9FAF7CCFF3146E5
:10E310000246134804F0FAFDEFE76B6E012BEBD1D8
:10E32000002406E02B68185D1BF078FE0028E3D07F
:10E3300001342868F7F72EFFA042F3D828680A2294
:10E3400000211CF0BBFD0128D6D8C0B2FAF7ADFF02
:10E35000041E18BF0124D0E70824CEE72DFF0208D1
:10E360002CFD020838B50D461446FBF773F801285A
:10E3700014D1636E012B02D00224204638BD2068E0
:10E380000749F7F7FDFE04460028F5D1FAF790FF9C
:10E3900029460246034804F0B9FDEEE70824ECE7FD
:10E3A0002DFF02082CFD02082DE9F04186B00F4632
:10E3B0001546FBF74FF8012877D13E4B0FCB02AE45
:10E3C00086E80F006B6E012B1CD13B492868F7F7DC
:10E3D000D7FE0446B0B9FBF7B5FC0546FBF7B4FC25
:10E3E0000646FBF7B3FC8046FBF7B2FC3346CDE9AB
:10E3F00000802A463148394604F088FD204606B0A0
:10E40000BDE8F0816B6E042B2EDD0224F6E755F893
:10E410002430D85D1BF002FE0028F6D0013755F8F5
:10E420002400F7F7B7FEB842F1D801346B6EA3426F
:10E4300018DC00246B6EA34218DC002B20D10123D2
:10E440000293DDE90423DDE90201FBF703FF044643
:10E450000028D3D0831D2AD010F1110F0CBF0A243D
:10E460000124CBE70027DAE70024DFE755F8240092
:10E470000A2200211CF022FD013446F8040BD9E7E2
:10E48000029ADEDD012AC0D8012B039AD9D0012AD5
:10E49000BBD8022B049AD4D0073AF82AB5D8042B5B
:10E4A000059ACED1FF2ACCD9AFE70824A6E70324EA
:10E4B000A4E700BF8CD302082DFF020834FD020838
:10E4C00070B50E461546FAF7C5FF012838D16B6EB8
:10E4D000012B02D00224204670BD1A492868F7F7A4
:10E4E0004FFE044638B9FAF7C4FF314602461648D3
:10E4F00004F00CFDEFE76B6E012BEBD1002406E07E
:10E500002B68185D1BF08AFD0028E3D001342868D1
:10E51000F7F740FEA042F3D828680A2200211CF039
:10E52000CDFC0128D6D80121C0B2FCF73DF8044645
:10E530000028D0D010F1110F0CBF0A240124CAE723
:10E540000824C8E72DFF02082CFD020838B50D4647
:10E550001446FAF77FFF012814D1636E012B02D015
:10E560000224204638BD20680749F7F709FE044613
:10E570000028F5D1FAF77FFF29460246034804F048
:10E58000C5FCEEE70824ECE72DFF02082CFD02088D
:10E590002DE9F041C2B00E461446FAF75BFF0128A0
:10E5A0002FD1636E012B04D00224204642B0BDE877
:10E5B000F08120681449F7F7E3FD04460028F3D101
:10E5C0004FF4807202A90DF10700FBF7C3FB31463F
:10E5D00005469DF807200D48DFF8348004F096FCCE
:10E5E000EDB202AE2746FBB29D4203D8094804F0C3
:10E5F0008DFCDAE716F8011B404604F087FC013772
:10E60000F1E70824D1E700BF2DFF020845FD02080D
:10E61000C4E10208FEDE02082DE9F043ADF61C0D50
:10E620001546FAF717FF012870D16B6E022B4DD1FA
:10E63000374B28681B8AADF80C3000248DF80E404B
:10E64000F7F7A8FD0646B44228683BD11BF0AFFCA3
:10E65000C0B2431EDBB2DE2B38D808238DF8100081
:10E6600068688DF81230F7F795FD10F0010404AEDC
:10E6700007462BD1431EB3F5FA7F27D2BC4229D1DE
:10E680000DF1180864080027C146A7422AD10023CB
:10E69000F3707370009396E80C0039464846FBF718
:10E6A00075F858B110F10C0F2CD0821D2CD0C31C62
:10E6B0000CD010F1110F0CBF0A2001200DF61C0D1B
:10E6C000BDE8F083005D1BF0A9FC08B90220F5E766
:10E6D0000134B8E76B68185D1BF0A8FC0028F5D082
:10E6E0000134CBE76968022201EB470103A81BF064
:10E6F000C5FC1022002103A81CF0E0FB013708F83C
:10E70000010BC2E70620D9E70320D7E70820D5E7A9
:10E710008CD30208F0B5ADF2044D1446FAF79AFE18
:10E7200001287AD1636E012B55D0636E032B58D12B
:10E7300000252068F7F72EFDA84256D8002560680E
:10E74000F7F728FDA84258D80025A068F7F722FD62
:10E75000A8425AD82068F7F71DFD032841D8606801
:10E76000F7F718FD01283CD80A22002120681CF088
:10E77000A5FB00210A22054660681CF09FFB0646A7
:10E78000A068F7F707FDC10787B22AD4B7F5006F75
:10E7900027D8B3B2012B24D86A1E92B2DE2A20D821
:10E7A000A0686A463946FFF79BF9D0B97B086A46EC
:10E7B00006F00101E8B2FDF753FB98B110F10C0F20
:10E7C0002DD0821D2DD0C31C0BD010F1110F0CBF0A
:10E7D0000A20012006E014492068F7F7D1FC002840
:10E7E000A3D102200DF2044DF0BD2368585D1BF04B
:10E7F00015FC0028F5D001359BE76368585D1BF0D8
:10E800000DFC0028EDD0013599E7A368585D1BF099
:10E810000DFC0028E5D0013597E70820E2E7062047
:10E82000E0E70320DEE700BF2DFF020870B50E46CB
:10E830001546FAF70FFE01283CD16B6E012B02D072
:10E840000224204670BD1D492868F7F799FC04464C
:10E8500038B9FAF7D8FE31460246194804F056FB9B
:10E86000EFE76B6E012BEBD1002406E02B68185DFF
:10E870001BF0D4FB0028E3D001342868F7F78AFCAA
:10E88000A042F3D828680A2200211CF017FB0128B7
:10E89000D6D801210840FBF714FE04460028D0D04A
:10E8A000821D09D0C31CCBD010F1110F0CBF0A245C
:10E8B0000124C6E70824C4E70324C2E72DFF0208A9
:10E8C0004CFD02082DE9F0410E469046FAF7C2FDD4
:10E8D00001285ED1D8F86470012F58D13049D8F89A
:10E8E0000000F7F74DFC054620BBFAF78EFE012825
:10E8F0000AD002281BD000284DD12A48314604F006
:10E9000005FB2846BDE8F081FBF73CFB31460328B8
:10E910000BD8DFE800F0020406082348EFE723489D
:10E92000EDE72348EBE72348E9E72348E7E72348F7
:10E930003146E4E7D8F86450012D28D12049D8F8B1
:10E9400000001CF06FF930B92946FBF7E1FD0446E1
:10E9500008B90025D5E71B49D8F800001CF062F97A
:10E9600030B901210846FBF7D3FD04460028F0D05A
:10E970001549D8F800001CF055F930B901210220E2
:10E98000FBF7C6FD04460028E3D0113405D002256C
:10E99000B7E70825B5E73D46B3E70A25B1E700BF6D
:10E9A0002DFF020854FD02085BFD020865FD020808
:10E9B0006FFD020879FD020883FD02088AFD020846
:10E9C00091FD020871DC02087FF2020870B50E4664
:10E9D0001446FAF73FFD01282ED1636E012B12D0A9
:10E9E00000252068F7F7D6FB85421CD320680A2251
:10E9F00000211CF063FAC0B2012819D8BDE87040AC
:10EA00000121FAF70BBE0D492068F7F7B9FB05465F
:10EA10000028E5D1FAF7FBFD31460246084804F02C
:10EA200075FA284670BD2368585D1BF0F7FA08B9DF
:10EA30000225F6E70135D4E70825F2E72DFF0208A5
:10EA40004CFD020870B50E461546FAF703FD012885
:10EA500038D16B6E012B02D00224204670BD1A49BA
:10EA60002868F7F78DFB044638B9FAF7E4FD31461C
:10EA70000246164804F04AFAEFE76B6E012BEBD121
:10EA8000002406E02B68185D1BF0C8FA0028E3D0CC
:10EA900001342868F7F77EFBA042F3D80A22002150
:10EAA00028681CF00BFA0121C0B2FBF72DFE0446CA
:10EAB0000028D2D0C31CCFD010F1110F0CBF0A24F4
:10EAC0000124CAE70824C8E72DFF02082CFD02082C
:10EAD00070B50E461546FAF7BDFC012846D16B6E9F
:10EAE000012B02D00224204670BD21492868F7F787
:10EAF00047FB044650B9FAF7ABFD4FF47A72314642
:10EB0000B0FBF2F21B4804F001FAECE76B6E012B4C
:10EB1000E8D1002406E02B68185D1BF07FFA00287E
:10EB2000E0D001342868F7F735FBA042F3D8286815
:10EB30000A2200211CF0C2F9431E0D2B0446D1D835
:10EB4000FAF788FD4FF47A72B0FBF2F3A342C9D909
:10EB500002FB04F00121FBF745FF04460028C2D068
:10EB600010F1110F0CBF0A240124BCE70824BAE7F6
:10EB70002DFF02082CFD020870B50E461546FAF767
:10EB800069FC012846D16B6E012B02D0022420467D
:10EB900070BD21492868F7F7F3FA044650B9FAF72F
:10EBA00059FD4FF47A723146B0FBF2F21B4804F083
:10EBB000ADF9ECE76B6E012BE8D1002406E02B6881
:10EBC000185D1BF02BFA0028E0D001342868F7F715
:10EBD000E1FAA042F3D828680A2200211CF06EF95D
:10EBE000831E0D2B0446D1D8FAF732FD4FF47A720A
:10EBF000B0FBF2F3A342C9D202FB04F00121FBF700
:10EC000010FF04460028C2D010F1110F0CBF0A24D7
:10EC10000124BCE70824BAE72DFF02082CFD0208F6
:10EC200070B50E461546FAF715FC012838D16B6E03
:10EC3000012B02D00224204670BD1A492868F7F73C
:10EC40009FFA044638B9FAF707FD314602461648DE
:10EC500004F05CF9EFE76B6E012BEBD1002406E0CA
:10EC60002B68185D1BF0DAF90028E3D0013428681E
:10EC7000F7F790FAA042F3D828680A2200211CF086
:10EC80001DF90128D6D801210840FBF7E9FE04460A
:10EC90000028D0D010F1110F0CBF0A240124CAE7BC
:10ECA0000824C8E72DFF02084CFD020870B50E4687
:10ECB0001546FAF7CFFB01283ED16B6E012B02D02F
:10ECC0000224204670BD1D492868F7F759FA04460A
:10ECD00050B9FAF7C3FC4FF47A723146B0FBF2F246
:10ECE000174804F013F9ECE76B6E012BE8D1002410
:10ECF00006E02B68185D1BF091F90028E0D0013484
:10ED00002868F7F747FAA042F3D828680A220021BA
:10ED10001CF0D4F8431E0E2BD2D84FF47A73012185
:10ED20005843FBF7BDFE04460028CAD010F1110F6E
:10ED30000CBF0A240124C4E70824C2E72DFF0208FF
:10ED40002CFD020870B50E461546FAF783FB012824
:10ED50003ED16B6E012B02D00224204670BD1D49AE
:10ED60002868F7F70DFA044650B9FAF790FC4FF40B
:10ED70007A723146B0FBF2F2174804F0C7F8ECE7BC
:10ED80006B6E012BE8D1002406E02B68185D1BF0A8
:10ED900045F90028E0D001342868F7F7FBF9A042D4
:10EDA000F3D828680A2200211CF088F8831E0E2B55
:10EDB000D2D84FF47A7301215843FBF7A0FE0446E2
:10EDC0000028CAD010F1110F0CBF0A240124C4E797
:10EDD0000824C2E72DFF02082CFD020870B50E467C
:10EDE0001546FAF737FB012838D16B6E012B02D09C
:10EDF0000224204670BD1A492868F7F7C1F9044675
:10EE000038B9FAF7A9FC31460246164804F07EF8F4
:10EE1000EFE76B6E012BEBD1002406E02B68185D49
:10EE20001BF0FCF80028E3D001342868F7F7B2F9AA
:10EE3000A042F3D80A22002128681CF03FF80121E3
:10EE4000C0B2FBF7DBFE04460028D2D0C31CCFD0F3
:10EE500010F1110F0CBF0A240124CAE70824C8E7E7
:10EE60002DFF02082CFD020870B50E461546FAF774
:10EE7000F1FA012837D16B6E012B02D00224204613
:10EE800070BD1A492868F7F77BF9044638B9FAF7D4
:10EE900053FC31460246164804F038F8EFE76B6E33
:10EEA000012BEBD1002406E02B68185D1BF0B6F8AF
:10EEB0000028E3D001342868F7F76CF9A042F3D8B2
:10EEC0000A22002128681BF0F9FF0121FBF770FEE0
:10EED00004460028D3D0C31CD0D010F1110F0CBFB2
:10EEE0000A240124CBE70824C9E700BF2DFF02084C
:10EEF0002CFD020870B50E461546FAF7ABFA01284C
:10EF00003AD16B6E012B02D00224204670BD1B4902
:10EF10002868F7F735F9044638B9FAF7BAFB3146ED
:10EF20000246174803F0F2FFEFE76B6E012BEBD1BF
:10EF3000002406E02B68185D1BF070F80028E3D071
:10EF400001342868F7F726F9A042F3D828680A2286
:10EF500000211BF0B3FFC0B20F28D5D80121FBF769
:10EF6000FDFD04460028D0D0C31CCDD010F1110FF8
:10EF70000CBF0A240124C8E70824C6E72DFF0208B5
:10EF80002CFD020873B50E461546FAF763FA012800
:10EF900022D16B6E012B0FD110492868F7F7F0F8DA
:10EFA000044648B9FAF7E8FB314602460C4803F03C
:10EFB000ADFF204602B070BD28680DF10701FEF7D5
:10EFC000CFFD38B99DF80700022803D8FAF7D6FB21
:10EFD0000446EEE70224ECE70824EAE72DFF0208E6
:10EFE0004CFD020873B50E461546FAF733FA0128B0
:10EFF00025D16B6E012B0FD112492868F7F7C0F8A5
:10F00000044648B9FAF784FE314602460E4803F03A
:10F010007DFF204602B070BD28680DF10701FEF7A4
:10F020009FFD50B99DF80700012806D8FAF776FE33
:10F0300040B2FEF7EFFD0446EBE70224E9E70824BF
:10F04000E7E700BF2DFF02084CFD020873B50E462E
:10F050001546FAF7FFF9012825D16B6E012B0FD168
:10F0600012492868F7F78CF8044648B9FAF7EDFF1B
:10F07000314602460E4803F049FF204602B070BDFB
:10F0800028680DF10701FEF76BFD50B99DF80700E8
:10F09000012806D8FAF7DBFF40B2FEF7BBFD0446B5
:10F0A000EBE70224E9E70824E7E700BF2DFF0208A9
:10F0B0004CFD020870B50E461546FAF7CBF901284B
:10F0C0001CD16B6E012B0ED10D492868F7F758F84B
:10F0D000044640B9FAF7BDFF31460246094803F03D
:10F0E00015FF204670BD28681AF061FF00B2FAF7DC
:10F0F000B2FF40B2FEF78EFD0446F2E70824F0E7C7
:10F100002DFF02084CFD020873B50E461546FAF7AE
:10F11000A1F9012821D16B6E012B0FD1104928686C
:10F12000F7F72EF8044648B9FAF797FF314602463A
:10F130000C4803F0EBFE204602B070BD286801A920
:10F14000FEF70EFD08B10224F5E70198FAF787FFF4
:10F1500040B2FEF75FFD0446EDE70824EBE700BF91
:10F160002DFF02084CFD020870B50E461446FAF752
:10F1700071F9012830D1636E012B02D00225284697
:10F1800070BD16492068F6F7FBFF054638B9FAF757
:10F1900082FA31460246124803F0B8FEEFE7636E8A
:10F1A000012BEBD1002506E02368585D1AF036FFED
:10F1B0000028E3D001352068F6F7ECFFA842F3D829
:10F1C00020680A2200211BF079FEC0B20728D5D89A
:10F1D000FAF763FA0025D2E70825D0E72DFF0208E9
:10F1E0002CFD0208F7B50E461546FAF733F901284B
:10F1F00027D1164B1B78042B25D1FAF75CFA07466A
:10F20000FAF74DFA6B6E012B044603D0022528460F
:10F2100003B0F0BD28680E49F6F7B2FF0546002896
:10F22000F4D10C48B4FBF0F3FAB200FB13443146BE
:10F230004FF47A70B4FBF0F40748009403F066FED4
:10F24000E5E70825E3E70525E1E700BFCC2100203D
:10F250002DFF020840420F0093FD020838B50D460D
:10F260001446FAF7F7F8012818D10E4B1B78042B37
:10F2700016D1636E012B02D00224204638BD2068CF
:10F280000949F6F77DFF04460028F5D1FAF720FA80
:10F2900029460246054803F039FEEEE70824ECE76C
:10F2A0000524EAE7CC2100202DFF02082CFD0208EE
:10F2B00030B58BB00D461446FAF7CCF8012822D1B0
:10F2C000134B1B78042B20D1636E012B03D0022437
:10F2D00020460BB030BD20680E49F6F751FF0446BA
:10F2E0000028F4D105A8FAF74FFD079B0293069B6F
:10F2F0000193099B0093BDF81420089B06482946FA
:10F3000003F004FEE4E70824E2E70524E0E700BF99
:10F31000CC2100202DFF0208A1FD020830B589B0E4
:10F320000D461446FAF796F801281CD1636E012B9E
:10F3300003D00224204609B030BD20680B49F6F7FF
:10F340001FFF04460028F4D1014600901A2201A8AC
:10F350001AF0BCFE6846FAF7CDF96A462946044819
:10F3600003F0D4FDE6E70824E4E700BF2DFF020820
:10F37000B5FD020838B50D461446FAF76BF8A0B192
:10F38000636E012B02D00224204638BD2068084954
:10F39000F6F7F6FE04460028F5D1FAF79FF929465C
:10F3A0000246044803F0B2FDEEE70824ECE700BF94
:10F3B0002DFF02084CFD0208F7B50D461446FAF77A
:10F3C00049F801282DD1636E012B03D00224204679
:10F3D00003B0F0BD20681449F6F7D2FE04460028B9
:10F3E000F4D129461148124E124F03F08FFD2546E5
:10F3F0006846FCF729FF0E3003D00F4803F086FD66
:10F40000E5E7BDF80430002BF2D015B1304603F02B
:10F410007DFD9DF906200099384603F077FD013502
:10F42000E6E70824D3E700BF2DFF020828FD020805
:10F43000BDFD020871DA0208FEDE020838B50D468D
:10F440001446FAF707F8A0B1636E012B02D002242C
:10F45000204638BD20680849F6F792FE0446002889
:10F46000F5D1FAF741F929460246044803F04EFD6A
:10F47000EEE70824ECE700BF2DFF02084CFD020870
:10F4800030B599B01446F9F7E5FF012840F08580C2
:10F49000636E043B032B02D9022019B030BD4049F2
:10F4A0002068F6F76DFE002854D1012360688DF8BE
:10F4B0002C300CA9FEF745FB0028EDD1A06811AA5D
:10F4C0002021FEF70DFB0028E6D1E0680DAA2021DF
:10F4D000FEF706FB0028DFD1636E1590052B8DF833
:10F4E0005800ADF85A00D7D012DD206915A9FEF7F3
:10F4F00037FB0028D0D160690378302B46D12949E9
:10F50000F6F73EFE002839D10A900A9B8DF8583054
:10F51000636E072B0ED1A0690AA9FEF721FB002814
:10F52000BAD10A9B072BB7D89DF82C20012A2FD1DE
:10F53000ADF85A300FAD0FCD6C460FC40FCD0FC4D0
:10F540002B6823600BAB0FCBFCF7CEFC40B2FEF771
:10F5500061FBA2E714492068F6F712FE0028A4D048
:10F5600012492068F6F70CFE08B902239EE71049FD
:10F570002068F6F705FE0028F7D08DE760690AA934
:10F580000130FEF7EDFA0028BFD085E70AA9F8E7B9
:10F59000022ACFD1002BCDD07EE708207DE700BF27
:10F5A000BFFD020823FF020871DC0208E9FE020821
:10F5B0007FF2020813B51446F9F74CFF01280ED16B
:10F5C000636E012B08D1206801A9FEF7BAFA18B9B9
:10F5D0000198FCF781FD00B1022002B010BD0820A7
:10F5E000FBE700002DE9F04F8FB01546F9F732FF29
:10F5F0000128044662D16B6E012B04D002252846F7
:10F600000FB0BDE8F08F28682D49F6F7B9FD054623
:10F610000028F3D1DFF8AC80DFF8AC90DFF8ACA0C5
:10F6200001A8FCF77DFD0E3003D0294803F06EFCE5
:10F63000E5E7012C02D9404603F068FC029B002B51
:10F6400035D12448DFF890B003F060FC02992348DC
:10F6500003F05CFC07AF002617F8011B5846013683
:10F6600003F054FC102EF7D11D48DFF86CB003F006
:10F670004DFC03AF002617F8011B5846013603F076
:10F6800045FC102EF7D1164803F040FC0B991548A5
:10F6900003F03CFC9DF93010134803F037FC0134B3
:10F6A000BDF83210114803F031FCE4B2B8E79DF820
:10F6B0000430012B0CBF50464846C3E708259EE79F
:10F6C0002DFF0208BDFD0208C7FD0208C4FD0208A7
:10F6D000FEDE0208C1FD0208C4E10208CAFD0208FC
:10F6E000C2FD0208D0FD0208D6FD020874DA020845
:10F6F000F7B50F461646F9F7ADFE012849D1F9F7DF
:10F70000DDFD746E012C054601D002241AE0224969
:10F710003068F6F735FDC0B90DF10600F9F7D0FDF8
:10F7200080B93946BDF806201C4803F0EFFBFAF714
:10F73000E7FB011E02DD1A4803F0E8FB194803F05D
:10F74000E5FB0024204603B0F0BD736E012BDCD135
:10F7500030680DF10601FEF7E5F90028D5D1082D36
:10F7600001D0012D0ED1BDF80630B3F5807FCCD885
:10F7700001210DF10600F9F7D1FD40B2FEF74AFA7A
:10F780000446DFE7022DF3D1BDF80630B3F5006F74
:10F79000EDE70824D6E700BF2DFF0208DCFD0208D4
:10F7A000E4FD0208FEDE02082DE9F3410F4615468E
:10F7B000F9F750FE012840F0BA806E6E012E38D164
:10F7C0005C492868F6F7DCFC98BB0DF10600F9F7F8
:10F7D00077FD0446002840F0AA8039465648574F26
:10F7E000DFF85C8103F092FB3546BDF80630DB079D
:10F7F00009D5012D02D0404603F088FB314638463A
:10F8000003F084FB0135BDF806305B080136ADF826
:10F810000630002BE9D1FAF773FB011E02DD4948DF
:10F8200003F074FB484803F071FB204602B0BDE8CA
:10F83000F0816B6E013B0B2B0AD80024ADF806401B
:10F84000002608E055F82430985D1AF0E7FB08B967
:10F850000224EAE7013655F82400F6F79BFCB04293
:10F86000F0D855F824000A2200211BF027FB0C28B1
:10F870000646EDD8F9F722FD082801D0012801D16C
:10F88000082EE5D8013E0B2E0DD8DFE806F006194C
:10F890001E23282D32373C41464BBDF8063043F03D
:10F8A0000103ADF806306B6E0134A342C8DC0121C0
:10F8B0000DF10600F9F732FD041E18BF0324B4E76A
:10F8C000BDF8063043F00203EBE7BDF8063043F025
:10F8D0000403E6E7BDF8063043F00803E1E7BDF8AE
:10F8E000063043F01003DCE7BDF8063043F0200398
:10F8F000D7E7BDF8063043F04003D2E7BDF8063045
:10F9000043F08003CDE7BDF8063043F48073C8E7C9
:10F91000BDF8063043F40073C3E7BDF8063043F486
:10F920008063BEE7BDF8063043F40063B9E70824FE
:10F930007BE700BF2DFF020828FD0208FEFD02083C
:10F94000C2FD0208E4FD0208FEDE020870B50E46A4
:10F950001546F9F77FFD012840F08C806B6E012B76
:10F9600002D00224204670BD44492868F6F708FCFE
:10F970000446002831D13146414803F0C7FAF9F76F
:10F980009DFC162878D8DFE800F01E1A10770C16B8
:10F990001C14181226777777777777777777202276
:10F9A0002400384803F0B2FADCE73748FAE7374872
:10F9B000F8E73748F6E73748F4E73748F2E73748DB
:10F9C000F0E73748EEE73748ECE73748EAE73748EB
:10F9D000E8E73748E6E73748E4E76C6E012CC0D12A
:10F9E00000262CE02B68985D1AF018FB30BB3249DA
:10F9F0002868F6F7C5FB80B130492868F6F7C0FBE8
:10FA000080B12F492868F6F7BBFB68B12D492868FB
:10FA1000F6F7B6FB0028A4D11620FBF7A9FA28B9FF
:10FA200000249FE71420F8E71520F6E7821D01D196
:10FA3000032497E7113095D10A2493E7013628680B
:10FA4000F6F7A8FBB042CDD828680A2200211BF0A7
:10FA500035FA0C2885D81C4B185CFBF789FA00286E
:10FA6000DED0831DE4D010F1110FE5D003307FF418
:10FA700079AF76E7082475E7012473E72DFF0208C4
:10FA800028FD02081AFE02081FFE020824FE0208D2
:10FA90007FFD020801FE020805FE020809FE0208B9
:10FAA0000DFE020811FE020815FE020819FE0208EA
:10FAB0001EFE020823FE020828FE02082CFE020891
:10FAC00030FE020834FE020838FE020870B50E4609
:10FAD0001546F9F7BFFC012802D00824204670BD66
:10FAE0006B6E012B01D00224F8E717492868F6F75E
:10FAF00047FB044658B9FAF703FA0028EDDBFAF79A
:10FB0000FFF931460246114803F000FAE6E76B6E52
:10FB1000012BE8D1002406E02B68185D1AF07EFA6C
:10FB20000028E0D001342868F6F734FBA042F3D86F
:10FB30000A22002128681BF0C1F9FAF731F940B216
:10FB4000FEF768F80446C9E72DFF02084CFD0208DD
:10FB500037B5536E0D461BB10224204603B030BDAD
:10FB60000DF10600FBF7B2FC044630B9BDF90620E2
:10FB70000548294603F0CAF9EFE7C21CECD0831D03
:10FB80000CBF03240124E8E74CFD020810B5536EB6
:10FB900013B10224204610BDFBF74CFC044618B9F3
:10FBA000054803F0B3F9F5E7C21CF2D0831D0CBF82
:10FBB00003240124EEE700BF45FE020807B5536E9B
:10FBC000012B03D0022003B05DF804FB106801A9EB
:10FBD000FDF7C6FF0028F5D10198FBF711FD0028BD
:10FBE000F1D0C21CEED0831D0CBF03200120EAE738
:10FBF00007B5536E012B03D0022003B05DF804FB60
:10FC0000106801A9FDF7ACFF0028F5D10198FBF7BA
:10FC10007BFD0028F1D0C21CEED0831D0CBF032059
:10FC20000120EAE770B5536E012BA0B00E461446D2
:10FC300028D142491068F6F7A3FA054610BB0BA875
:10FC4000FBF7D4FC1B9B09931A9B0893159B079306
:10FC50009DF8433006930B9B0593199B0493189BC7
:10FC600003939DF8383002930D9B01930C9B0093F6
:10FC7000179A9DF950303248314603F047F928462B
:10FC800020B070BD636E0C2B01D00225F7E7206811
:10FC900017A9FDF765FF0028F7D1606814A9FDF7E3
:10FCA0005FFF0028F1D1A0680CA9FDF759FF0028DB
:10FCB000EBD1E0680DA9FDF753FF0028E5D12069DD
:10FCC0000EA9FDF74DFF0028DFD1606918A9FDF7E7
:10FCD00047FF0028D9D1A06919A9FDF741FF0028E5
:10FCE000D3D1E0690BA9FDF73BFF0028CDD1206AF5
:10FCF0000DF14301FDF734FF0028C6D1606A15A954
:10FD0000FDF72EFF0028C0D1A06A1AA9FDF728FF31
:10FD10000028BAD1E06A1BA9FDF722FF0028B4D160
:10FD20000BA8FBF72DFC05460028A8D0C21CACD0C0
:10FD3000831D0CBF03250125A1E700BF2DFF02088D
:10FD40004DFE020870B5536E012B98B00E46144656
:10FD500015D11E491068F6F713FA054678B903A8BD
:10FD6000FBF744FC179B0193169B00931848DDE9B1
:10FD70001423314603F0CAF8284618B070BD636EEC
:10FD8000042B01D00225F7E7206814A9FDF7E8FE4F
:10FD90000028F7D1606815A9FDF7E2FE0028F1D12F
:10FDA000A06816A9FDF7DCFE0028EBD1E06817A9D2
:10FDB000FDF7D6FE0028E5D1DDE914239A42E1D80B
:10FDC00003A8FBF713FD0546D6E700BF2DFF020889
:10FDD00034FD020870B5536E012B98B00E461446E0
:10FDE00015D11E491068F6F7CBF9054678B903A876
:10FDF000FBF7FCFB179B0193169B00931848DDE96A
:10FE00001423314603F082F8284618B070BD636EA3
:10FE1000042B01D00225F7E7206814A9FDF7A0FE06
:10FE20000028F7D1606815A9FDF79AFE0028F1D1E6
:10FE3000A06816A9FDF794FE0028EBD1E06817A989
:10FE4000FDF78EFE0028E5D1DDE914239A42E1D8C2
:10FE500003A8FBF757FD0546D6E700BF2DFF0208B4
:10FE600034FD020810B5546E1CB9FBF705FB2046A3
:10FE700010BD0224FBE7000070B5536E012B0E4647
:10FE8000154602D00224204670BD0F491068F6F7CF
:10FE900077F9044630B90D4B0D481A68314603F026
:10FEA00035F8F0E76B6E012BECD10A2228680021AF
:10FEB0001BF004F8054A01281060E3D8FBF7C6FEE2
:10FEC000041E18BF0124DEE72DFF0208A43E002017
:10FED0002CFD020870B5536E012B86B00E461546F8
:10FEE00013D11B491068F6F74BF9044668B903A80B
:10FEF000FBF780FE059B00931648DDE9032331469E
:10FF000003F004F8204606B070BD6C6E032C01D0DF
:10FF10000224F7E7286803A9FDF722FE0028F7D19D
:10FF2000686804A9FDF71CFE0028F1D1A86805A99E
:10FF3000FDF716FE0028EBD103A8FBF765FE28B1FC
:10FF4000C31CE5D0063018BF0124DBE70446D9E71F
:10FF50002DFF020876FE020870B5084E451E00F11E
:10FF60000F0415F8011F304602F0D0FFA542F8D16A
:10FF7000BDE87040024802F0C9BF00BFC4E10208FA
:10FF8000FEDE020870B5536E012B0E46154602D0F8
:10FF90000224204670BD19491068F6F7F1F80446AE
:10FFA00038B9F9F757FA31460246154802F0AEFF64
:10FFB000EFE76C6E012CEBD12868F6F7EBF801281F
:10FFC000E6D1FCF76BFA20B10E4802F09FFF032444
:10FFD000DFE728680378303B022BD9D819F0E7FF18
:10FFE000C0B2F9F73CFA05460028D2D1064802F023
:10FFF0008DFF2C4603F082F9CBE700BF2DFF0208EE
:020000040801F1
:100000002CFD020884FE020873DC020873B50E465C
:100010001546FCF73DFA012833D06B6E012B01D059
:1000200002240CE018492868F6F7AAF8044648B9F3
:10003000FCF740FA31460246144802F067FF2046BA
:1000400002B070BD6B6E012BEAD1286801A9FDF7E3
:1000500087FD0028E4D1019A0D4B13440D4A9342C9
:10006000DED8FCF71BFA20B10B4802F04FFF032447
:10007000E5E70198FCF79AFB40B2FDF7CBFD04469B
:10008000DDE70824DBE700BF2DFF02082CFD020896
:10009000802E0FF7809E473084FE020873B50E460F
:1000A0001546FCF7F5F9012831D06B6E012B01D014
:1000B00002240CE017492868F6F762F8044648B9AC
:1000C000FCF708FA31460246134802F01FFF2046AB
:1000D00002B070BD6B6E012BEAD1286801A9FDF753
:1000E0003FFD0028E4D1019B053B072BE0D8FCF73E
:1000F000D5F920B1094802F009FF0324E7E79DF88C
:100100000400FCF767FB041E18BF0124DFE7082486
:10011000DDE700BF2DFF02082CFD020884FE020867
:1001200073B50E461546FCF7B3F901282DD06B6E5A
:10013000012B01D002240CE015492868F6F720F8BD
:10014000044648B9FCF7CFF931460246114802F09F
:10015000DDFE204602B070BD6B6E012BEAD128682F
:1001600001A9FDF7FDFC0028E4D1FCF797F920B1C7
:10017000094802F0CBFE0324EBE70198FCF738FBBB
:1001800040B2FDF747FD0446E3E70824E1E700BF7E
:100190002DFF02082CFD020884FE020873B50E46EE
:1001A0001546FCF775F901282ED06B6E012B01D096
:1001B00002240CE015492868F5F7E2FF044648B927
:1001C000FCF764FB31460246114802F09FFE2046D0
:1001D00002B070BD6B6E012BEAD1286801A9FDF752
:1001E000BFFC0028E4D1FCF759F920B1094802F01E
:1001F0008DFE0324EBE79DF80400FCF749FB40B2B9
:10020000FDF708FD0446E2E70824E0E72DFF0208B9
:100210002CFD020884FE020873B50E461546FCF755
:1002200037F9012833D06B6E012B01D002240CE08A
:1002300018492868F5F7A4FF044648B9FCF73AFBCB
:1002400031460246144802F061FE204602B070BDFD
:100250006B6E012BEAD1286801A9FDF781FC00280B
:10026000E4D1019B4FF6FA72053B9342DED8FCF7CE
:1002700015F920B1094802F049FE0324E5E7BDF86D
:100280000400FCF719FB041E18BF0124DDE7082455
:10029000DBE700BF2DFF02082CFD020884FE0208E8
:1002A00073B50E461546FCF7F3F8012831D06B6E96
:1002B000012B01D002240CE017492868F5F760FFF4
:1002C000044648B9FCF70AFB31460246134802F0DF
:1002D0001DFE204602B070BD6B6E012BEAD128686E
:1002E00001A9FDF73DFC0028E4D1019B053B112B42
:1002F000E0D8FCF7D3F820B1094802F007FE032448
:10030000E7E79DF80400FCF7EBFA041E18BF012490
:10031000DFE70824DDE700BF2DFF02082CFD0208FF
:1003200084FE020830B5C1B01446FCF7B1F80128CC
:100330002BD0636E012B02D0022041B030BD144996
:100340002068F5F71DFF0028F6D0636E012BF3D16E
:100350002068F5F71FFFC2070546EDD4B0F5007F12
:10036000EAD801466A462068FDF7BAFB0028E3D1C7
:10037000FCF7D6FAC5F3470102466846FCF718FBBE
:10038000831D0CBF03200020D7E70820D5E700BF5E
:100390002DFF020837B51546FCF77AF8012829D059
:1003A0006B6E012B01D002240BE013492868F5F78E
:1003B000E7FE044650B9FCF771F828B10F4802F087
:1003C000A5FD204603B030BD0D48F8E76B6E012B4C
:1003D000E9D1286801A9FDF7C3FB0028E3D1019802
:1003E000B0F5803FDFD2FCF78FF940B2FDF712FC89
:1003F0000446E6E70824E4E72DFF0208BFFE0208F2
:10040000CBFE020873B50E461546FCF741F80128ED
:1004100032D06B6E012B01D002240CE01749286802
:10042000F5F7AEFE044648B9FCF76EFA31460246CF
:10043000134802F06BFD204602B070BD6B6E012BBD
:10044000EAD1286801A9FDF78BFB0028E4D1019BC4
:10045000012BE1D8FCF722F820B10A4802F056FD42
:100460000324E8E70198003818BF0120FCF74EFA92
:10047000041E18BF0124DEE70824DCE72DFF020874
:100480002CFD020884FE020873B50E461546FBF7E4
:10049000FFFF012828D06B6E012B01D002240CE055
:1004A00012492868F5F76CFE044648B9FCF738FA9B
:1004B000314602460E4802F029FD204602B070BDCA
:1004C0006B6E012BEAD1286801A9FDF749FB0028D2
:1004D000E4D101980128E1D800F00100FCF727FAE7
:1004E000041E18BF0124E8E70824E6E72DFF0208F0
:1004F0002CFD020870B586B00E461546FBF7C8FF06
:1005000001283ED06C6E012C01D0022417E01E4958
:100510002868F5F735FE0146A0B9112201A819F0A7
:10052000D5FD102101A8FCF7F3F9054638B931468D
:10053000164802F0EBFC01A8FFF70EFD2C46204602
:1005400006B070BD6B6E012BDFD12868F5F722FE77
:1005500020280146D9D1286801AAFDF7C1FA002850
:10056000D3D1FBF79BFF20B1094802F0CFFC032455
:10057000E5E7102101A8FCF7CDF9041E18BF0124FE
:10058000DDE70824DBE700BF2DFF020828FD020895
:1005900084FE020870B586B00E461546FBF778FF5C
:1005A00001283ED06C6E012C01D0022417E01E49B8
:1005B0002868F5F7E5FD0146A0B9112201A819F058
:1005C00085FD102101A8FCF7A7F9054638B9314689
:1005D000164802F09BFC01A8FFF7BEFC2C46204603
:1005E00006B070BD6B6E012BDFD12868F5F7D2FD28
:1005F00020280146D9D1286801AAFDF771FA002800
:10060000D3D1FBF74BFF20B1094802F07FFC032454
:10061000E5E7102101A8FCF781F9041E18BF0124A9
:10062000DDE70824DBE700BF2DFF020828FD0208F4
:1006300084FE02082DE9F04F8FB00F461546FBF7F8
:1006400027FF012800F0F3816B6E012B56D1AB49D7
:100650002868F5F795FD044600284FD102F0AEF961
:1006600030B308A802F0B6F93946A54802F04EFCAE
:100670000899A44802F04AFC9DF82410A14802F011
:1006800045FC0A999F4802F041FC9DF830109D48B6
:1006900002F03CFCBDF832109A4802F037FC9DF89D
:1006A0003410994802F032FC20460FB0BDE8F08FBC
:1006B0003946934802F02AFCFBF7FCFE01469148BC
:1006C00002F024FCFBF706FF01468E4802F01EFCF8
:1006D000FBF709FF01468B4802F018FCFCF7D6F83F
:1006E0000146884802F012FCFCF7E4F80146854810
:1006F00002F00CFCFCF7F2F80146D2E76B6E062B19
:1007000053D1FBF7D7FE8346FBF7E4FE8246FBF7A7
:10071000EAFE8146FCF7BAF88046FCF7CBF80746BC
:10072000FCF7DCF803A906462868FDF719FA00284B
:100730003DD1686804A9FDF713FA002837D1A868ED
:1007400005A9FDF70DFA002831D1E86806A9FDF7E3
:1007500007FA60BB286907A9FDF702FA38BB686988
:1007600008A9FDF7FDF910BB039A684B1344684ACA
:1007700093421CD8049B053B072B18D8069B032BE0
:1007800015D8079B4FF6FA72053B93420FD8089B8A
:10079000053B112B0BD8FBF781FE002800F0C08031
:1007A0005C4802F0B3FB03247EE7072B01D0022450
:1007B0007AE75949A869F5F7E3FC0028A1D06B6EE8
:1007C000072BF4D15549A869F5F7DAFC044600284F
:1007D000EDD102F0F3F80190002800F0EA8008A8BB
:1007E00002F0F8F8DDF820B09DF824A0FBF750FEE9
:1007F000002840F0D8800A9E9DF83090BDF83280E5
:100800009DF83470286802A9FDF7AAF90028CED116
:10081000686803A9FDF7A4F90028C8D1A86804A94D
:10082000FDF79EF90028C2D1E86805A9FDF798F9FF
:100830000028BCD1286906A9FDF792F90028B6D195
:10084000686907A9FDF78CF90028B0D1FBF726FEEF
:100850000028A5D1FBF71CFE20B9049B7D2B40F09E
:10086000BB8004900298FBF727FE10F0FF0540F0D4
:10087000C5809DF80C00FBF72FFE10F0FF0540F03F
:10088000BD800498FBF7E2FF10F0FF0540F0B68052
:100890009DF81400FCF708F810F0FF0540F0AE805A
:1008A000BDF81800FCF714F810F0FF0540F0A68022
:1008B0009DF81C00FCF721F810F0FF0540F09E8029
:1008C000029B0893039B8DF82430FBF7E1FD002881
:1008D00040F08D80049B0A93059B8DF83030069B79
:1008E000ADF8323008A8079B8DF8343002F07CF860
:1008F000012002F069F8FBF707FED5E62DFF02089C
:1009000028FD020848FD020846DB0208802E0FF78A
:10091000809E473084FE020823FF02082AFE020858
:100920000398FBF743FF10F0FF0425D19DF810005A
:10093000FBF750FF10F0FF041ED10598FBF758FF9E
:1009400010F0FF0418D19DF81800FBF7A1FF10F07C
:10095000FF0411D1BDF81C00FBF7AEFF10F0FF043F
:100960000AD19DF82000FBF7BBFF10F0FF0403D174
:10097000204602F029F897E65846FBF717FF504645
:10098000FBF728FF4846FBF733FF4046FBF780FFA5
:100990003846FBF791FF3046FBF7A2FF60B2FDF748
:1009A00039F9044680E6FBF773FD022808BF0B9E69
:1009B00022E7FBF77FFD8346FBF78CFD8246FBF7C2
:1009C00092FD0646FBF762FF8146FBF773FF804608
:1009D000FBF784FF074615E7FA2B02D101230493A6
:1009E00040E7B3F5FA7F7FF43DAF0223F7E7FBF76B
:1009F0004FFD022804BF049B0B936DE7019BA3B935
:100A00005846FBF7D3FE5FFA8AF0FBF7E3FE304669
:100A1000FBF7EEFE5FFA89F0FBF73AFF1FFA88F06A
:100A2000FBF74AFFF8B2FBF75BFF68B2B7E70824B1
:100A30003AE600BFF7B50F461546FBF729FD022839
:100A400032D16B6E012B03D00224204603B0F0BDDF
:100A500016492868F5F794FB044638B9FCF7DAFA2A
:100A600039460246124802F051FAEEE76B6E012B4E
:100A7000EAD1286801A9FDF773F80028E4D1019BA9
:100A80000C4AA3F516739342DED8FBF707FD20B19D
:100A9000094802F03BFA0324D7E70198FCF7D2FAA1
:100AA000041E18BF0124D0E70824CEE72DFF02085A
:100AB0002CFD02088891040084FE0208F7B50F4659
:100AC0001546FBF7E5FC022832D16B6E012B03D0F3
:100AD0000224204603B0F0BD16492868F5F750FB04
:100AE000044638B9FCF798FA39460246124802F033
:100AF0000DFAEEE76B6E012BEAD1286801A9FDF72C
:100B00002FF80028E4D1019B0C4AA3F516739342F9
:100B1000DED8FBF7C3FC20B1094802F0F7F9032443
:100B2000D7E70198FCF77AFA041E18BF0124D0E732
:100B30000824CEE72DFF02082CFD0208E80A030076
:100B400084FE020873B50E461546FBF7A1FC01288A
:100B500031D06B6E012B01D002240CE017492868BC
:100B6000F5F70EFB044648B9FCF780FA3146024619
:100B7000134802F0CBF9204602B070BD6B6E012B1A
:100B8000EAD1286801A9FCF7EBFF0028E4D1019C19
:100B90000CB1012CE0D1FBF781FC20B1094802F037
:100BA000B5F90324E7E72046FCF762FA40B2FDF707
:100BB00031F80446DFE70824DDE700BF2DFF020817
:100BC0002CFD020884FE020873B50E461546FBF79D
:100BD0005FFC01282FD06B6E012B01D002240CE0AA
:100BE00016492868F5F7CCFA044648B9FCF746FAE6
:100BF00031460246124802F089F9204602B070BD23
:100C00006B6E012BEAD128680DF10601FCF78AFF13
:100C10000028E3D1FBF742FC20B10A4802F076F944
:100C20000324EAE7BDF80600FCF72AFA40B2FCF715
:100C3000F1FF0446E1E70824DFE700BF2DFF0208CB
:100C4000D8FE020884FE020873B50E461546FBF76F
:100C50001FFC01282DD06B6E012B01D002240CE06B
:100C600015492868F5F78CFA044648B9FBF722FCC9
:100C700031460246114802F049F9204602B070BDE3
:100C80006B6E012BEAD1286801A9FCF769FF0028E7
:100C9000E4D1FBF703FC20B1094802F037F9032443
:100CA000EBE70198FBF782FD40B2FCF7B3FF044687
:100CB000E3E70824E1E700BF2DFF02082CFD02084E
:100CC00084FE020873B50E461546FBF7E1FB0128CA
:100CD00032D06B6E012B01D002240CE0174928683A
:100CE000F5F74EFA044648B9FBF7F8FD31460246DF
:100CF000134802F00BF9204602B070BD6B6E012B59
:100D0000EAD1286801A9FCF72BFF0028E4D1019B58
:100D1000053B112BE0D8FBF7C1FB20B1094802F0DD
:100D2000F5F80324E7E79DF80400FBF7D9FD40B28E
:100D3000FCF770FF0446DEE70824DCE72DFF02081D
:100D40002CFD020884FE0208FFF7EAB973B50E46CF
:100D50001546FBF79DFB012832D06B6E012B01D0AD
:100D600002240CE017492868F5F70AFA044648B946
:100D7000FBF7B0FB31460246134802F0C7F82046A5
:100D800002B070BD6B6E012BEAD1286801A9FCF797
:100D9000E7FE0028E4D1019B053B072BE0D8FBF7D9
:100DA0007DFB20B1094802F0B1F80324E7E79DF884
:100DB0000400FBF70FFD40B2FCF72CFF0446DEE712
:100DC0000824DCE72DFF02082CFD020884FE02083F
:100DD00073B50E461546FBF75BFB012831D06B6EF1
:100DE000012B01D002240CE017492868F5F7C8F957
:100DF000044648B9FBF74AFD31460246134802F063
:100E000085F8204602B070BD6B6E012BEAD12868D0
:100E100001A9FCF7A5FE0028E4D1019B032BE1D832
:100E2000FBF73CFB20B10A4802F070F80324E8E726
:100E30009DF80400FBF72CFD40B2FCF7EBFE0446E6
:100E4000DFE70824DDE700BF2DFF02082CFD0208C4
:100E500084FE020873B50E461546FBF719FB012800
:100E600034D06B6E012B01D002240CE018492868A5
:100E7000F5F786F9044648B9FBF71CFD31460246F2
:100E8000144802F043F8204602B070BD6B6E012B8F
:100E9000EAD1286801A9FCF763FE0028E4D1019B90
:100EA0004FF6FA72053B9342DED8FBF7F7FA20B112
:100EB000094802F02BF80324E5E7BDF80400FBF72E
:100EC000FBFC40B2FCF7A6FE0446DCE70824DAE7A8
:100ED0002DFF02082CFD020884FE020873B50E46A1
:100EE0001546FBF7D5FA012831D06B6E012B01D0E6
:100EF00002240CE017492868F5F742F9044648B97E
:100F0000FCF7B8F831460246134801F0FFFF2046CF
:100F100002B070BD6B6E012BEAD1286801A9FCF705
:100F20001FFE0028E4D1019C0CB1012CE0D1FBF79D
:100F3000B5FA20B1094801F0E9FF0324E7E72046AC
:100F4000FCF79AF840B2FCF765FE0446DFE7082498
:100F5000DDE700BF2DFF02082CFD020884FE020819
:100F600010B5546E1CB901F04BFD204610BD022493
:100F7000FBE7506E002818BF0220704730B51446BA
:100F80008BB00D462122002101A819F09FF8636E55
:100F9000012B03D0022420460BB030BD2068084945
:100FA000F5F7EEF804460028F4D10649202201A8FE
:100FB00019F064F801AA2946034801F0A7FFEAE7FF
:100FC0002DFF020800500008B5FD020873B5536EEE
:100FD000012B0E46154603D00124204602B070BDF9
:100FE00011491068F5F7CCF8044650B918F026FA04
:100FF000314602460D4801F089FF0D4801F086FF99
:10100000EBE76B6E012BE7D128680DF10701FCF7C8
:10101000A7FD044630B99DF80700012802D818F052
:101020000BFADAE70224D8E72DFF0208E2FE0208F5
:10103000FEDE020810B5546E1CB902F05FF92046BE
:1010400010BD0224FBE710B5536E73B9F9F746FFE4
:1010500048B900F0EDFB044618B902F04FF92046FC
:1010600010BD063403D00124F9E70224F7E7032476
:10107000F5E710B5546E4CB900F00EFD20B9012013
:1010800000F010FD204610BD2046F9E70224F9E7E4
:1010900070B5566E012E86B00D46144603D002265A
:1010A000304606B070BD2C491068F5F769F8C8B92C
:1010B000122101A800F0C0FC04460028F0D1294606
:1010C0002648274E01F022FF01AD15F8011B3046DE
:1010D000013401F01BFF122CF7D1224801F016FF5A
:1010E0000026DDE7636E012BD9D12068F5F752F8B1
:1010F0000028D4D02068F5F74DF81228CFD8122157
:1011000001A800F099FC05460028C9D101AB0246B0
:1011100013F8011B0029C3D10132122AF8D120682B
:10112000F5F738F8A84226680AD83046F5F732F8BD
:101130000146304600F08EFC061E18BF0126AFE7C0
:10114000735DA3F13002092A04D923F02003413B47
:10115000192BA4D80135E2E72DFF020828FD02086B
:10116000E8FE0208FEDE020870B5556E012D86B05D
:101170000E4603D00225284606B070BD0F49106800
:10118000F4F7FEFF0028F5D1122101A800F054FC6D
:1011900004460028EFD1314609480A4E01F0B6FE58
:1011A00001AD15F8011B3046013401F0AFFE122CE1
:1011B000F7D1054801F0AAFE0025DCE72DFF020863
:1011C00028FD0208E8FE0208FEDE020837B5536E6D
:1011D000012B0D4603D00224204603B030BD0A493E
:1011E0001068F4F7CDFF04460028F4D101A818F0E8
:1011F000B3F80198F5F790F902460B4603482946E3
:1012000001F084FEE8E700BF2DFF0208EBFE0208B4
:1012100037B5536E012B0D4603D00224204603B090
:1012200030BD0A491068F4F7ABFF04460028F4D13A
:1012300001A818F0D3F80198F5F76EF902460B46AD
:101240000348294601F062FEE8E700BF2DFF0208CF
:10125000EBFE020838B5536E012B0D4602D0022476
:10126000204638BD07491068F4F78AFF0446002875
:10127000F5D1054B054A1B6812680548294601F05F
:1012800045FEEDE72DFF0208900D00208C0D00209B
:10129000F3FE020838B5536E012B0D4602D002242E
:1012A000204638BD06491068F4F76AFF0446002856
:1012B000F5D1044B04481A68294601F027FEEFE7F0
:1012C0002DFF0208940D0020B5FD020838B5536EBD
:1012D000012B0D4602D00224204638BD0649106875
:1012E000F4F74EFF04460028F5D1044B04481A6871
:1012F000294601F00BFEEFE72DFF0208800D0020CC
:10130000B5FD020830B5536E012B8BB00D4603D0EE
:10131000022420460BB030BD09491068F4F730FFB5
:1013200004460028F4D18DF82400202101A800F003
:10133000F9FA01AA2946034801F0E8FDE9E700BFF0
:101340002DFF0208B5FD020830B5536E012B8BB09E
:101350000D4603D0022420460BB030BD0949106869
:10136000F4F70EFF04460028F4D18DF82400202164
:1013700001A800F0F3FA01AA2946034801F0C6FDCE
:10138000E9E700BF2DFF0208B5FD020838B5536E2E
:10139000012B0D4602D00224204638BD06491068B4
:1013A000F4F7EEFE04460028F5D1044B04481A6811
:1013B000294601F0ABFDEFE72DFF02089C0D002050
:1013C000B5FD020830B5536E012B8BB00D4603D02E
:1013D000022420460BB030BD09491068F4F7D0FE56
:1013E00004460028F4D18DF82400202101A800F043
:1013F000A7FA01AA2946034801F088FDE9E700BFE2
:101400002DFF0208B5FD020838B5536E012B0D46BD
:1014100002D00224204638BD06491068F4F7B0FE19
:1014200004460028F5D1044B04481A68294601F007
:101430006DFDEFE72DFF0208880D0020B5FD0208C5
:101440007FB5556E012D0E46144603D00225284661
:1014500004B070BD24491068F4F792FEC8B9102199
:10146000684600F0B1FA04460028F0D131461F4822
:101470001F4E01F04BFD6D4615F8011B304601343F
:1014800001F044FD102CF7D11A4801F03FFD002572
:10149000DDE7636E012BD9D12068F4F77BFE0028CD
:1014A000D4D02068F4F776FE1028CFD810216846F3
:1014B00000F08AFA06460028C9D12068F4F76AFECF
:1014C000B04225680AD82846F4F764FE014628464B
:1014D00000F088FA051E18BF0125B8E7AB5D203B78
:1014E0005E2BB3D80136E8E72DFF020828FD02087D
:1014F000E8FE0208FEDE020838B5556E144625B92E
:10150000284601F049FC284638BD012D20D002258F
:10151000F9E72368585D18F081FD0028F7D0013500
:101520002068F4F737FEA842F3D820680A22002189
:1015300019F0C4FC431C05460CD108492068F4F797
:101540001FFE0028E3D1284601F026FC0025DAE73B
:101550000025E5E70028DAD0F5E700BFFEFE020827
:1015600070B5536E012B0E46154602D0022420465C
:1015700070BD16491068F4F703FE044638B900F050
:10158000A9F931460246124801F0C0FCEFE76B6E44
:10159000012BEBD1002406E02B68185D18F03EFD0E
:1015A0000028E3D001342868F4F7F4FDA042F3D812
:1015B00028680A22002119F081FC0128D6D800F001
:1015C0008FF9041E18BF0124D1E700BF2DFF0208C8
:1015D0002CFD020870B5536E012B0E46154602D045
:1015E0000224204670BD16491068F4F7C9FD044670
:1015F00038B900F081F931460246124801F086FC04
:10160000EFE76B6E012BEBD1002406E02B68185D31
:1016100018F004FD0028E3D001342868F4F7BAFD7F
:10162000A042F3D828680A22002119F047FC431E83
:10163000012BD5D800F066F9041E18BF0124D0E7AD
:101640002DFF02082CFD020838B5536E012B1546FC
:101650000AD109491068F4F793FD044620B90748F8
:1016600001F054FC204638BD6C6E14B901F0C2FC88
:10167000F8E70224F6E700BF2DFF020809FF020881
:10168000F0B5546E012C85B00F46154603D00224E8
:10169000204605B0F0BD20491068F4F771FD0646FC
:1016A000E8B9092101A801F067FD051EF0DD1B481E
:1016B000394601F02BFC3446194EE3B2AB4204F13B
:1016C000010404DB174801F021FC0024E0E704AA30
:1016D0001344304613F80C1C01F018FCEDE76E6E55
:1016E000012ED4D12868F4F755FD0028CFD0286802
:1016F000F4F750FD0828CAD82C682046F4F74AFDB4
:101700000146204601F03FFD04460028C0D00334C6
:10171000BDD03446BCE700BF2DFF020828FD0208FB
:10172000E8FE0208FEDE0208F7B5536E012B0646FE
:101730000F46154603D00224204603B0F0BD1B49D6
:101740001068F4F71DFD044638B900F02BF939464E
:101750000246174801F0DAFBEEE76B6E012BEAD187
:10176000002406E02B68185D18F058FC0028E2D031
:1017700001342868F4F70EFDA042F3D828680A2245
:10178000002119F09BFBB0F5E13F0446D3D80023BC
:101790000146CDE900330322304601F033FB2046F9
:1017A00000F006F9041E18BF0124C5E72DFF02084A
:1017B0002CFD020838B5546E05468CB900F042F88D
:1017C000C0B258B1084801F0A1FB2146284600F0FC
:1017D00041F8044630B92846FBF794FE204638BD50
:1017E0000224FBE70124F9E73FFF0208B0B5546E7D
:1017F00000AFBCB96D46ADF5006D6A464FF40061AF
:10180000094801F0FFF84FF40061084801F026FA9A
:101810006A4606484FF4006101F09EF9AD46204645
:10182000BD46B0BD0224FAE700F0030800700308CB
:10183000024A03484FF4257101F08EB9A83E0020FA
:1018400000F00308024B034493F8BC01704700BF4B
:10185000A83E0020044A104480F8BC1103484FF40D
:10186000257101F079B900BFA83E002000F00308FF
:10187000082908B508D90649092218F0FFFBBDE878
:1018800008400348F4F786BC6FF0080008BD00BFAD
:1018900071400020082938B505460C4611D80922A8
:1018A0000021094818F012FC22462946064818F083
:1018B000E5FBBDE83840054A05484FF4257101F0C5
:1018C0004BB96FF0020038BD71400020A83E0020E7
:1018D00000F00308014BD3F8D4017047A83E002064
:1018E000034A4FF42571C2F8D401024801F034B91B
:1018F000A83E002000F00308014B93F870027047E7
:10190000A83E0020054A08B54FF4257182F8700200
:10191000034801F021F9C0B208BD00BFA83E002075
:1019200000F003081F2908B505D90449202218F042
:10193000A5FB002008BDF720FCE700BFA340002066
:101940001F2908B505D90449202218F097FB00206B
:1019500008BDF720FCE700BFC34000201F2908B5E1
:1019600005D90449202218F089FB002008BDF72082
:10197000FCE700BFE3400020024B034493F8BF01A3
:10198000704700BFA83E0020044A104480F8BF11F1
:1019900003484FF4257101F0DFB800BFA83E0020D6
:1019A00000F00308014BD3F8C4017047A83E0020A3
:1019B000034A4FF42571C2F8C401024801F0CCB8C3
:1019C000A83E002000F003080F2908B505D90449F6
:1019D000102218F053FB002008BD6FF00800FBE751
:1019E00092400020102938B504460D461BD804D07B
:1019F0000E481022002118F069FB234629198B425A
:101A00000CD12A462146094818F038FBBDE8384079
:101A1000074A08484FF4257101F09EB813F8012BCE
:101A2000203A5E2AEBD96FF0020038BD92400020C8
:101A3000A83E002000F00308112908B505D9044983
:101A4000122218F01BFB002008BD6FF00800FBE716
:101A500080400020122938B505460C4612D804D023
:101A60000A481222002118F031FB22462946074875
:101A700018F004FBBDE83840054A06484FF42571CC
:101A800001F06AB86FF0020038BD00BF804000204E
:101A9000A83E002000F00308014B93F8C8017047EE
:101AA000A83E0020034A4FF4257182F8C80102487D
:101AB00001F052B8A83E002000F00308034A4FF49A
:101AC000257182F8FA01024801F046B8A83E0020CC
:101AD00000F00308014B93F8FA017047A83E00207C
:101AE000014B93F830007047A83E0020034A4FF4A2
:101AF000257182F83000024801F02EB8A83E00207F
:101B000000F0030808B503490C2218F0B7FA0020CA
:101B100008BD00BF4A3F002010B5074C01460C220B
:101B200004F1A20018F0AAFA22460448BDE81040C9
:101B30004FF4257101F010B8A83E002000F0030812
:101B4000072908B505D90449082218F097FA00209A
:101B500008BD6FF00800FBE7E13E0020082908B54A
:101B60000A460BD10146074818F088FABDE808403C
:101B7000054A06484FF4257100F0EEBF6FF00200F1
:101B800008BD00BFE13E0020A83E002000F0030891
:101B90000F2908B505D90449102218F06FFA002062
:101BA00008BD6FF00800FBE7E93E0020102908B5EA
:101BB0000A460BD10146074818F060FABDE8084014
:101BC000054A06484FF4257100F0C6BF6FF00200C9
:101BD00008BD00BFE93E0020A83E002000F0030839
:101BE0000F2908B505D90449102218F047FA00203A
:101BF00008BD6FF00800FBE7F93E0020102908B58A
:101C00000A460BD10146074818F038FABDE80840EB
:101C1000054A06484FF4257100F09EBF6FF00200A0
:101C200008BD00BFF93E0020A83E002000F00308D8
:101C3000032908B505D90449042218F01FFA002029
:101C400008BD6FF00800FBE7093F0020042908B534
:101C50000A460BD10146074818F010FABDE80840C3
:101C6000054A06484FF4257100F076BF6FF0020078
:101C700008BD00BF093F0020A83E002000F0030877
:101C8000072908B505D90449082218F0F7F90020FA
:101C900008BD6FF00800FBE7D93E0020082908B511
:101CA0000A460BD10146074818F0E8F9BDE808409C
:101CB000054A06484FF4257100F04EBF6FF0020050
:101CC00008BD00BFD93E0020A83E002000F0030858
:101CD000032908B505D90449042218F0CFF90020DA
:101CE00008BD6FF00800FBE70D3F00200F2908B585
:101CF00005D90449102218F0C1F9002008BD6FF081
:101D00000800FBE7113F0020102908B50A460BD157
:101D10000146074818F0B2F9BDE80840054A0648F0
:101D20004FF4257100F018BF6FF0020008BD00BF2E
:101D3000113F0020A83E002000F00308014B93F85B
:101D4000B1007047A83E0020034A4FF4257182F885
:101D5000B100024800F000BFA83E002000F00308D8
:101D6000014B93F8B0007047A83E0020034A4FF49F
:101D7000257182F8B000024800F0EEBEA83E0020B7
:101D800000F00308014B187A704700BFA83E0020FE
:101D9000034A4FF425711072024800F0DDBE00BF07
:101DA000A83E002000F00308014B93F8AE007047F6
:101DB000A83E0020034A4FF4257182F8AE00024885
:101DC00000F0CABEA83E002000F00308014B93F8C3
:101DD000B4007047A83E0020034A4FF4257182F8F2
:101DE000B400024800F0B8BEA83E002000F003088E
:101DF000014B93F8AF007047A83E0020034A4FF410
:101E0000257182F8AF00024800F0A6BEA83E00206F
:101E100000F00308014B93F8B2007047A83E002081
:101E2000034A4FF4257182F8B200024800F094BED4
:101E3000A83E002000F00308014B93F8B300704760
:101E4000A83E0020034A4FF4257182F8B3000248EF
:101E500000F082BEA83E002000F00308014BD3F83A
:101E6000B8007047A83E0020034A4FF42571C2F81D
:101E7000B800024800F070BEA83E002000F0030841
:101E8000014BD3F8BC007047A83E0020034A4FF432
:101E90002571C2F8BC00024800F05EBEA83E0020DA
:101EA00000F00308034A4FF42571C2F8C800024845
:101EB00000F052BEA83E002000F00308014BD3F80A
:101EC000C8007047A83E0020014B93F8CC00704733
:101ED000A83E0020034A4FF4257182F8CC00024846
:101EE00000F03ABEA83E002000F00308014BD3F8F2
:101EF000C0007047A83E0020034A4FF42571C2F885
:101F0000C000024800F028BEA83E002000F00308F0
:101F1000014BD3F8C4007047A83E0020034A4FF499
:101F20002571C2F8C400024800F016BEA83E002089
:101F300000F00308014B93F8B5007047A83E00205D
:101F4000034A4FF4257182F8B500024800F004BE40
:101F5000A83E002000F00308014B93F8CD00704725
:101F6000A83E0020034A4FF4257182F8CD000248B4
:101F700000F0F2BDA83E002000F00308014B93F8EA
:101F8000CE007047A83E0020034A4FF4257182F826
:101F9000CE00024800F0E0BDA83E002000F003089B
:101FA000014B93F8CF007047A83E0020034A4FF43E
:101FB000257182F8CF00024800F0CEBDA83E002077
:101FC00000F00308014B93F8D0007047A83E0020B2
:101FD000034A4FF4257182F8D000024800F0BCBDDE
:101FE000A83E002000F00308014BD3F8D40070474E
:101FF000A83E0020034A4FF42571C2F8D4000248DD
:1020000000F0AABDA83E002000F00308014BD3F861
:10201000D8007047A83E0020034A4FF42571C2F84B
:10202000D800024800F098BDA83E002000F0030848
:10203000014B93F868027047A83E0020034A4FF412
:10204000257182F86802024800F086BDA83E002093
:1020500000F00308014BB3F96A027047A83E002064
:10206000034A4FF42571A2F86A02024800F074BDD9
:10207000A83E002000F00308014BD3F86C02704723
:10208000A83E0020034A4FF42571C2F86C020248B2
:1020900000F062BDA83E002000F003080048704731
:1020A000843F002010B5074C0146D02204F1DC002B
:1020B00017F0E4FF22460448BDE810404FF42571B4
:1020C00000F04ABDA83E002000F00308014BD3F801
:1020D000AC017047A83E0020034A4FF42571C2F8B6
:1020E000AC01024800F038BDA83E002000F0030813
:1020F000014BD868704700BFA83E0020034A4FF448
:102100002571D060024800F027BD00BFA83E002026
:1021100000F00308014B187C704700BFA83E002068
:10212000034A4FF425711074024800F015BD00BF3A
:10213000A83E002000F00308034B1A7A0AB9588A17
:102140007047D86A704700BFA83E0020064B1A7A35
:1021500032B95882044A05484FF4257100F0FCBC9E
:10216000022A08BFD862F5E7A83E002000F0030865
:10217000014B187D704700BFA83E0020034A4FF472
:1021800025711075024800F0E7BC00BFA83E002092
:1021900000F00308014BD88A704700BFA83E00201A
:1021A000034A4FF42571D082024800F0D5BC00BF2D
:1021B000A83E002000F00308014B187E704700BFC6
:1021C000A83E0020034A4FF425711076024800F023
:1021D000C3BC00BFA83E002000F00308014B987E5E
:1021E000704700BFA83E0020034A4FF42571907647
:1021F000024800F0B1BC00BFA83E002000F0030878
:102200000F2908B505D90449102217F037FF00201F
:1022100008BD6FF00800FBE719410020102908B540
:102220000A460BD10146074817F028FFBDE80840D1
:10223000054A06484FF4257100F08EBC6FF002008D
:1022400008BD00BF19410020A83E002000F003088F
:102250000F2908B505D90449102217F00FFF0020F7
:1022600008BD6FF00800FBE729410020102908B5E0
:102270000A460BD10146074817F000FFBDE80840A9
:10228000054A06484FF4257100F066BC6FF0020065
:1022900008BD00BF29410020A83E002000F003082F
:1022A000034A4FF425719062024800F055BC00BF0C
:1022B000A83E002000F00308034A4FF42571506245
:1022C000024800F049BC00BFA83E002000F003080F
:1022D000014B586A704700BFA83E0020014B986A26
:1022E000704700BFA83E0020034A4FF4257182F8D2
:1022F000B600024800F030BCA83E002000F0030801
:10230000014B93F8B6007047A83E0020014B93F8AC
:102310005C027047A83E0020034A4FF4257182F802
:102320005C02024800F018BCA83E002000F0030840
:10233000014BD3F860027047A83E0020014B93F890
:1023400067027047A83E0020034A4FF4257182F8C7
:102350006702024800F000BCA83E002000F003081D
:10236000014BB3F864027047A83E0020034A4FF4C3
:102370002571A2F86402024800F0EEBBA83E0020DE
:1023800000F00308014B93F891027047A83E00202B
:10239000034A4FF4257182F89102024800F0DCBB39
:1023A000A83E002000F00308F8B5002500F2FB1657
:1023B00004462022294680F8FA51304617F086FE5E
:1023C000274B1F683846F3F7E5FE3946024630468C
:1023D00004F21B2617F052FE20222946304617F041
:1023E00075FE204B1F683846F3F7D4FE3946024687
:1023F000304604F23B2617F041FE202229463046A3
:1024000017F064FE184B1F683846F3F7C3FE3946D1
:102410000246304617F032FE41F22443C4F86432DB
:102420004FF6B073A4F86A320523C4F86C32012366
:1024300084F870321022294684F85C52C4F8605245
:1024400084F8685204F2712017F040FE10222946E9
:1024500004F2812017F03AFE84F89152F8BD00BFD3
:10246000800D0020840D0020980D0020F0B50C4652
:10247000ADF5497D6A464FF4487100F0C3FAB44E99
:1024800023687E9AB348009FB34208BF6568B24B89
:1024900018BF00254FF4FA719A4208BF032500F0D7
:1024A00093FF4FF4F871874208BF0225A948009FA7
:1024B00000F08AFF4FF42572874208BF01250021F2
:1024C000204617F003FE002D52D0012D53D12A468D
:1024D00001A904F1080017F0D1FD242202A904F19A
:1024E0000C0017F0CBFD4FF4C2720BA904F13000C1
:1024F00017F0C4FD08226CA904F5DA7017F0BEFDD0
:1025000003226EA904F5DE7017F0B8FD04226FA94E
:1025100004F5E27017F0B2FD2A4670A904F5E470E4
:1025200017F0ACFD09220DF2C11104F2C91017F029
:10253000A5FD042273A904F5EA7017F09FFD12228D
:1025400074A904F5EC7017F099FD10220DF5F171E6
:1025500004F5F57017F092FD0322002104F2BF107C
:1025600017F0B4FD2046FFF71FFF042326606360C9
:102570000DF5497DF0BDAB1E012B4CD801A9012200
:1025800004F1080017F07AFD02A9242204F10C00DE
:1025900017F074FD0BA94FF4C27204F1300017F06C
:1025A0006DFD6CA9082204F5DA7017F067FD6EA9BD
:1025B000032204F5DE7017F061FD0DF2BB1103225A
:1025C00004F2BF1017F05AFD70A9042204F5E2705E
:1025D00017F054FD71A9012204F5E47017F04EFDC7
:1025E0000DF2C511092204F2C91017F047FD74A9B4
:1025F000042204F5EA7017F041FD75A9122204F5D2
:10260000EC7017F03BFD10220DF5F37104F5F57039
:1026100017F034FDA6E7042DAAD14FF425726946C0
:10262000204617F02BFD94F8FA31FF2B04BF00234E
:1026300084F8FA3194F8FB31FF2B10D104F2FB152A
:1026400020220021284617F041FD444B1F683846E0
:10265000F3F7A0FD39460246284617F00FFD94F81F
:102660001B32FF2B10D104F21B252022002128460B
:1026700017F02CFD3A4B1F683846F3F78BFD3946AF
:102680000246284617F0FAFC94F83B32FF2B10D193
:1026900004F23B2520220021284617F017FD314B7C
:1026A0001F683846F3F776FD39460246284617F08C
:1026B000E5FC94F87032FF2B04BF012384F87032DC
:1026C00094F85C32FF2B04BF002384F85C32D4F80A
:1026D000603213B10023C4F8603294F86632FF2BE5
:1026E00001BF41F22443A4F86432002384F8663227
:1026F00094F86732FF2B04BF002384F8673294F804
:102700006832FF2B04BF002384F8683294F86A32E1
:10271000FF2B04BF4FF6B073A4F86A3294F86C3202
:10272000FF2B04BF0523C4F86C3294F88132FF2BD1
:1027300005D11022002104F2812017F0C7FC94F883
:102740009132FF2B04BF002384F891320DE700BFC4
:10275000DDCCBBAAAC3E00201EDD0E00800D0020AB
:10276000840D0020980D0020F0B57B4A7B4E106848
:102770005168ADF5297D01AB03C379481A464FF482
:10278000257100F03FF9039BB34202D1049B042B57
:102790001CD0734803A9FFF769FE039BB34217D10E
:1027A000049D2C1F654265416E4C4FF4257200213B
:1027B000204617F08BFC6DB14FF4257203A920461B
:1027C00017F05CFC00200DF5297DF0BD0125EBE73D
:1027D0000025E9E70423636040F20113A4F8BC314B
:1027E00008224FF4E13301A984F8BE5104F2C91064
:1027F0002660C4F8C43141F2883717F03FFC41F23B
:102800007071C4E92E714FF47A704FF4FA610123AC
:10281000C4E9300105224FF6B071082684F8302053
:10282000A4F8AE30A4F8B430A4F86A12C4F86C224C
:102830002946D022A4F8B05004F1DC00C4E9356583
:10284000237284F8B63084F8CC3084F87032C4F83F
:10285000D45184F8C85184F8FA5184F8B25084F8FD
:10286000CF5084F8D05084F8685217F02FFC3E4BBC
:10287000E360072323740E23237641F23333C4E944
:10288000093744F620633246E362294641F2244385
:1028900004F11B00A4F86432E6826582334E25758C
:1028A000A57684F85C52C4F8605284F8675217F039
:1028B0000DFC1022294604F2712017F007FC1022AB
:1028C000294604F2812017F001FC306884F8915207
:1028D000F3F760FC1F284FF0200237D8294604F296
:1028E000FB1017F0F3FB35682846F3F753FC294635
:1028F000024604F2FB101E4C17F0C0FB2068F3F7F1
:1029000049FC1F284FF0200222D80021194817F057
:10291000DDFB24682046F3F73DFC21460246164CB9
:10292000144817F0ABFB2068F3F734FC1F284FF076
:1029300020020FD80021114817F0C8FB2468204658
:10294000F3F728FC214602460C4839E73168D0E706
:102950002168E4E72168F7E71CFF0208DDCCBBAA89
:1029600000700308A83E002000A1BC33800D0020A9
:10297000840D0020C3400020980D0020E34000207B
:1029800010B50B4C0B4822464FF4257100F03AF875
:1029900008482146FFF76AFD2268074B9A4202D198
:1029A0006368042B03D0BDE81040FFF7DDBE10BD07
:1029B000A83E002000F00308DDCCBBAA014B18782C
:1029C000704700BF54410020014B1870704700BF92
:1029D0005441002008B50349182217F04FFB01208D
:1029E00008BD00BF3C41002008B50146182202483E
:1029F00017F044FB012008BD3C41002015F0BCBE8F
:102A000015F012BF2DE9F04F87B083460E461546EC
:102A100015F006FFB0F5805F044659D8BBFBF0F80F
:102A200000FB08F8ABEB080301933344B3FBF0F26F
:102A300000FB123109B102FB0003A4EB0B02DFF82B
:102A400098A00492019AB3FBF4F3C146039337466E
:102A5000002302EB0A0B039A9A4203D1002007B02D
:102A6000BDE8F08F22461C490293484615F0A8FEA7
:102A7000029B5A1C0292CBB9049B03EB0802B242A0
:102A80000CD228465946059217F0F8FA019B059A90
:102A90001B1B15441F44029BA144DCE72846324619
:102AA000594617F0EBFA3544BF1BF4E7DDE9023273
:102AB000934205D33A465146284617F0DFFAEAE733
:102AC00028462246514617F0D9FA25443F1BE2E733
:102AD0006FF00800C3E700BF584100202DE9F84F10
:102AE00000AF81460C46924615F09AFEADF5806D1A
:102AF0006E464FEA90284FF0000B5FFA8BF1884545
:102B000001D8012021E0B4F5806F09EB81200AEBA8
:102B1000812532460ED34FF48061FFF773FF4FF4E7
:102B200080622946304617F099FA0BF1010B78B113
:102B300000200AE02146FFF765FF2246294630467D
:102B400017F08CFAB0FA80F04009BD46BDE8F88F66
:102B5000A4F58064D1E700002DE9F04F87B08346EB
:102B60000D46144615F05CFEB0F5805F074670D840
:102B7000224629465846FFF7B1FF18B1002007B09A
:102B8000BDE8F08FBBFBF7F807FB08F8ABEB0803D9
:102B90005A19B2FBF7F107FB1120029308B101FBB0
:102BA0000772B2FBF7F3039300230193A7EB0B0328
:102BB000DFF8A4A00493029BC1462E4603EB0A0B48
:102BC000039B019A9342D9D023493A46484615F0CF
:102BD000F7FD019BF3B9049B03EB0802AA4211D253
:102BE00021465846059217F049FA059A029B14446B
:102BF000DA1B16443946484615F0EAFDE8B16FF095
:102C00000600BCE721462A46584617F037FA2C44FE
:102C1000761BEFE7019B5A1C039B9A4205D3324671
:102C20002146504617F02AFAE4E721463A46504634
:102C300017F024FA3C44F61BDCE748463A46514676
:102C400015F09CFDB9440028D9D1019B01330193B3
:102C5000B6E76FF0080092E75841002038B5054606
:102C60000C4615F0DDFDAB070AD1B4FBF0F300FB19
:102C7000134040B921462846BDE8384015F0A8BDAC
:102C80006FF0090038BD6FF00A00FBE7F6F72EB8C9
:102C9000F6F768B8F5F762BF2DE9F0412D4D022037
:102CA00000F0AAF8D5E90032C01A2B4B1B6861EB83
:102CB0000201984271F1000303D26FF00500BDE8F4
:102CC000F08116F01DF98028F7D1FEF715FE234E8E
:102CD0000746002456F8043B03B198470134102CF2
:102CE000F8D11F4EDFF87C8000F0F4FA16F0B3FB49
:102CF00000F07EF800F08EFA00F018FBFFF7C6FF38
:102D000000F07CF8F368984798F80040F4B9B3688D
:102D1000154E984700F074F8FFF7BAFF00F0DCFAA0
:102D200000F00AFB00F078FA00F064F816F095FB6A
:102D300056F8043B03B198470134102CF8D1022017
:102D400000F05AF8C5E900010020B8E733683846BA
:102D50009847D9E7605100205C0A002068510020A4
:102D60004C0A00205A510020A8510020014B00229B
:102D70001A7070475A510020024A136801331360D9
:102D8000704700BFE8510020024A13680BB1013BB5
:102D900013607047E851002038B5114B1D68044698
:102DA000D5B9F8F7A7F90F4B18700F4B01221A701D
:102DB0004CB129460D4815F091FC15F0B3FC29469D
:102DC000204615F09FFCF8F77FF9FFF765FF0446F2
:102DD000F8F78AF9204638BD6FF00704FAE700BF1C
:102DE000E8510020595100205A5100206D2D010852
:102DF00015F052BF15F0AABFF4F7B0BEF4F7C0BE8D
:102E0000F4F7BFBE2DE9F04702289DF820909DF809
:102E100024A004460D4616461F4615D8DFF82C8020
:102E200058F820300BB15B689847CDE9089A084BF9
:102E300048F82430D3F800E032463B462946204685
:102E4000F446BDE8F0476047BDE8F087EC5100204C
:102E5000680A002002282DE9F04104460D46164676
:102E600010D8FEF789FD88B90B4B53F8243083B195
:102E70009F680A4B324629462046BC461B68BDE87F
:102E8000F04160476FF00200BDE8F0816FF007008D
:102E9000FAE74FF0FF30F7E7EC510020880A0020F6
:102EA0000EB430B50446ADF5027DFEF7CBFC022C26
:102EB0001FD82046FEF760FDF0B9124D55F82430BA
:102EC000EBB186AA8599019202A818F05BF855F833
:102ED000243002A89D68F3F75DF90B4B02461B688E
:102EE00002A92046A8470DF5027DBDE8304003B099
:102EF00070476FF00200F6E76FF00700F3E74FF05E
:102F0000FF30F0E7EC510020880A00200FB42DE9D3
:102F1000F047ADF5027D8AAF002457F8049B174EA9
:102F2000DFF85CA025465FFA84F84046FEF78AFC8D
:102F3000B8B94046FEF720FD98B933688BB13A46E0
:102F4000494602A8019718F01DF8336802A89D6849
:102F5000F3F720F9DAF80030024602A94046A84704
:102F600005460134032C06F10406DCD128460DF594
:102F7000027DBDE8F04704B0704700BFEC5100206F
:102F8000880A0020022810B409D8084C54F82030D0
:102F90004BB1DC68064BA4461B6810BC60476FF061
:102FA000020010BC70474FF0FF30FAE7EC510020F0
:102FB000880A0020022805D8054A52F8203023B19B
:102FC0001B6918476FF0020070474FF0FF307047E1
:102FD000EC510020022807D8044A52F820301BB1D7
:102FE000034A5B6911681847704700BFEC51002025
:102FF000880A00202DE9F8430E4FDFF83C80DFF807
:103000003C900025EEB23046FEF7B6FC044658B9B7
:1030100001213046FEF7B8FC0922214648463C60B3
:10302000C8F8004017F052F80135032DEAD1BDE889
:10303000F88300BF00520020FC5100200452002001
:1030400038B50024E5B22846FEF796FC012803D1E6
:1030500000212846FEF798FC0134032CF2D138BD3C
:103060002DE9F04786B004468DF8071003A8092122
:10307000FEF7FEFB9DF80730364D0D2B074629D095
:1030800019D8082B19D00A2B24D02A68082A0ED860
:10309000511C296030498B54304B53F824309D68C3
:1030A0002F4B01221B680DF107012046A8472D4A2E
:1030B000136801330CE07F2BE7D12B68002B3ED047
:1030C000013B254A2B600021D154264A1368013B5D
:1030D000136034E0234E336853B3DFF88090DFF899
:1030E000808059F824302049D3F808A0D8F800305F
:1030F00002222046D0473268092A0ED11B491648C1
:1031000017F0B2FD48B959F8243019499F68D8F82A
:10311000003015222046B8470AE03368BB4211D17F
:103120000D483A4603A916F099FF58B9FFF788FFF2
:103130000021094829600922316016F0C7FF06B056
:10314000BDE8F08759F824300A499F68D8F8003064
:103150001122DFE70052002004520020EC51002031
:10316000880A0020FC510020FEDE020825FF02082C
:103170002FFF020844FF0208082901D9FEF778BB97
:103180006FF002007047082910B40BD803460C18E2
:10319000A34202D110BCFEF77DBB13F8012B203AED
:1031A0005E2AF5D96FF0020010BC7047022801D8E2
:1031B000FEF7E2BB00207047022810B5044612D883
:1031C000FEF7DAFB012803D000212046FEF7DCFBE6
:1031D000054B064800211960054B1960BDE81040F9
:1031E000092216F073BF10BD0052002004520020C7
:1031F000FC510020022805D8054A52F8203023B19E
:103200009B6918476FF0020070474FF0FF3070471E
:10321000EC510020F4F7C6BEF4F714BFF8B52A4EFF
:103220000546375C0C46FEF70DFB00284AD04F2CB4
:10323000715D3BD020D82B2C2ED014D80A2C2DD049
:103240000D2C14BF07230623204A02EBC102D35CD6
:1032500073550B2B36D1072F2AD100237355BDE8A8
:10326000F840FFF7CDBB422C1ED04D2C18D0412C7E
:1032700014BF07230023E7E76D2C11D008D8612C79
:1032800010D0622C10D0542C14BF07230123DBE78D
:103290006F2C0BD0742CF7E70223D5E70623D3E776
:1032A0000523D1E70023CFE70323CDE70423CBE7B2
:1032B0000A2F07D10648002345607355BDE8F84042
:1032C00000F014B8F8BD00BFF851002055FF020807
:1032D000600A0020F4F76EBCF4F76EBC024A80214D
:1032E000082015F04FBD00BF10520020014A0821F0
:1032F00015F0A2BD5D75000815F06ABD15F0BEBBE6
:1033000015F0CEBB15F0D1BB15F0D4BB704770479C
:10331000014B1B68184700BF8C0A002015F046BB04
:1033200015F06CBB15F08CBB15F0CCBA014B5B698A
:10333000184700BF9C0A0020014B9B69184700BF3B
:103340009C0A0020074B08491A6843F2390001FB28
:10335000020018606FF00043B0FBF3F3C3EBC373DC
:10336000C01A7047B80A00206D4EC641014B186064
:10337000704700BFB80A002038B505460C46FFF775
:10338000E1FF611B013190FBF1F303FB11002844C5
:1033900038BD01380A44914200D1704711F8013B11
:1033A00000F8013FF7E710440A44914200D170470A
:1033B00011F8013B00F8013DF7E70244904200D1CB
:1033C000704700F8011BF9E730B530B10A4D0144F0
:1033D0004FF0FF33814201D1D84330BD10F8012BAB
:1033E0005340082243F30004013A2C4092B284EA8D
:1033F0005303002AF6D1EDE72083B8ED38B5104C21
:10340000237805460BB9012038BD01F0DBFC22789A
:103410004FF47A73B3FBF2F3B0FBF3F002F0E8F889
:1034200004460028EFD10F2DEDD8024629464FF073
:10343000FF3002F089F8034B20461D60E4E700BF2F
:10344000BC0A0020C00A002010B5032002F06AF870
:1034500001F0B8FC064B18600F20FFF7CFFF0446C1
:1034600018B914F08DFE204610BD0124FBE700BF03
:10347000A80B0020034A044B11681B780B4413600F
:10348000704700BF205A0020BC0A0020014B18687A
:10349000704700BF205A002038B50446FFF7F6FFFA
:1034A000631C1CBF054B1B78054618BFE418FFF7CB
:1034B000EDFF431BA342FAD338BD00BFBC0A002076
:1034C0004FF0E022136923F00203136170474FF0BD
:1034D000E022136943F00203136170478068C0F370
:1034E00080007047F7B5002301930446002800F0E0
:1034F0001181856D25B9F5F7EDF9E56584F854502E
:1035000022689368D90040F1B48020688368DA00AB
:1035100000F1C680A36D43F01003A365E36D43F093
:103520000103E3650122FFF7D9FFA36D03F0100348
:103530001843A36D40F0F08023F4817343F002033D
:103540002168A3658B68DB0700F1AC80CB68A568B8
:1035500023F018032B43CB60636803F04045E36C12
:1035600045EA030194F83C30012B08D1D4E9103628
:1035700033430B43A16C0B432B4343F001012568FC
:10358000674B2E6933400B432B61656825F0004380
:10359000B3F1804F0CD0B5F1004F09D0614ED6F891
:1035A000083705F4701523F470132B43C6F8083759
:1035B000637E257E266BA77E94F82CC0DB0343EA4E
:1035C0008533E5682B432569002E43EA473318BF4E
:1035D0004FF4805643EA4C03002DB4BF25F000455C
:1035E0004FF4001533432B4394F82050012D03D1A1
:1035F000002F59D143F48033656A25B1A66A05F4DA
:10360000E07535432B432668F56825F4FE3525F42F
:10361000F3751D43F5602668434D37693D402943E6
:1036200031612568666B696921F007013143696181
:103630002568A66B696921F0700141EA061169618C
:103640002169002939D12068816A61F00F01816206
:103650002168C86835490140994251D10023E3658A
:10366000A36D23F0030343F00103A365104603B0E9
:10367000F0BD936823F0104323F0170343F0805309
:1036800093602B4B2B4A1B68B3FBF2F301335B00B7
:103690000193019B002B3FF438AF019B013BF7E7FF
:1036A000002240E7014683E7A56D45F02005A565AA
:1036B000E56D45F00105E5659EE7B1F5001FC7D151
:1036C000266E850026FA05F505F00F050F2D0FD0A3
:1036D00001300828F5D12568A96AE1690139890016
:1036E00001F01C016FF00F0000FA01F1314305E019
:1036F00001282568EFD1A96A61F00F01A962A7E747
:10370000A36D23F0120343F01003A365E36D43F0B0
:103710000103E3650122A9E743F01003A365F9E77C
:1037200002FCFF1F0020014002FCFFDFE7FF3F8398
:10373000A80B0020400D0300F8B54569082D04468C
:103740000E460AD00368DB68D90705D5836D43F0C0
:10375000200383650120F8BD0425FFF797FE074687
:10376000206803682B4222D0A36D43F40073A36545
:10377000C36813F4406F14D1A37E93B903681B0789
:103780000FD5FFF7ABFE38BB2268536823F00C035C
:103790005360A36D23F4807323F0010343F001030E
:1037A000A365207E08BB23680C221A60D3E7721C35
:1037B000D7D0FFF76BFEC01BB04201D8002ECFD18F
:1037C00023681B682B40CBD1A26D84F8543042F0A3
:1037D0000402A2650320BEE7A36D43F02003A365A6
:1037E000E36D43F00103E365DBE70020B3E7036823
:1037F000186C7047F7B50023019390F85430012BF3
:10380000024600F0CC80012380F854300068FFF7B6
:1038100065FE002840F0BD80486815690B680228E5
:1038200025F0040500F08780B5F1004F1468C3F35C
:10383000110715D1A36A3B43A3620D6814688B6816
:10384000606903EA052323F07C4320EA052023F086
:10385000FF03034363610868002828DB002057E06A
:103860000F2500F01F0005FA00F6156E25EA060583
:10387000C7B9C3F3846383402B4313664868D56993
:1038800083080133AB42D8D80B68A56A00F01F004B
:10389000C3F383630F26834006FA00F025EA000095
:1038A0000343C9E793FAA3F3B3FA83F3E3E73D498C
:1038B0003D4DD1F80837A84203F0E07419D11B023E
:1038C000CCD4D1F8083723F0E073234343F400034A
:1038D000C1F80837354B36491B68B3FBF1F10C23AF
:1038E00001FB03330193019B002BB7D0019B013BEC
:1038F000F8E7304DA84210D113F08070AED1D1F866
:10390000083723F0E073234343F08073C1F808378E
:10391000002382F8543003B0F0BD274DA8429DD15A
:1039200013F480009AD1D1F8083723F0E0732343D1
:1039300043F48003EAE7B5F1004F06D11468A06AAA
:10394000C3F3110320EA0303A3620868002885DAA1
:10395000154C1449A042D1F8083709D1D1F808070D
:1039600003F0A07320F0E0700343C1F8083775E757
:10397000104CA04204D1D1F8080703F44003F1E74A
:103980000D4CA0427FF46AAFD1F8080703F0C07372
:10399000E8E7916D41F0200191651846B8E70220F3
:1039A000B9E700BF00200140001000B0A80B0020C4
:1039B000400D0300004000B8002000B438B50446B4
:1039C0000068FFF78BFD08B9002038BD22689368B6
:1039D000990707D4936823F0004323F0170343F0BB
:1039E00010039360FFF752FD054623689B685B0751
:1039F000EAD5FFF74BFD401B0228F6D923689B68E8
:103A00005A07F2D5A36D43F01003A365E36D43F0AD
:103A10000103E3650120D8E773B500230268019331
:103A20009368DD07044602D5002002B070BD91689E
:103A3000214B194209D0A36D43F01003A365E36D38
:103A400043F00103E3650120EFE7936823F00043AF
:103A500023F0170343F001039360184BD3F80837A2
:103A600018021CD4637E012BDED0FFF70FFD144E2D
:103A7000054622681368DB07D6D49368D9075FBF71
:103A80009368334043F001039360FFF7FFFC401B52
:103A90000228EED923681B68DA07EAD4CBE7094B82
:103AA000094A1B68B3FBF2F301330193019B002B1E
:103AB000D8D0019B013BF8E71700008000200140AF
:103AC000E8FFFF7FA80B0020400D030038B5044637
:103AD0000068FFF703FD054628BB94F85430012B1E
:103AE00021D0012384F854302046FFF795FFB8B960
:103AF000A36D23F4706323F0010343F48073A36583
:103B00002368E0651C221A60226884F854009368D8
:103B100023F0004323F0170343F00403936038BD00
:103B200084F85450FBE70220F9E738B5026893683F
:103B300091680446C80701D4002038BD9907FBD41A
:103B4000936803F00503012B1AD1936823F0004317
:103B500023F0170343F002039360236803221A60E3
:103B6000FFF794FC054623689B68DB07E4D5FFF765
:103B70008DFC401B0228F6D923689B68DA07F2D532
:103B8000A36D43F01003A365E36D43F00103E36508
:103B90000120D2E770B50446002849D0836D43F078
:103BA00002038365FFF70AFF054668B92046FFF761
:103BB000BCFF054608B90123A3652268936823F07A
:103BC000104323F0170393602268536823F467734C
:103BD00023F003035360236840F29F321A60226887
:103BE000144BD1680B40D3602268136923F0404323
:103BF00013612268536923F0070353612268136A33
:103C000003F0F0231362236800269A6A0A4A9E6230
:103C1000D2F8083723F0FE73C2F808372046F4F7CD
:103C200025FFE6652666A66584F85460284670BDC3
:103C30000125FBE700023E830020014010B590F80B
:103C40005430012B044615D0012380F85430FFF77F
:103C5000B5FE58B92046FFF768FF38B9A36D23F4C5
:103C6000807323F0010343F00103A365002384F86C
:103C7000543010BD0220FCE713B50023019390F8E7
:103C80005430012B044642D0012380F85430FFF712
:103C90004CFF2268936813F0010FA36D34D123F415
:103CA000817343F00203A365D168D36823F0030353
:103CB000D3602268936843F000439360236801F067
:103CC00003019A68002A12DA019A01320192019ADC
:103CD000B2F52E3FF5D3A36D23F0120343F010038A
:103CE000A365002384F85430012002B010BDDA68C7
:103CF0000A43DA60A36D23F0030343F00103A365D5
:103D0000002384F85430F0E743F01003F7E7022073
:103D1000EBE7026852E8003F23F0C00342E80031BD
:103D20000029F6D1026802F1080353E8003F23F4AA
:103D30000003083242E800310029F3D12023C0F803
:103D40008430704710B5026852E8003F23F4907346
:103D500042E800310029F6D10F4C026802F1080355
:103D600053E8003F2340083242E800310029F4D1F3
:103D7000C36E012B08D1026852E8003F23F0100304
:103D800042E800310029F6D12023C0F88830002312
:103D9000C366036710BD00BFFEFFFFEF38B50446E2
:103DA000D8B102682423C0F88430136823F00103DB
:103DB0001360036800251D6003685D6003689D60F3
:103DC00014F0B8FAC4F88C5084F88050C4F88450C9
:103DD0002846C4F88850E56638BD0120FCE738B5B0
:103DE0000268D0F88430D0F88850926812060446F1
:103DF0001FD5212B1DD1226802F1080353E8003F93
:103E000023F08003083242E800310029F3D1A06F8B
:103E100060B101F0A3FD48B1A06F01F074FE20284D
:103E200004D11023C4F88C30032038BD2046FFF79E
:103E300070FF2368986810F04000F6D0222D18D14A
:103E4000226802F1080353E8003F23F040030832E0
:103E500042E800310029F3D1E06F38B101F07EFD76
:103E600020B1E06F01F04FFE2028DAD02046FFF7A6
:103E700069FF0020D9E770477047704710B5806A26
:103E80000268D0F88430D0F888409268120606D5CF
:103E9000212B04D10023A0F85630FFF73AFF036826
:103EA0009B685B0606D5222C04D10023A0F85E3067
:103EB000FFF748FFD0F88C3043F01003C0F88C3087
:103EC000FFF7DBFF10BD08B5806A0023A0F85E3065
:103ED000A0F85630FFF7D1FF08BD70472DE9F0413B
:103EE0000568EB692A68A96840F60F063342044664
:103EF00010D19E0640F19A8002F0200601F0805712
:103F00003E4300F09380036F002B00F08880BDE8F3
:103F1000F0411847A34EA4480E401040304300F033
:103F20008580D80709D5D70507D501202862D4F8A0
:103F30008C0040F00100C4F88C0098070AD5CF0728
:103F400008D5206802250562D4F88C0040F00400F2
:103F5000C4F88C005D070AD5C80708D52068042579
:103F60000562D4F88C0040F00200C4F88C001F07F2
:103F70000BD502F02000304307D0206808250562E9
:103F8000D4F88C002843C4F88C001D050BD55001D3
:103F900009D520684FF400650562D4F88C0040F024
:103FA0002000C4F88C00D4F88C00002837D09B0681
:103FB0000AD502F0200201F0805152EA010303D039
:103FC000236F0BB1204698472368D4F88C509B6828
:103FD00005F0280503F040031D43204621D0FFF7DC
:103FE000B1FE23689B685F0616D5226802F10803BC
:103FF00053E8003F23F04003083242E80031002933
:10400000F3D1E36F43B1694A9A63E06F01F0DCFCDE
:1040100028B1E06F836B7AE72046FFF72EFFBDE8FB
:10402000F081FFF72AFFC4F88C50F8E7E06E012812
:1040300040F08980DE0640F18680D00640F1838022
:1040400010232B6223689B685B064AD5E26F1368D6
:104050005B689BB2002BE2D0B4F85C109942DED9C9
:10406000A4F85E3013681B689F0630D4226852E8BB
:10407000003F23F4807342E800310029F6D1226822
:1040800002F1080353E8003F23F00103083242E83D
:1040900000310029F3D1216801F1080353E8003F02
:1040A00023F04003083141E80032002AF3D12023F5
:1040B000C4F88830E266226852E8003F23F010031B
:1040C00042E800310029F6D1E06F01F047FCB4F876
:1040D0005E30B4F85C10C91A89B22046FFF7FDFEC5
:1040E0009DE7B4F85E10B4F85E2092B28BB2002A5D
:1040F00095D0B4F85C10C91A89B200298FD0226813
:1041000052E8003F23F4907342E800300028F6D1D3
:10411000274D206800F1080353E8003F2B4008308A
:1041200040E80032002AF4D12023C4F88830226706
:10413000E266226852E8003F23F0100342E80030B4
:104140000028F6D1C9E7DE0209D5480207D54FF4A9
:1041500080132B622046BDE8F041F4F747B81F06F4
:104160000BD502F0800001F40001014305D0636F1C
:10417000002B3FF454AF2046C9E65E061AD555061B
:1041800018D5216851E8003F23F0400341E8003290
:10419000002AF6D12023C4F8843062672046FFF756
:1041A0006AFE3CE70100001020010004C73E010840
:1041B000FEFFFFEF180206D5510004D52046BDE8EA
:1041C000F04100F024BCDB017FF529AF002ABFF6E7
:1041D00026AF2046BDE8F04100F018BC08B5806A63
:1041E000C36E012B05D1B0F85C104908FFF775FECE
:1041F00008BDFFF741FEFBE708B50346806A1B6870
:104200001B6813F0200331D1A0F85E30026852E839
:10421000003F23F4807342E800310029F6D10268A0
:1042200002F1080353E8003F23F00103083242E89B
:1042300000310029F3D1026802F1080353E8003F7E
:1042400023F04003083242E800310029F3D1202353
:10425000C0F88830C36E012B08D1026852E8003FD5
:1042600023F0100342E800310029F6D1C36E012B80
:1042700004D1B0F85C10FFF730FE08BDF3F7FEFE86
:10428000FBE790F88030012B1ED0012380F88030AE
:104290002423C0F88430026852E8003F23F00C0366
:1042A00042E800310029F6D1016851E8002F42F0C0
:1042B000080241E80023002BF6D12022C0F8842018
:1042C00080F88030184670470220704790F88030A0
:1042D000012B1ED0012380F880302423C0F88430C5
:1042E000026852E8003F23F00C0342E80031002945
:1042F000F6D1016851E8002F42F0040241E80023A2
:10430000002BF6D12022C0F8842080F88030184697
:10431000704702207047000038B5044601682269E2
:10432000A3680868134362691343E2691343814A2F
:10433000024013430B602268E168536823F4405342
:104340000B43536022687C4BA1699A421CBF236ACD
:104350001943936823F06E4323F430630B43936057
:104360002268616AD36A23F00F030B43D362236888
:10437000724A93421CD14FF0B043D3F8883003F017
:10438000030343F44033A3F54033013B022B6BD8C6
:104390006B4A9B5CE069B0F5004F40F09180082BC0
:1043A00024D8DFE803F065858B2388232323690065
:1043B000644A934209D14FF0B043634AD3F888303E
:1043C00003F00C0343F44023E3E75B4A93424DD1EF
:1043D0004FF0B043D3F8883003F44063B3F5006F77
:1043E0001AD005D853B1B3F5806F12D0012009E07F
:1043F000B3F5406FFAD14FF400400EE001F072F8CF
:1044000058B900204FF00113A3660023C4E91C3300
:1044100038BD00F069FCF3E74C4865684C4B626AB4
:1044200005EB450133F81220B0FBF2F39942DDD8D9
:10443000B3EB053FDAD800231946F2F7C1FE0902B3
:1044400041EA10616B080002C0182A464FF00003D1
:1044500041F10001F2F7B4FE3E4BA0F540729A42E2
:10446000C4D82368D860CCE7012393E7102391E7F1
:1044700001F038F80028C4D06268616A344B33F820
:104480001130B0FBF3F0530803EB4000B0FBF2F047
:1044900083B2A3F110014FF6EF729142A6D820F03B
:1044A0000F00226880B2C3F342031843D060A8E72C
:1044B00001F028F8DEE700F017FCDBE72348DBE734
:1044C000082B93D801A252F823F000BF174501082A
:1044D000234501082F450108ED430108294501083E
:1044E000ED430108ED430108ED430108F1440108E3
:1044F0004FF400406368616A154A32F81120B0FB3E
:10450000F2F000EB5300B0FBF3F080B2A0F1100228
:104510004FF6EF73A3E700F0E5FF00283FF471AF1B
:10452000E8E700F0EFFFF8E700F0DEFBF5E707480B
:10453000E0E700BFF369FFCF008000400038014092
:10454000B5FF020800440040B8FFF6070024F4005D
:10455000C6FF0208FFFC0F00836ADA0706D502686F
:10456000C16A536823F400330B435360836A9B078B
:1045700006D50268016B536823F480330B43536004
:10458000836A590706D50268416B536823F4802378
:104590000B435360836A1A0706D50268816B536820
:1045A00023F400430B435360836ADB0606D502689D
:1045B000C16B936823F480530B439360836A99061D
:1045C00006D50268016C936823F400530B43936093
:1045D000836A5A0611D50268416C536823F480132C
:1045E0000B435360436CB3F5801F06D10268816CA6
:1045F000536823F4C0030B435360836A1B0606D53C
:104600000268C16C536823F400230B435360704766
:104610002DE9F041DDF8188004460E4615461F4688
:104620002268D36936EA03030CBF01230023AB429F
:1046300001D0002028E0B8F1FF3FF2D0FEF726FFBE
:10464000C01B404503D82368B8F1000F1ED1226873
:1046500052E8003F23F4D07342E800310029F6D13C
:10466000216801F1080353E8003F23F001030831FA
:1046700041E80032002AF3D12023C4F88430C4F882
:10468000883084F880200320BDE8F0811A68510743
:10469000C6D5DA691205C3D54FF400621A622268E2
:1046A00052E8003F23F4D07342E800310029F6D1EC
:1046B000216801F1080353E8003F23F001030831AA
:1046C00041E80032002AF3D12023C4F88430C4F832
:1046D0008830C4F88C30D4E72DE9F7439846D0F8F9
:1046E0008430202B04460E4617464FD100294BD06C
:1046F000002A49D090F88030012B47D0012380F860
:10470000803000252123C0F88C50C0F88430FEF79B
:10471000BDFEA368A4F85470B3F5805F8146A4F889
:10472000567003D123690BB935461E46002384F821
:104730008030B4F85620CDF8008092B24B4642B992
:1047400040212046FFF764FF48B92023C4F8843095
:1047500006E0002280212046FFF75AFF18B103200F
:1047600003B0BDE8F08322685EB935F8023BC3F3BD
:1047700008039362B4F85620013A92B2A4F8562086
:10478000D7E716F8013BF4E70120E9E70220E7E765
:1047900073B504460026C0F88C60FEF777FE2368E8
:1047A0001B681A07054618D423681B685B070AD5DF
:1047B0006FF07E43009300222B464FF48001204689
:1047C000FFF726FFA8B920230020C4F8843084F81E
:1047D0008000C4F88830E0660CE06FF07E43009300
:1047E000324603464FF400112046FFF711FF002820
:1047F000DAD0032002B070BD10B5044660B3D0F823
:1048000084301BB980F8803013F0BCFC226824236C
:10481000C4F88430136823F0010313602046FFF7C7
:104820007BFD012818D0A36A13B12046FFF794FE40
:104830002268536823F4904353602268936823F0FE
:104840002A0393602268136843F001031360204633
:10485000BDE81040FFF79CBF012010BD10B5044615
:10486000002831D0D0F884301BB980F8803013F0A4
:1048700089FC22682423C4F88430136823F00103E0
:1048800013602046FFF748FD01281DD0A36A13B12D
:104890002046FFF761FE2268536823F4904353607B
:1048A0002268936823F0220393602268936843F0A0
:1048B000080393602268136843F0010313602046E5
:1048C000BDE81040FFF764BF012010BD38B51346A6
:1048D000A0F85C2000252222C0F88C50C0F8882067
:1048E000C26F81650446D2B11F49D162C26F1F49B0
:1048F0001163C26F1E495163C26F95630168826D77
:10490000C06F243100F0E2FF48B11023C4F88C30AE
:10491000202384F88050C4F88830012038BD00235B
:1049200084F88030226852E8003F43F4807342E804
:1049300000310029F6D1226802F1080353E8003F54
:1049400043F00103083242E800310029F3D1226824
:1049500002F1080353E8003F43F04003083242E805
:1049600000300028F3D1D9E7F9410108DD41010801
:104970007D3E010830B4D0F88830202B20D1E1B141
:10498000DAB190F88030012B1AD0012380F8803002
:1049900000230C4CC3660368A3420BD05B681B0268
:1049A00008D5046854E8003F43F0806344E80035CC
:1049B000002DF6D130BCFFF789BF012030BC704715
:1049C0000220FBE700800040436E30B51BB94FF07A
:1049D0000113836630BD03680A4D9A6899680A4CD2
:1049E000490FC2F342626B5C615CDB00B3FBF1F325
:1049F000A0F86A30AB5CA25CDB00B3FBF2F3A0F87A
:104A00006830E7E7E6FF0208DEFF020870477047FC
:104A10001FB504AB03E9060090F88030012B044673
:104A20000A463ED0012380F8803001682423C0F874
:104A300084300B6823F001030B6001688B6823F45A
:104A4000401313438B6082B92168BDF80C304A686B
:104A50009DF80E0022F010021A434A602268536843
:104A600023F07F4343EA006353602268136843F0F6
:104A700001031360FEF70AFD6FF07E4203460092C9
:104A80004FF4800100222046FFF7C2FD38B92023F1
:104A9000C4F88430002384F8803004B010BD0320B3
:104AA000F8E70220F9E790F88020012A03460ED0AB
